:040000000DEF00F010
:040008001BEF50F0AA
:0A001800FF0011EECFF17DEF5FF065
:10100000000200000100E652E652E652FB0E6F00BD
:101010008FFFE6FF6F008FFFE6FFCFEC62F0FE0E62
:101020006000BFF0E3FFFD0E6000BBF0E3FFFD0ECC
:101030006F008FFFF6FFFE0E6F008FFFF7FF000EB1
:10104000F86E0F0EF76403D00800F55007D06F005C
:10105000DBFFE9FF6F00DFFFEAFFEF50396EFF0EA5
:101060006000E7F0E3FFFB0E6F008FFFE6FF6F000D
:101070008FFFE6FF8FEC63F0FB0E6F008FFFE6FF44
:101080006F008FFFE6FF31EC62F0F80EE126FF0EF5
:10109000E22230EF0DF0FD0EE350010F386EFE0E30
:1010A0006F008CFF39F0000E39226000E3F0E6FF9C
:1010B0006000E7F0E6FF73EC54F0FB0E6F008FFF6B
:1010C000D9FFFC0E6F008FFFDAFFDF50140AD8A49F
:1010D0006CEF08F06EEF08F087EF08F0FD0E6F0080
:1010E0008FFFF6FFFE0E6F008FFFF7FF000EF86E0A
:1010F0000F0EF76404D0150EF56E0C0008D06F00CB
:10110000DBFFE9FF6F00DFFFEAFF150EEF6EFB0E5E
:101110006F008FFFD9FFFC0E6F008FFFDAFFDF50EB
:10112000150AD8A496EF08F098EF08F06FEF0DF0CD
:10113000FD0E6F008FFFF6FFFE0E6F008FFFF7FFB3
:10114000000EF86E0F0EF76404D0190EF56E0C0049
:1011500008D06F00DBFFE9FF6F00DFFFEAFF190E29
:10116000EF6E000EE66E000EE66E000EE66E000EEE
:10117000E66E000EE66E000EE66E000EE66E000EE7
:10118000E66EF50EE3501E0F386EF60E6F008CFF04
:1011900039F0000E39226000E3F0F6FF6000E7F05E
:1011A000F7FF000EF86E0F0EF76403D00800F5503D
:1011B00007D06F00DBFFE9FF6F00DFFFEAFFEF50B2
:1011C0000A0D6F00CCFF38F06F00D0FF39F06000DF
:1011D000E3F0E6FF6000E7F0E6FFF30E6F008FFF3D
:1011E000E6FF6F008FFFE6FFD3EC5EF06FEF0DF0D0
:1011F000FB0E6F008FFFD9FFFC0E6F008FFFDAFF31
:10120000DF50160AD8A407EF09F009EF09F06FEFD5
:101210000DF0FD0E6F008FFFF6FFFE0E6F008FFFCB
:10122000F7FF000EF86E0F0EF76404D0160EF56E81
:101230000C0008D06F00DBFFE9FF6F00DFFFEAFF63
:10124000160EEF6E6FEF0DF0FB0E6F008FFFD9FFE4
:10125000FC0E6F008FFFDAFFDF50170AD8A433EFC0
:1012600009F035EF09F06FEF0DF0FD0E6F008FFF05
:10127000F6FFFE0E6F008FFFF7FF000EF86E0F0EE9
:10128000F76404D0170EF56E0C0008D06F00DBFF7A
:10129000E9FF6F00DFFFEAFF170EEF6E000EE66E4C
:1012A000000EE66E000EE66E000EE66E000EE66EB6
:1012B000000EE66E000EE66E000EE66EF50EE350D2
:1012C0001E0F386EF60E6F008CFF39F0000E3922BB
:1012D0006000E3F0F6FF6000E7F0F7FF000EF86E45
:1012E0000F0EF76403D00800F55007D06F00DBFF46
:1012F000E9FF6F00DFFFEAFFEF50140D6F00CCFF36
:1013000038F06F00D0FF39F06000E3F0E6FF6000D6
:10131000E7F0E6FFF30E6F008FFFE6FF6F008FFF31
:10132000E6FFD3EC5EF06FEF0DF0FB0E6F008FFF6A
:10133000D9FFFC0E6F008FFFDAFFDF50180AD8A428
:10134000A4EF09F0A6EF09F06FEF0DF0FD0EE350EA
:101350001E0F386EFE0E6F008CFF39F0000E392222
:101360006000E3F0F6FF6000E7F0F7FF000EF86EB4
:101370000F0EF76403D00800F55007D06F00DBFFB5
:10138000E9FF6F00DFFFEAFFEF500009D8A4CBEFC1
:1013900009F0CDEF09F00FEF0AF0FD0EE3501D0F3D
:1013A000386EFE0E6F008CFF39F0000E392260009F
:1013B000E3F0F6FF6000E7F0F7FF000EF86E0F0EA7
:1013C000F76403D00800F55007D06F00DBFFE9FF9A
:1013D0006F00DFFFEAFFEF500009D8B4F2EF09F029
:1013E000F4EF09F0AFEF0AF0FD0E6F008FFFF6FF8C
:1013F000FE0E6F008FFFF7FF000EF86E0F0EF76402
:1014000004D01A0EF56E0C0008D06F00DBFFE9FF68
:101410006F00DFFFEAFF1A0EEF6EAFEF0AF0FD0E6E
:10142000E3501A0F386EFE0E6F008CFF39F0000E7D
:1014300039226000E3F0F6FF6000E7F0F7FF000EEE
:10144000F86E0F0EF76403D00800F55007D06F0058
:10145000DBFFE9FF6F00DFFFEAFFEF500009D8B4C0
:1014600034EF0AF036EF0AF096EF0AF0FD0E6F0047
:101470008FFFF6FFFE0E6F008FFFF7FF000EF86E76
:101480000F0EF76404D0170EF56E0C0008D06F0035
:10149000DBFFE9FF6F00DFFFEAFF170EEF6E000EC4
:1014A000E66E000EE66E000EE66E000EE66E000EB4
:1014B000E66E000EE66E000EE66E000EE66EF50EAF
:1014C000E3501E0F386EF60E6F008CFF39F0000EE1
:1014D00039226000E3F0F6FF6000E7F0F7FF000E4E
:1014E000F86E0F0EF76403D00800F55007D06F00B8
:1014F000DBFFE9FF6F00DFFFEAFFEF50140D6F0025
:10150000CCFF38F06F00D0FF39F06000E3F0E6FF69
:101510006000E7F0E6FFF30E6F008FFFE6FF6F005D
:101520008FFFE6FFD3EC5EF0AFEF0AF0FD0E6F0029
:101530008FFFF6FFFE0E6F008FFFF7FF000EF86EB5
:101540000F0EF76404D0180EF56E0C0008D06F0073
:10155000DBFFE9FF6F00DFFFEAFF180EEF6EFD0E05
:10156000E3501A0F386EFE0E6F008CFF39F0000E3C
:1015700039226000E3F0F6FF6000E7F0F7FF000EAD
:10158000F86E0F0EF76404D0000EF56E0C0008D054
:101590006F00DBFFE9FF6F00DFFFEAFF000EEF6E79
:1015A0006FEF0DF0FB0E6F008FFFD9FFFC0E6F0089
:1015B0008FFFDAFFDF501A0AD8A4E1EF0AF0E3EF59
:1015C0000AF06FEF0DF0FD0E6F008FFFF6FFFE0EBD
:1015D0006F008FFFF7FF000EF86E0F0EF76404D058
:1015E000150EF56E0C0008D06F00DBFFE9FF6F00F1
:1015F000DFFFEAFF150EEF6E6FEF0DF0FB0E6F00D1
:101600008FFFD9FFFC0E6F008FFFDAFFDF50180A43
:10161000D8A40DEF0BF00FEF0BF06FEF0DF0FD0EF8
:10162000E3502F0F386EFE0E6F008CFF39F0000E66
:1016300039226000E3F0F6FF6000E7F0F7FF000EEC
:10164000F86E0F0EF76409D009006F00D4FF38F070
:1016500009006F00D4FF39F00CD06F00DBFFE9FF09
:101660006F00DFFFEAFF6F00B8FF38F06F00B8FFD0
:1016700039F038503910D8B440EF0BF042EF0BF08E
:10168000A8EF0BF0FD0EE350310F386EFE0E6F0029
:101690008CFF39F0000E39226000E3F0F6FF6000A5
:1016A000E7F0F7FF000EF86E0F0EF76409D009009F
:1016B0006F00D4FF38F009006F00D4FF39F00CD070
:1016C0006F00DBFFE9FF6F00DFFFEAFF6F00B8FF8D
:1016D00038F06F00B8FF39F06000E3F0E6FF60001B
:1016E000E7F0E6FFFB0EE3502F0F386EFC0E6F00A5
:1016F0008CFF39F0000E39226000E3F0F6FF600045
:10170000E7F0F7FF000EF86E0F0EF76409D009003E
:101710006F00D4FF38F009006F00D4FF39F00CD00F
:101720006F00DBFFE9FF6F00DFFFEAFF6F00B8FF2C
:1017300038F06F00B8FF39F002D8A8EF0BF00500C1
:10174000FA6E3850FD6E3950FE6EFF6AFA50120084
:10175000FD0EE3501E0F386EFE0E6F008CFF39F049
:10176000000E39226000E3F0F6FF6000E7F0F7FFBB
:10177000000EF86E0F0EF76403D00800F55007D086
:101780006F00DBFFE9FF6F00DFFFEAFFEF500009AA
:10179000D8A4CDEF0BF0CFEF0BF011EF0CF0FD0E56
:1017A000E3501D0F386EFE0E6F008CFF39F0000EF7
:1017B00039226000E3F0F6FF6000E7F0F7FF000E6B
:1017C000F86E0F0EF76403D00800F55007D06F00D5
:1017D000DBFFE9FF6F00DFFFEAFFEF500009D8B43D
:1017E000F4EF0BF0F6EF0BF06FEF0DF0FD0E6F0066
:1017F0008FFFF6FFFE0E6F008FFFF7FF000EF86EF3
:101800000F0EF76404D01A0EF56E0C0008D06F00AE
:10181000DBFFE9FF6F00DFFFEAFF1A0EEF6E6FEFED
:101820000DF0000EE66E000EE66E000EE66E000E87
:10183000E66E000EE66E000EE66E000EE66E000E20
:10184000E66EF50EE3501E0F386EF60E6F008CFF3D
:1018500039F0000E39226000E3F0F6FF6000E7F097
:10186000F7FF000EF86E0F0EF76403D00800F55076
:1018700007D06F00DBFFE9FF6F00DFFFEAFFEF50EB
:10188000140D6F00CCFF38F06F00D0FF39F060000E
:10189000E3F0E6FF6000E7F0E6FFF30E6F008FFF76
:1018A000E6FF6F008FFFE6FFD3EC5EF06FEF0DF009
:1018B000FB0E6F008FFFD9FFFC0E6F008FFFDAFF6A
:1018C000DF50190AD8A467EF0CF069EF0CF06FEF46
:1018D0000DF0000EE66E000EE66E000EE66E000ED7
:1018E000E66E000EE66E000EE66E000EE66E000E70
:1018F000E66EF50EE3501E0F386EF60E6F008CFF8D
:1019000039F0000E39226000E3F0F6FF6000E7F0E6
:10191000F7FF000EF86E0F0EF76403D00800F550C5
:1019200007D06F00DBFFE9FF6F00DFFFEAFFEF503A
:101930000A0D6F00CCFF38F06F00D0FF39F0600067
:10194000E3F0E6FF6000E7F0E6FFF30E6F008FFFC5
:10195000E6FF6F008FFFE6FFD3EC5EF0FD0EE35075
:101960001B0F386EFE0E6F008CFF39F0000E39220F
:101970006000E3F0F6FF6000E7F0F7FF000EF86E9E
:101980000F0EF76403D00800F55007D06F00DBFF9F
:10199000E9FF6F00DFFFEAFFEF500009D8B4D3EF93
:1019A0000CF0D5EF0CF0EEEF0CF0FD0E6F008FFF9A
:1019B000F6FFFE0E6F008FFFF7FF000EF86E0F0EA2
:1019C000F76404D0170EF56E0C0008D06F00DBFF33
:1019D000E9FF6F00DFFFEAFF170EEF6EFD0EE35029
:1019E0001C0F386EFE0E6F008CFF39F0000E39228E
:1019F0006000E3F0F6FF6000E7F0F7FF000EF86E1E
:101A00000F0EF76403D00800F55007D06F00DBFF1E
:101A1000E9FF6F00DFFFEAFFEF500009D8B413EFD2
:101A20000DF015EF0DF06FEF0DF0FD0E6F008FFF55
:101A3000F6FFFE0E6F008FFFF7FF000EF86E0F0E21
:101A4000F76404D0190EF56E0C0008D06F00DBFFB0
:101A5000E9FF6F00DFFFEAFF190EEF6E6FEF0DF089
:101A6000FD0E6F008FFFF6FFFE0E6F008FFFF7FF7A
:101A7000000EF86E0F0EF76403D00800F55007D083
:101A80006F00DBFFE9FF6F00DFFFEAFFEF50386E0A
:101A9000396A3950000AD8B450EF0DF06FEF0DF0ED
:101AA0003850140AD8B44BEF08F0010AD8B4F8EF54
:101AB00008F0030AD8B424EF09F0010AD8B495EF6E
:101AC00009F00F0AD8B4D2EF0AF0010AD8B4FEEF39
:101AD0000AF0030AD8B458EF0CF06FEF0DF0FF0EC8
:101AE0006F008CFF39F0FD0E6F008FFFF6FFFE0ECA
:101AF0006F008FFFF7FF000EF86E0F0EF76403D034
:101B00000800F55007D06F00DBFFE9FF6F00DFFF33
:101B1000EAFFEF503918D8B490EF0DF092EF0DF0C6
:101B2000C0EF11F0BCEF0DF0FD0EE350020F386E68
:101B3000FE0E6F008CFF39F0000E39226000E3F0DA
:101B4000E6FF6000E7F0E6FFEAEC60F081EF11F0FD
:101B5000FD0EE350020F386EFE0E6F008CFF39F061
:101B6000000E39226000E3F0E6FF6000E7F0E6FFD8
:101B7000EAEC60F081EF11F0FF0EE350386E396A45
:101B80003950000AD8B4C7EF0DF081EF11F038508A
:101B9000140AD8B481EF11F0010AD8B481EF11F022
:101BA000030AD8B481EF11F0010AD8B494EF0DF014
:101BB0000F0AD8B481EF11F0010AD8B4A8EF0DF0E4
:101BC000030AD8B481EF11F081EF11F0FD0EE3505C
:101BD0001B0F386EFE0E6F008CFF39F0000E39229D
:101BE0006000E3F0F6FF6000E7F0F7FF000EF86E2C
:101BF0000F0EF76404D0010EF56E0C0008D06F00D4
:101C0000DBFFE9FF6F00DFFFEAFF010EEF6EFD0E65
:101C1000E3501F0F386EFE0E6F008CFF39F0000E80
:101C200039226000E3F0F6FF6000E7F0F7FF000EF6
:101C3000F86E0F0EF76409D009006F00D4FF38F07A
:101C400009006F00D4FF39F00CD06F00DBFFE9FF13
:101C50006F00DFFFEAFF6F00B8FF38F06F00B8FFDA
:101C600039F038503910D8B438EF0EF03AEF0EF0A2
:101C7000C0EF11F0FD0EE350210F386EFE0E6F0025
:101C80008CFF39F0000E39226000E3F0F6FF6000AF
:101C9000E7F0F7FF000EF86E0F0EF76409D00900A9
:101CA0006F00D4FF38F009006F00D4FF39F00CD07A
:101CB0006F00DBFFE9FF6F00DFFFEAFF6F00B8FF97
:101CC00038F06F00B8FF39F06000E3F0E6FF600025
:101CD000E7F0E6FFFB0EE3501F0F386EFC0E6F00BF
:101CE0008CFF39F0000E39226000E3F0F6FF60004F
:101CF000E7F0F7FF000EF86E0F0EF76409D0090049
:101D00006F00D4FF38F009006F00D4FF39F00CD019
:101D10006F00DBFFE9FF6F00DFFFEAFF6F00B8FF36
:101D200038F06F00B8FF39F002D8A0EF0EF00500D0
:101D3000FA6E3850FD6E3950FE6EFF6AFA5012008E
:101D4000C0EF11F0FD0EE350230F386EFE0E6F0052
:101D50008CFF39F0000E39226000E3F0F6FF6000DE
:101D6000E7F0F7FF000EF86E0F0EF76409D00900D8
:101D70006F00D4FF38F009006F00D4FF39F00CD0A9
:101D80006F00DBFFE9FF6F00DFFFEAFF6F00B8FFC6
:101D900038F06F00B8FF39F038503910D8B4D3EFAD
:101DA0000EF0D5EF0EF0C0EF11F0FD0EE350250F51
:101DB000386EFE0E6F008CFF39F0000E3922600085
:101DC000E3F0F6FF6000E7F0F7FF000EF86E0F0E8D
:101DD000F76409D009006F00D4FF38F009006F00E4
:101DE000D4FF39F00CD06F00DBFFE9FF6F00DFFF9D
:101DF000EAFF6F00B8FF38F06F00B8FF39F06000FD
:101E0000E3F0E6FF6000E7F0E6FFFB0EE350230F90
:101E1000386EFC0E6F008CFF39F0000E3922600026
:101E2000E3F0F6FF6000E7F0F7FF000EF86E0F0E2C
:101E3000F76409D009006F00D4FF38F009006F0083
:101E4000D4FF39F00CD06F00DBFFE9FF6F00DFFF3C
:101E5000EAFF6F00B8FF38F06F00B8FF39F002D822
:101E60003BEF0FF00500FA6E3850FD6E3950FE6EF4
:101E7000FF6AFA501200C0EF11F0FD0EE350010F9F
:101E8000386EFE0E6F008CFF39F0000E39226000B4
:101E9000E3F0E6FF6000E7F0E6FFE7EC54F0000E49
:101EA000E66E000EE66EFB0EE350020F386EFC0E7F
:101EB0006F008CFF39F0000E39226000E3F0E6FF7E
:101EC0006000E7F0E6FFD3EC5FF0FD0EE350270F74
:101ED000386EFE0E6F008CFF39F0000E3922600064
:101EE000E3F0F6FF6000E7F0F7FF000EF86E0F0E6C
:101EF000F76409D009006F00D4FF38F009006F00C3
:101F0000D4FF39F00CD06F00DBFFE9FF6F00DFFF7B
:101F1000EAFF6F00B8FF38F06F00B8FF39F03850B3
:101F20003910D8B496EF0FF098EF0FF0C0EF11F022
:101F3000FD0EE350290F386EFE0E6F008CFF39F056
:101F4000000E39226000E3F0F6FF6000E7F0F7FFD3
:101F5000000EF86E0F0EF76409D009006F00D4FF71
:101F600038F009006F00D4FF39F00CD06F00DBFFB0
:101F7000E9FF6F00DFFFEAFF6F00B8FF38F06F0086
:101F8000B8FF39F06000E3F0E6FF6000E7F0E6FF3D
:101F9000FB0EE350270F386EFC0E6F008CFF39F0FC
:101FA000000E39226000E3F0F6FF6000E7F0F7FF73
:101FB000000EF86E0F0EF76409D009006F00D4FF11
:101FC00038F009006F00D4FF39F00CD06F00DBFF50
:101FD000E9FF6F00DFFFEAFF6F00B8FF38F06F0026
:101FE000B8FF39F002D8FEEF0FF00500FA6E385056
:101FF000FD6E3950FE6EFF6AFA501200C0EF11F00C
:10200000FD0EE3502B0F386EFE0E6F008CFF39F083
:10201000000E39226000E3F0F6FF6000E7F0F7FF02
:10202000000EF86E0F0EF76409D009006F00D4FFA0
:1020300038F009006F00D4FF39F00CD06F00DBFFDF
:10204000E9FF6F00DFFFEAFF6F00B8FF38F06F00B5
:10205000B8FF39F038503910D8B431EF10F033EF01
:1020600010F0C0EF11F0FD0EE3502D0F386EFE0E94
:102070006F008CFF39F0000E39226000E3F0F6FFAC
:102080006000E7F0F7FF000EF86E0F0EF76409D05E
:1020900009006F00D4FF38F009006F00D4FF39F059
:1020A0000CD06F00DBFFE9FF6F00DFFFEAFF6F007E
:1020B000B8FF38F06F00B8FF39F06000E3F0E6FFDA
:1020C0006000E7F0E6FFFB0EE3502B0F386EFC0ECE
:1020D0006F008CFF39F0000E39226000E3F0F6FF4C
:1020E0006000E7F0F7FF000EF86E0F0EF76409D0FE
:1020F00009006F00D4FF38F009006F00D4FF39F0F9
:102100000CD06F00DBFFE9FF6F00DFFFEAFF6F001D
:10211000B8FF38F06F00B8FF39F002D899EF10F02F
:102120000500FA6E3850FD6E3950FE6EFF6AFA50A7
:102130001200C0EF11F0FD0EE350010F386EFE0EDD
:102140006F008CFF39F0000E39226000E3F0E6FFEB
:102150006000E7F0E6FFE7EC54F0000EE66E000EDC
:10216000E66EFB0EE350020F386EFC0E6F008CFF24
:1021700039F0000E39226000E3F0E6FF6000E7F07E
:10218000E6FFD3EC5FF0FD0EE3501C0F386EFE0E41
:102190006F008CFF39F0000E39226000E3F0F6FF8B
:1021A0006000E7F0F7FF000EF86E0F0EF76404D042
:1021B000010EF56E0C0008D06F00DBFFE9FF6F0029
:1021C000DFFFEAFF010EEF6EC0EF11F0FD0EE350EE
:1021D000330F386EFE0E6F008CFF39F0000E39227F
:1021E0006000E3F0F6FF6000E7F0F7FF000EF86E26
:1021F0000F0EF76409D009006F00D4FF38F0090012
:102200006F00D4FF39F00CD06F00DBFFE9FF6F00E7
:10221000DFFFEAFF6F00B8FF38F06F00B8FF39F05A
:1022200038503910D8B417EF11F019EF11F0C0EF92
:1022300011F0FD0EE350350F386EFE0E6F008CFF6F
:1022400039F0000E39226000E3F0F6FF6000E7F09D
:10225000F7FF000EF86E0F0EF76409D009006F004B
:10226000D4FF38F009006F00D4FF39F00CD06F00B4
:10227000DBFFE9FF6F00DFFFEAFF6F00B8FF38F018
:102280006F00B8FF39F06000E3F0E6FF6000E7F0B0
:10229000E6FFFB0EE350330F386EFC0E6F008CFF31
:1022A00039F0000E39226000E3F0F6FF6000E7F03D
:1022B000F7FF000EF86E0F0EF76409D009006F00EB
:1022C000D4FF38F009006F00D4FF39F00CD06F0054
:1022D000DBFFE9FF6F00DFFFEAFF6F00B8FF38F0B8
:1022E0006F00B8FF39F002D87FEF11F00500FA6EE9
:1022F0003850FD6E3950FE6EFF6AFA501200C0EF82
:1023000011F0FD0E6F008FFFF6FFFE0E6F008FFFC6
:10231000F7FF000EF86E0F0EF76403D00800F550BB
:1023200007D06F00DBFFE9FF6F00DFFFEAFFEF5030
:10233000386E396A3950000AD8B4A1EF11F0C0EFF5
:1023400011F03850140AD8B4C0EF11F0010AD8B413
:10235000E6EF0DF0030AD8B4A2EF0EF0010AD8B4EC
:102360003DEF0FF00F0AD8B400EF10F0010AD8B417
:102370009BEF10F0030AD8B4E6EF10F0C0EF11F0B5
:10238000FB0EE126FF0EE2221200E652E6526F003B
:102390003CFE39F00F0E3916FE0E6000E7F0E3FF49
:1023A000FF0E6F0047FEE3FFFE0EE350100F911289
:1023B00098EF1AF080AEDFEF11F0E1EF11F0C6EF09
:1023C0001AF082A6E6EF11F0E8EF11F018EF12F024
:1023D000FC0E6F008FFFD9FFFD0E6F008FFFDAFF3D
:1023E000020EDF6E8250E66E8150E66E8450E66E1D
:1023F0008350E66E2FEC49F0FC0E6F008CFF38F036
:10240000FD0E6F008CFF39F0010E3824D96E000EDE
:102410003920DA6E6000BBF0DEFF6000BFF0DEFF47
:102420006000C3F0DEFF6000C7F0DEFF42EF12F095
:10243000FC0E6F008FFFD9FFFD0E6F008FFFDAFFDC
:10244000010EDF6E8250E66E8150E66E5BEC55F059
:10245000FC0E6F008CFF38F0FD0E6F008CFF39F022
:10246000010E3824D96E000E3920DA6E6000BBF000
:10247000DEFF6000BFF0DEFF6000C3F0DEFF600043
:10248000C7F0DEFFFC0E6F008CFF38F0FD0E6F0012
:102490008CFF39F0050E3824D96E000E3920DA6E23
:1024A00085500F0BDF6EFC0E6F008CFF38F0FD0EB9
:1024B0006F008CFF39F00E0E3824D96E000E3920D3
:1024C000DA6E8544E846030BDF6EFC0E6F008CFF6E
:1024D00038F0FD0E6F008CFF39F0060E3824D96EEF
:1024E000000E3920DA6E6F001BFEDFFFFC0E6F005E
:1024F0008CFF38F0FD0E6F008CFF39F0070E38248A
:10250000D96E000E3920DA6E6F001FFEDFFFFC0E61
:102510006F008CFF38F0FD0E6F008CFF39F0080E55
:102520003824D96E000E3920DA6E6F0023FEDFFFEB
:10253000FC0E6F008CFF38F0FD0E6F008CFF39F041
:10254000090E3824D96E000E3920DA6E6F0027FE8E
:10255000DFFFFC0E6F008CFF38F0FD0E6F008CFF6C
:1025600039F00A0E3824D96E000E3920DA6E6F0069
:102570002BFEDFFFFC0E6F008CFF38F0FD0E6F00AE
:102580008CFF39F00B0E3824D96E000E3920DA6E2C
:102590006F002FFEDFFFFC0E6F008CFF38F0FD0E8A
:1025A0006F008CFF39F00C0E3824D96E000E3920E4
:1025B000DA6E6F0033FEDFFFFC0E6F008CFF38F029
:1025C000FD0E6F008CFF39F00D0E3824D96E000E11
:1025D0003920DA6E6F0037FEDFFF809EC6EF1AF0FB
:1025E0003701F0AFF6EF12F0F8EF12F0C6EF1AF085
:1025F00082A6FDEF12F0FFEF12F02FEF13F0FC0EAA
:102600006F008FFFD9FFFD0E6F008FFFDAFF020E04
:10261000DF6E8250E66E8150E66E8450E66E835027
:10262000E66E2FEC49F0FC0E6F008CFF38F0FD0ECB
:102630006F008CFF39F0010E3824D96E000E39205E
:10264000DA6E6000BBF0DEFF6000BFF0DEFF60000E
:10265000C3F0DEFF6000C7F0DEFF59EF13F0FC0EA1
:102660006F008FFFD9FFFD0E6F008FFFDAFF010EA5
:10267000DF6E8250E66E8150E66E5BEC55F0FC0E2C
:102680006F008CFF38F0FD0E6F008CFF39F0010EEB
:102690003824D96E000E3920DA6E6000BBF0DEFF00
:1026A0006000BFF0DEFF6000C3F0DEFF6000C7F037
:1026B000DEFFFC0E6F008CFF38F0FD0E6F008CFF0C
:1026C00039F0050E3824D96E000E3920DA6E8550A7
:1026D0000F0BDF6EFC0E6F008CFF38F0FD0E6F00ED
:1026E0008CFF39F00E0E3824D96E000E3920DA6EC8
:1026F0008544E846030BDF6EFC0E6F008CFF38F05C
:10270000FD0E6F008CFF39F0060E3824D96E000ED6
:102710003920DA6E6F001BFEDFFFFC0E6F008CFFAE
:1027200038F0FD0E6F008CFF39F0070E3824D96E9B
:10273000000E3920DA6E6F001FFEDFFFFC0E6F0007
:102740008CFF38F0FD0E6F008CFF39F0080E382436
:10275000D96E000E3920DA6E6F0023FEDFFFFC0E0B
:102760006F008CFF38F0FD0E6F008CFF39F0090E02
:102770003824D96E000E3920DA6E6F0027FEDFFF95
:10278000FC0E6F008CFF38F0FD0E6F008CFF39F0EF
:102790000A0E3824D96E000E3920DA6E6F002BFE37
:1027A000DFFFFC0E6F008CFF38F0FD0E6F008CFF1A
:1027B00039F00B0E3824D96E000E3920DA6E6F0016
:1027C0002FFEDFFFFC0E6F008CFF38F0FD0E6F0058
:1027D0008CFF39F00C0E3824D96E000E3920DA6ED9
:1027E0006F0033FEDFFFFC0E6F008CFF38F0FD0E34
:1027F0006F008CFF39F00D0E3824D96E000E392091
:10280000DA6E6F0037FEDFFF3701F09FEEEF12F058
:10281000370140AF0EEF14F010EF14F0C6EF1AF0CE
:1028200082A615EF14F017EF14F047EF14F0FC0E2A
:102830006F008FFFD9FFFD0E6F008FFFDAFF020ED2
:10284000DF6E8250E66E8150E66E8450E66E8350F5
:10285000E66E2FEC49F0FC0E6F008CFF38F0FD0E99
:102860006F008CFF39F0010E3824D96E000E39202C
:10287000DA6E6000BBF0DEFF6000BFF0DEFF6000DC
:10288000C3F0DEFF6000C7F0DEFF71EF14F0FC0E56
:102890006F008FFFD9FFFD0E6F008FFFDAFF010E73
:1028A000DF6E8250E66E8150E66E5BEC55F0FC0EFA
:1028B0006F008CFF38F0FD0E6F008CFF39F0010EB9
:1028C0003824D96E000E3920DA6E6000BBF0DEFFCE
:1028D0006000BFF0DEFF6000C3F0DEFF6000C7F005
:1028E000DEFFFC0E6F008CFF38F0FD0E6F008CFFDA
:1028F00039F0050E3824D96E000E3920DA6E855075
:102900000F0BDF6EFC0E6F008CFF38F0FD0E6F00BA
:102910008CFF39F00E0E3824D96E000E3920DA6E95
:102920008544E846030BDF6EFC0E6F008CFF38F029
:10293000FD0E6F008CFF39F0060E3824D96E000EA4
:102940003920DA6E6F001BFEDFFFFC0E6F008CFF7C
:1029500038F0FD0E6F008CFF39F0070E3824D96E69
:10296000000E3920DA6E6F001FFEDFFFFC0E6F00D5
:102970008CFF38F0FD0E6F008CFF39F0080E382404
:10298000D96E000E3920DA6E6F0023FEDFFFFC0ED9
:102990006F008CFF38F0FD0E6F008CFF39F0090ED0
:1029A0003824D96E000E3920DA6E6F0027FEDFFF63
:1029B000FC0E6F008CFF38F0FD0E6F008CFF39F0BD
:1029C0000A0E3824D96E000E3920DA6E6F002BFE05
:1029D000DFFFFC0E6F008CFF38F0FD0E6F008CFFE8
:1029E00039F00B0E3824D96E000E3920DA6E6F00E4
:1029F0002FFEDFFFFC0E6F008CFF38F0FD0E6F0026
:102A00008CFF39F00C0E3824D96E000E3920DA6EA6
:102A10006F0033FEDFFFFC0E6F008CFF38F0FD0E01
:102A20006F008CFF39F00D0E3824D96E000E39205E
:102A3000DA6E6F0037FEDFFF3701409FEEEF12F0D6
:102A4000370150AF26EF15F028EF15F0C6EF1AF05A
:102A500082A62DEF15F02FEF15F05FEF15F0FC0EAD
:102A60006F008FFFD9FFFD0E6F008FFFDAFF020EA0
:102A7000DF6E8250E66E8150E66E8450E66E8350C3
:102A8000E66E2FEC49F0FC0E6F008CFF38F0FD0E67
:102A90006F008CFF39F0010E3824D96E000E3920FA
:102AA000DA6E6000BBF0DEFF6000BFF0DEFF6000AA
:102AB000C3F0DEFF6000C7F0DEFF89EF15F0FC0E0B
:102AC0006F008FFFD9FFFD0E6F008FFFDAFF010E41
:102AD000DF6E8250E66E8150E66E5BEC55F0FC0EC8
:102AE0006F008CFF38F0FD0E6F008CFF39F0010E87
:102AF0003824D96E000E3920DA6E6000BBF0DEFF9C
:102B00006000BFF0DEFF6000C3F0DEFF6000C7F0D2
:102B1000DEFFFC0E6F008CFF38F0FD0E6F008CFFA7
:102B200039F0050E3824D96E000E3920DA6E855042
:102B30000F0BDF6EFC0E6F008CFF38F0FD0E6F0088
:102B40008CFF39F00E0E3824D96E000E3920DA6E63
:102B50008544E846030BDF6EFC0E6F008CFF38F0F7
:102B6000FD0E6F008CFF39F0060E3824D96E000E72
:102B70003920DA6E6F001BFEDFFFFC0E6F008CFF4A
:102B800038F0FD0E6F008CFF39F0070E3824D96E37
:102B9000000E3920DA6E6F001FFEDFFFFC0E6F00A3
:102BA0008CFF38F0FD0E6F008CFF39F0080E3824D2
:102BB000D96E000E3920DA6E6F0023FEDFFFFC0EA7
:102BC0006F008CFF38F0FD0E6F008CFF39F0090E9E
:102BD0003824D96E000E3920DA6E6F0027FEDFFF31
:102BE000FC0E6F008CFF38F0FD0E6F008CFF39F08B
:102BF0000A0E3824D96E000E3920DA6E6F002BFED3
:102C0000DFFFFC0E6F008CFF38F0FD0E6F008CFFB5
:102C100039F00B0E3824D96E000E3920DA6E6F00B1
:102C20002FFEDFFFFC0E6F008CFF38F0FD0E6F00F3
:102C30008CFF39F00C0E3824D96E000E3920DA6E74
:102C40006F0033FEDFFFFC0E6F008CFF38F0FD0ECF
:102C50006F008CFF39F00D0E3824D96E000E39202C
:102C6000DA6E6F0037FEDFFF3701509FEEEF12F094
:102C7000370160AF3EEF16F040EF16F0C6EF1AF0E6
:102C800082A645EF16F047EF16F077EF16F0FC0E30
:102C90006F008FFFD9FFFD0E6F008FFFDAFF020E6E
:102CA000DF6E8250E66E8150E66E8450E66E835091
:102CB000E66E2FEC49F0FC0E6F008CFF38F0FD0E35
:102CC0006F008CFF39F0010E3824D96E000E3920C8
:102CD000DA6E6000BBF0DEFF6000BFF0DEFF600078
:102CE000C3F0DEFF6000C7F0DEFFA1EF16F0FC0EC0
:102CF0006F008FFFD9FFFD0E6F008FFFDAFF010E0F
:102D0000DF6E8250E66E8150E66E5BEC55F0FC0E95
:102D10006F008CFF38F0FD0E6F008CFF39F0010E54
:102D20003824D96E000E3920DA6E6000BBF0DEFF69
:102D30006000BFF0DEFF6000C3F0DEFF6000C7F0A0
:102D4000DEFFFC0E6F008CFF38F0FD0E6F008CFF75
:102D500039F0050E3824D96E000E3920DA6E855010
:102D60000F0BDF6EFC0E6F008CFF38F0FD0E6F0056
:102D70008CFF39F00E0E3824D96E000E3920DA6E31
:102D80008544E846030BDF6EFC0E6F008CFF38F0C5
:102D9000FD0E6F008CFF39F0060E3824D96E000E40
:102DA0003920DA6E6F001BFEDFFFFC0E6F008CFF18
:102DB00038F0FD0E6F008CFF39F0070E3824D96E05
:102DC000000E3920DA6E6F001FFEDFFFFC0E6F0071
:102DD0008CFF38F0FD0E6F008CFF39F0080E3824A0
:102DE000D96E000E3920DA6E6F0023FEDFFFFC0E75
:102DF0006F008CFF38F0FD0E6F008CFF39F0090E6C
:102E00003824D96E000E3920DA6E6F0027FEDFFFFE
:102E1000FC0E6F008CFF38F0FD0E6F008CFF39F058
:102E20000A0E3824D96E000E3920DA6E6F002BFEA0
:102E3000DFFFFC0E6F008CFF38F0FD0E6F008CFF83
:102E400039F00B0E3824D96E000E3920DA6E6F007F
:102E50002FFEDFFFFC0E6F008CFF38F0FD0E6F00C1
:102E60008CFF39F00C0E3824D96E000E3920DA6E42
:102E70006F0033FEDFFFFC0E6F008CFF38F0FD0E9D
:102E80006F008CFF39F00D0E3824D96E000E3920FA
:102E9000DA6E6F0037FEDFFF3701609FEEEF12F052
:102EA000370170AF56EF17F058EF17F0C6EF1AF072
:102EB00082A65DEF17F05FEF17F08FEF17F0FC0EB3
:102EC0006F008FFFD9FFFD0E6F008FFFDAFF020E3C
:102ED000DF6E8250E66E8150E66E8450E66E83505F
:102EE000E66E2FEC49F0FC0E6F008CFF38F0FD0E03
:102EF0006F008CFF39F0010E3824D96E000E392096
:102F0000DA6E6000BBF0DEFF6000BFF0DEFF600045
:102F1000C3F0DEFF6000C7F0DEFFB9EF17F0FC0E74
:102F20006F008FFFD9FFFD0E6F008FFFDAFF010EDC
:102F3000DF6E8250E66E8150E66E5BEC55F0FC0E63
:102F40006F008CFF38F0FD0E6F008CFF39F0010E22
:102F50003824D96E000E3920DA6E6000BBF0DEFF37
:102F60006000BFF0DEFF6000C3F0DEFF6000C7F06E
:102F7000DEFFFC0E6F008CFF38F0FD0E6F008CFF43
:102F800039F0050E3824D96E000E3920DA6E8550DE
:102F90000F0BDF6EFC0E6F008CFF38F0FD0E6F0024
:102FA0008CFF39F00E0E3824D96E000E3920DA6EFF
:102FB0008544E846030BDF6EFC0E6F008CFF38F093
:102FC000FD0E6F008CFF39F0060E3824D96E000E0E
:102FD0003920DA6E6F001BFEDFFFFC0E6F008CFFE6
:102FE00038F0FD0E6F008CFF39F0070E3824D96ED3
:102FF000000E3920DA6E6F001FFEDFFFFC0E6F003F
:103000008CFF38F0FD0E6F008CFF39F0080E38246D
:10301000D96E000E3920DA6E6F0023FEDFFFFC0E42
:103020006F008CFF38F0FD0E6F008CFF39F0090E39
:103030003824D96E000E3920DA6E6F0027FEDFFFCC
:10304000FC0E6F008CFF38F0FD0E6F008CFF39F026
:103050000A0E3824D96E000E3920DA6E6F002BFE6E
:10306000DFFFFC0E6F008CFF38F0FD0E6F008CFF51
:1030700039F00B0E3824D96E000E3920DA6E6F004D
:103080002FFEDFFFFC0E6F008CFF38F0FD0E6F008F
:103090008CFF39F00C0E3824D96E000E3920DA6E10
:1030A0006F0033FEDFFFFC0E6F008CFF38F0FD0E6B
:1030B0006F008CFF39F00D0E3824D96E000E3920C8
:1030C000DA6E6F0037FEDFFF3701709FEEEF12F010
:1030D000370180AF6EEF18F070EF18F0C6EF1AF0FE
:1030E00082A675EF18F077EF18F0A7EF18F0FC0E36
:1030F0006F008FFFD9FFFD0E6F008FFFDAFF020E0A
:10310000DF6E8250E66E8150E66E8450E66E83502C
:10311000E66E2FEC49F0FC0E6F008CFF38F0FD0ED0
:103120006F008CFF39F0010E3824D96E000E392063
:10313000DA6E6000BBF0DEFF6000BFF0DEFF600013
:10314000C3F0DEFF6000C7F0DEFFD1EF18F0FC0E29
:103150006F008FFFD9FFFD0E6F008FFFDAFF010EAA
:10316000DF6E8250E66E8150E66E5BEC55F0FC0E31
:103170006F008CFF38F0FD0E6F008CFF39F0010EF0
:103180003824D96E000E3920DA6E6000BBF0DEFF05
:103190006000BFF0DEFF6000C3F0DEFF6000C7F03C
:1031A000DEFFFC0E6F008CFF38F0FD0E6F008CFF11
:1031B00039F0050E3824D96E000E3920DA6E8550AC
:1031C0000F0BDF6EFC0E6F008CFF38F0FD0E6F00F2
:1031D0008CFF39F00E0E3824D96E000E3920DA6ECD
:1031E0008544E846030BDF6EFC0E6F008CFF38F061
:1031F000FD0E6F008CFF39F0060E3824D96E000EDC
:103200003920DA6E6F001BFEDFFFFC0E6F008CFFB3
:1032100038F0FD0E6F008CFF39F0070E3824D96EA0
:10322000000E3920DA6E6F001FFEDFFFFC0E6F000C
:103230008CFF38F0FD0E6F008CFF39F0080E38243B
:10324000D96E000E3920DA6E6F0023FEDFFFFC0E10
:103250006F008CFF38F0FD0E6F008CFF39F0090E07
:103260003824D96E000E3920DA6E6F0027FEDFFF9A
:10327000FC0E6F008CFF38F0FD0E6F008CFF39F0F4
:103280000A0E3824D96E000E3920DA6E6F002BFE3C
:10329000DFFFFC0E6F008CFF38F0FD0E6F008CFF1F
:1032A00039F00B0E3824D96E000E3920DA6E6F001B
:1032B0002FFEDFFFFC0E6F008CFF38F0FD0E6F005D
:1032C0008CFF39F00C0E3824D96E000E3920DA6EDE
:1032D0006F0033FEDFFFFC0E6F008CFF38F0FD0E39
:1032E0006F008CFF39F00D0E3824D96E000E392096
:1032F000DA6E6F0037FEDFFF3701809FEEEF12F0CE
:10330000370190AF86EF19F088EF19F0C6EF1AF089
:1033100082A68DEF19F08FEF19F0BFEF19F0FC0EB8
:103320006F008FFFD9FFFD0E6F008FFFDAFF020ED7
:10333000DF6E8250E66E8150E66E8450E66E8350FA
:10334000E66E2FEC49F0FC0E6F008CFF38F0FD0E9E
:103350006F008CFF39F0010E3824D96E000E392031
:10336000DA6E6000BBF0DEFF6000BFF0DEFF6000E1
:10337000C3F0DEFF6000C7F0DEFFE9EF19F0FC0EDE
:103380006F008FFFD9FFFD0E6F008FFFDAFF010E78
:10339000DF6E8250E66E8150E66E5BEC55F0FC0EFF
:1033A0006F008CFF38F0FD0E6F008CFF39F0010EBE
:1033B0003824D96E000E3920DA6E6000BBF0DEFFD3
:1033C0006000BFF0DEFF6000C3F0DEFF6000C7F00A
:1033D000DEFFFC0E6F008CFF38F0FD0E6F008CFFDF
:1033E00039F0050E3824D96E000E3920DA6E85507A
:1033F0000F0BDF6EFC0E6F008CFF38F0FD0E6F00C0
:103400008CFF39F00E0E3824D96E000E3920DA6E9A
:103410008544E846030BDF6EFC0E6F008CFF38F02E
:10342000FD0E6F008CFF39F0060E3824D96E000EA9
:103430003920DA6E6F001BFEDFFFFC0E6F008CFF81
:1034400038F0FD0E6F008CFF39F0070E3824D96E6E
:10345000000E3920DA6E6F001FFEDFFFFC0E6F00DA
:103460008CFF38F0FD0E6F008CFF39F0080E382409
:10347000D96E000E3920DA6E6F0023FEDFFFFC0EDE
:103480006F008CFF38F0FD0E6F008CFF39F0090ED5
:103490003824D96E000E3920DA6E6F0027FEDFFF68
:1034A000FC0E6F008CFF38F0FD0E6F008CFF39F0C2
:1034B0000A0E3824D96E000E3920DA6E6F002BFE0A
:1034C000DFFFFC0E6F008CFF38F0FD0E6F008CFFED
:1034D00039F00B0E3824D96E000E3920DA6E6F00E9
:1034E0002FFEDFFFFC0E6F008CFF38F0FD0E6F002B
:1034F0008CFF39F00C0E3824D96E000E3920DA6EAC
:103500006F0033FEDFFFFC0E6F008CFF38F0FD0E06
:103510006F008CFF39F00D0E3824D96E000E392063
:10352000DA6E6F0037FEDFFF3701909FEEEF12F08B
:10353000FE0EE350386E396A3950000AD8B4A3EF52
:103540001AF0C6EF1AF03850000AD8B4DAEF11F0CA
:10355000010AD8B4F0EF12F0030AD8B408EF14F05F
:10356000010AD8B420EF15F0070AD8B438EF16F0E6
:10357000010AD8B450EF17F0030AD8B468EF18F076
:10358000010AD8B480EF19F0C6EF1AF0FF0E6F00F1
:103590008FFF91FFE552E552E552E5521200240EED
:1035A000E126000EE222DA0E6F008FFFE6FF6F00C9
:1035B0008FFFE6FFCFEC62F0FC0E6000BFF0E3FF90
:1035C000FB0E6000BBF0E3FFFB0E6F008FFFF6FF0A
:1035D000FC0E6F008FFFF7FF000EF86E0F0EF76402
:1035E00003D00800F55007D06F00DBFFE9FF6F0044
:1035F000DFFFEAFFEF50396EFF0E6000E7F0E3FFF8
:10360000DA0E6F008FFFE6FF6F008FFFE6FF8FEC93
:1036100063F0DA0E6F008FFFE6FF6F008FFFE6FFAB
:1036200031EC62F0E5526F009CFF45F0E5526F000F
:103630009CFF44F0E5526F009CFF43F0E5526F00A1
:103640009CFF42F0E5526F009CFF41F0E5526F0095
:103650009CFF40F0E5526F009CFF3FF0E5526F0089
:103660009CFF3EF0EB0E6000FBF0E3FFEC0E600011
:10367000FFF0E3FFED0E600003F1E3FFEE0E6000EC
:1036800007F1E3FFEF0E60000BF1E3FFF00E6000C7
:103690000FF1E3FFF10E600013F1E3FFF20E6000A3
:1036A00017F1E3FFEB0E6F008CFF36F0EC0E6F00AE
:1036B0008CFF37F0ED0E6F008CFF38F0EE0E6F00D0
:1036C0008CFF39F0F70E6000DBF0E3FFF80E6000CE
:1036D000DFF0E3FFF90E6000E3F0E3FFFA0E6000B5
:1036E000E7F0E3FF85EF22F0DA0E6F008FFFD9FFDE
:1036F000DB0E6F008FFFDAFFDF500A0AD8A483EFDA
:103700001BF085EF1BF0B0EF22F0FB0E6F008FFF78
:10371000F6FFFC0E6F008FFFF7FF000EF86E0F0E26
:10372000F76404D00B0EF56E0C0008D06F00DBFFC1
:10373000E9FF6F00DFFFEAFF0B0EEF6EB0EF22F044
:10374000DA0E6F008FFFD9FFDB0E6F008FFFDAFFFD
:10375000DF500B0AD8A4AFEF1BF0B1EF1BF0BFEFA7
:103760001CF0FB0EE350020F386EFC0E6F008CFF56
:1037700039F0000E39226000E3F0F6FF6000E7F058
:10378000F7FF000EF86E0F0EF76409D009006F0006
:10379000D4FF38F009006F00D4FF39F00CD06F006F
:1037A000DBFFE9FF6F00DFFFEAFF6F00B8FF38F0D3
:1037B0006F00B8FF39F038503910D8B4E2EF1BF081
:1037C000E4EF1BF0BFEF1CF0EF0EE124D96EFF0E0B
:1037D000E220DA6E6F0078FF36F06F0078FF37F086
:1037E0006F0078FF38F06F0078FF39F036503E6E8A
:1037F00037503F6E3850406E3950416E426A436ACE
:10380000446A456AEB0E6000FBF0E3FFEC0E6000DB
:10381000FFF0E3FFED0E600003F1E3FFEE0E60004A
:1038200007F1E3FFEF0E60000BF1E3FFF00E600025
:103830000FF1E3FFF10E600013F1E3FFF20E600001
:1038400017F1E3FFEB0E6F008CFF36F0EC0E6F000C
:103850008CFF37F0ED0E6F008CFF38F0EE0E6F002E
:103860008CFF39F0F30E6000DBF0E3FFF40E600034
:10387000DFF0E3FFF50E6000E3F0E3FFF60E60001B
:10388000E7F0E3FFF30E6F008CFF2EF0FD0E6000FB
:10389000BBF0E3FFE150FD0FD96EE250DA6EFF0E90
:1038A000DA22DF3A0F0EDF16FD0E6F008CFF2EF0CE
:1038B0000F0E2E16FD0E6000BBF0E3FFF40EE124A8
:1038C000D96EFF0EE220DA6EDF50396EFE0E600018
:1038D000E7F0E3FFE150FE0FD96EE250DA6EFF0E23
:1038E000DA22DF3A0F0EDF16F70E6F008FFFE6FFCA
:1038F0006F008FFFE6FF6F008FFFE6FF6F008FFF07
:10390000E6FF000EE66EF80EE350E66EF80EE350AA
:10391000E66EF40EE350020F386EF50E6F008CFF6A
:1039200039F0000E39226000E3F0F6FF6000E7F0A6
:10393000F7FF000EF86E0F0EF76409D009006F0054
:10394000D4FF38F009006F00D4FF39F00CD06F00BD
:10395000DBFFE9FF6F00DFFFEAFF6F00B8FF38F021
:103960006F00B8FF39F002D8BFEF1CF00500FA6E07
:103970003850FD6E3950FE6EFF6AFA501200DA0EB2
:103980006F008FFFD9FFDB0E6F008FFFDAFFDF5074
:103990000C0AD8A4CEEF1CF0D0EF1CF0DEEF1DF027
:1039A000FB0EE350020F386EFC0E6F008CFF39F0F7
:1039B000000E39226000E3F0F6FF6000E7F0F7FF49
:1039C000000EF86E0F0EF76409D009006F00D4FFE7
:1039D00038F009006F00D4FF39F00CD06F00DBFF26
:1039E000E9FF6F00DFFFEAFF6F00B8FF38F06F00FC
:1039F000B8FF39F038503910D8B401EF1DF003EF9B
:103A00001DF0DEEF1DF0EF0EE124D96EFF0EE22077
:103A1000DA6E6F0078FF36F06F0078FF37F06F00D6
:103A200078FF38F06F0078FF39F036503E6E37502F
:103A30003F6E3850406E3950416E426A436A446A64
:103A4000456AEB0E6000FBF0E3FFEC0E6000FFF058
:103A5000E3FFED0E600003F1E3FFEE0E600007F1FF
:103A6000E3FFEF0E60000BF1E3FFF00E60000FF1DB
:103A7000E3FFF10E600013F1E3FFF20E600017F1B7
:103A8000E3FFEB0E6F008CFF36F0EC0E6F008CFF47
:103A900037F0ED0E6F008CFF38F0EE0E6F008CFFEC
:103AA00039F0F30E6000DBF0E3FFF40E6000DFF0AE
:103AB000E3FFF50E6000E3F0E3FFF60E6000E7F0D1
:103AC000E3FFF30E6F008CFF2EF0FD0E6000BBF0E5
:103AD000E3FFE150FD0FD96EE250DA6EFF0EDA22FD
:103AE000DF3A0F0EDF16FD0E6F008CFF2EF00F0E6B
:103AF0002E16FD0E6000BBF0E3FFF40EE124D96E3C
:103B0000FF0EE220DA6EDF50396EFE0E6000E7F045
:103B1000E3FFE150FE0FD96EE250DA6EFF0EDA22BB
:103B2000DF3A0F0EDF16F70E6F008FFFE6FF6F0014
:103B30008FFFE6FF6F008FFFE6FF6F008FFFE6FF4E
:103B4000010EE66EF80EE350E66EF80EE350E66EF8
:103B5000F40EE350020F386EF50E6F008CFF39F053
:103B6000000E39226000E3F0F6FF6000E7F0F7FF97
:103B7000000EF86E0F0EF76409D009006F00D4FF35
:103B800038F009006F00D4FF39F00CD06F00DBFF74
:103B9000E9FF6F00DFFFEAFF6F00B8FF38F06F004A
:103BA000B8FF39F002D8DEEF1DF00500FA6E38508C
:103BB000FD6E3950FE6EFF6AFA501200DA0E6F0089
:103BC0008FFFD9FFDB0E6F008FFFDAFFDF500D0A8A
:103BD000D8A4EDEF1DF0EFEF1DF0CCEF1EF0DC0EE2
:103BE000E36AE32AE10EE124D96EFF0EE220DA6EE9
:103BF000040EDF6EEA0EE124D96EFF0EE220DA6ECB
:103C0000DF6AE20EE124D96EFF0EE220DA6EEB0EDF
:103C10006F008FFFDFFF080E396EE150EB0FD96E9A
:103C2000E250DA6EFF0EDA223928DE5227EF1EF05C
:103C3000DE52DE52DE52DE52DE52DE52D890DD32ED
:103C4000DD32DD32DD32DD32DD32DD32DE32E82EF4
:103C500018EF1EF0E30EE124D96EFF0EE220DA6EBB
:103C6000EB0E6F008FFFDFFF080E396EE150EB0F98
:103C7000D96EE250DA6EFF0EDA223928DE5250EFAA
:103C80001EF0DE52DE52DE52DE52DE52DE52D8909E
:103C9000DD32DD32DD32DD32DD32DD32DD32DE32AB
:103CA000E82E41EF1EF0E40EE124D96EFF0EE22073
:103CB000DA6EEB0E6F008FFFDFFF080E396EE150FA
:103CC000EB0FD96EE250DA6EFF0EDA223928DE529F
:103CD00079EF1EF0DE52DE52DE52DE52DE52DE524E
:103CE000D890DD32DD32DD32DD32DD32DD32DD3203
:103CF000DE32E82E6AEF1EF0E50EE124D96EFF0EEB
:103D0000E220DA6EEB0E6F008FFFDFFF080E396ED8
:103D1000E150EB0FD96EE250DA6EFF0EDA2239284D
:103D2000DE52A2EF1EF0DE52DE52DE52DE52DE52D4
:103D3000DE52D890DD32DD32DD32DD32DD32DD3291
:103D4000DD32DE32E82E93EF1EF0E150EB0FD96E3C
:103D5000E250DA6EFF0EDA22DD0EE124E96EFF0E8C
:103D6000E220EA6E6F007BFFEEFF6F007BFFEEFF4D
:103D70006F007BFFEEFF6F007BFFEEFFDC0EE124A8
:103D80002E6EFF0EE2202F6E6000BBF0E6FF60009B
:103D9000BFF0E6FFE5EC37F0DA0E6F008FFFD9FFDA
:103DA000DB0E6F008FFFDAFFDF500E0AD8A4DBEFC7
:103DB0001EF0DDEF1EF0BAEF1FF0DC0EE36AE32A1F
:103DC000E10EE124D96EFF0EE220DA6E020EDF6E04
:103DD000EA0EE124D96EFF0EE220DA6EDF6AE20E0F
:103DE000E124D96EFF0EE220DA6EEB0E6F008FFF3A
:103DF000DFFF080E396EE150EB0FD96EE250DA6E3C
:103E0000FF0EDA223928DE5215EF1FF0DE52DE52A5
:103E1000DE52DE52DE52DE52D890DD32DD32DD324D
:103E2000DD32DD32DD32DD32DE32E82E06EF1FF02C
:103E3000E30EE124D96EFF0EE220DA6EEB0E6F0086
:103E40008FFFDFFF080E396EE150EB0FD96EE250A5
:103E5000DA6EFF0EDA223928DE523EEF1FF0DE5214
:103E6000DE52DE52DE52DE52DE52D890DD32DD32DC
:103E7000DD32DD32DD32DD32DD32DE32E82E2FEFB3
:103E80001FF0E40EE124D96EFF0EE220DA6EEB0E95
:103E90006F008FFFDFFF080E396EE150EB0FD96E18
:103EA000E250DA6EFF0EDA223928DE5267EF1FF099
:103EB000DE52DE52DE52DE52DE52DE52D890DD326B
:103EC000DD32DD32DD32DD32DD32DD32DE32E82E72
:103ED00058EF1FF0E50EE124D96EFF0EE220DA6EF6
:103EE000EB0E6F008FFFDFFF080E396EE150EB0F16
:103EF000D96EE250DA6EFF0EDA223928DE5290EFE8
:103F00001FF0DE52DE52DE52DE52DE52DE52D8901A
:103F1000DD32DD32DD32DD32DD32DD32DD32DE3228
:103F2000E82E81EF1FF0E150EB0FD96EE250DA6E10
:103F3000FF0EDA22DD0EE124E96EFF0EE220EA6ECA
:103F40006F007BFFEEFF6F007BFFEEFF6F007BFFDC
:103F5000EEFF6F007BFFEEFFDC0EE1242E6EFF0E06
:103F6000E2202F6E6000BBF0E6FF6000BFF0E6FFCE
:103F7000E5EC37F0DA0E6F008FFFD9FFDB0E6F0034
:103F80008FFFDAFFDF500F0AD8A4C9EF1FF0CBEF85
:103F90001FF0A8EF20F0DC0EE36AE32AE10EE12433
:103FA000D96EFF0EE220DA6E010EDF6EEA0EE1241A
:103FB000D96EFF0EE220DA6EDF6AE20EE124D96EDE
:103FC000FF0EE220DA6EEB0E6F008FFFDFFF080EB0
:103FD000396EE150EB0FD96EE250DA6EFF0EDA2245
:103FE0003928DE5203EF20F0DE52DE52DE52DE527E
:103FF000DE52DE52D890DD32DD32DD32DD32DD32AE
:10400000DD32DD32DE32E82EF4EF1FF0E30EE12484
:10401000D96EFF0EE220DA6EEB0E6F008FFFDFFF2E
:10402000080E396EE150EB0FD96EE250DA6EFF0EDA
:10403000DA223928DE522CEF20F0DE52DE52DE5238
:10404000DE52DE52DE52D890DD32DD32DD32DD323C
:10405000DD32DD32DD32DE32E82E1DEF20F0E40EFF
:10406000E124D96EFF0EE220DA6EEB0E6F008FFFB7
:10407000DFFF080E396EE150EB0FD96EE250DA6EB9
:10408000FF0EDA223928DE5255EF20F0DE52DE52E2
:10409000DE52DE52DE52DE52D890DD32DD32DD32CB
:1040A000DD32DD32DD32DD32DE32E82E46EF20F069
:1040B000E50EE124D96EFF0EE220DA6EEB0E6F0002
:1040C0008FFFDFFF080E396EE150EB0FD96EE25023
:1040D000DA6EFF0EDA223928DE527EEF20F0DE5251
:1040E000DE52DE52DE52DE52DE52D890DD32DD325A
:1040F000DD32DD32DD32DD32DD32DE32E82E6FEFF1
:1041000020F0E150EB0FD96EE250DA6EFF0EDA22AA
:10411000DD0EE124E96EFF0EE220EA6E6F007BFF08
:10412000EEFF6F007BFFEEFF6F007BFFEEFF6F0087
:104130007BFFEEFFDC0EE1242E6EFF0EE2202F6EE1
:104140006000BBF0E6FF6000BFF0E6FFE5EC37F093
:10415000DA0E6F008FFFD9FFDB0E6F008FFFDAFFE3
:10416000DF50100AD8A4B7EF20F0B9EF20F095EF98
:1041700021F0DC0EE36AE32AE10EE124D96EFF0EA2
:10418000E220DA6EDF6AEA0EE124D96EFF0EE22049
:10419000DA6EDF6AE20EE124D96EFF0EE220DA6EFB
:1041A000EB0E6F008FFFDFFF080E396EE150EB0F53
:1041B000D96EE250DA6EFF0EDA223928DE52F0EFC5
:1041C00020F0DE52DE52DE52DE52DE52DE52D89057
:1041D000DD32DD32DD32DD32DD32DD32DD32DE3266
:1041E000E82EE1EF20F0E30EE124D96EFF0EE2208D
:1041F000DA6EEB0E6F008FFFDFFF080E396EE150B5
:10420000EB0FD96EE250DA6EFF0EDA223928DE5259
:1042100019EF21F0DE52DE52DE52DE52DE52DE5265
:10422000D890DD32DD32DD32DD32DD32DD32DD32BD
:10423000DE32E82E0AEF21F0E40EE124D96EFF0E03
:10424000E220DA6EEB0E6F008FFFDFFF080E396E93
:10425000E150EB0FD96EE250DA6EFF0EDA22392808
:10426000DE5242EF21F0DE52DE52DE52DE52DE52EC
:10427000DE52D890DD32DD32DD32DD32DD32DD324C
:10428000DD32DE32E82E33EF21F0E50EE124D96E87
:10429000FF0EE220DA6EEB0E6F008FFFDFFF080EDD
:1042A000396EE150EB0FD96EE250DA6EFF0EDA2272
:1042B0003928DE526BEF21F0DE52DE52DE52DE5242
:1042C000DE52DE52D890DD32DD32DD32DD32DD32DB
:1042D000DD32DD32DE32E82E5CEF21F0E150EB0F13
:1042E000D96EE250DA6EFF0EDA22DD0EE124E96EBD
:1042F000FF0EE220EA6E6F007BFFEEFF6F007BFF98
:10430000EEFF6F007BFFEEFF6F007BFFEEFFDC0E2A
:10431000E1242E6EFF0EE2202F6E6000BBF0E6FF60
:104320006000BFF0E6FFE5EC37F0DA0E6F008FFFBC
:10433000D9FFDB0E6F008FFFDAFFDF50110AD8A420
:10434000A4EF21F0A6EF21F0B0EF22F0DC0EE36A3B
:10435000E32AE10EE124D96EFF0EE220DA6EDF6A75
:10436000EA0EE124D96EFF0EE220DA6E010EDF6E56
:10437000E20EE124D96EFF0EE220DA6EEB0E6F0042
:104380008FFFDFFF080E396EE150EB0FD96EE25060
:10439000DA6EFF0EDA223928DE52DEEF21F0DE522D
:1043A000DE52DE52DE52DE52DE52D890DD32DD3297
:1043B000DD32DD32DD32DD32DD32DE32E82ECFEFCE
:1043C00021F0E30EE124D96EFF0EE220DA6EEB0E4F
:1043D0006F008FFFDFFF080E396EE150EB0FD96ED3
:1043E000E250DA6EFF0EDA223928DE5207EF22F0B1
:1043F000DE52DE52DE52DE52DE52DE52D890DD3226
:10440000DD32DD32DD32DD32DD32DD32DE32E82E2C
:10441000F8EF21F0E40EE124D96EFF0EE220DA6E0F
:10442000EB0E6F008FFFDFFF080E396EE150EB0FD0
:10443000D96EE250DA6EFF0EDA223928DE5230EF02
:1044400022F0DE52DE52DE52DE52DE52DE52D890D2
:10445000DD32DD32DD32DD32DD32DD32DD32DE32E3
:10446000E82E21EF22F0E50EE124D96EFF0EE220C6
:10447000DA6EEB0E6F008FFFDFFF080E396EE15032
:10448000EB0FD96EE250DA6EFF0EDA223928DE52D7
:1044900059EF22F0DE52DE52DE52DE52DE52DE52A2
:1044A000D890DD32DD32DD32DD32DD32DD32DD323B
:1044B000DE32E82E4AEF22F0E150EB0FD96EE250E7
:1044C000DA6EFF0EDA22DD0EE124E96EFF0EE22045
:1044D000EA6E6F007BFFEEFF6F007BFFEEFF6F0069
:1044E0007BFFEEFF6F007BFFEEFFDC0EE1242E6E04
:1044F000FF0EE2202F6E6000BBF0E6FF6000BFF011
:10450000E6FFE5EC37F0B0EF22F0FB0E6F008FFF17
:10451000F6FFFC0E6F008FFFF7FF000EF86E0F0E18
:10452000F76403D00800F55007D06F00DBFFE9FF08
:104530006F00DFFFEAFFEF50386E396A3950000A2A
:10454000D8B4A5EF22F0B0EF22F038500A0AD8B460
:1045500074EF1BF0010AD8B4A0EF1BF0B0EF22F00B
:10456000FF0E6F008CFF39F0FB0E6F008FFFF6FF20
:10457000FC0E6F008FFFF7FF000EF86E0F0EF76452
:1045800003D00800F55007D06F00DBFFE9FF6F0094
:10459000DFFFEAFFEF503918D8B4D1EF22F0D3EFA4
:1045A00022F014EF23F0FF0EE350386E396A3950D1
:1045B000000AD8B4DEEF22F0E9EF22F038500A0A00
:1045C000D8B4E9EF22F0010AD8B4E9EF22F0E9EF1C
:1045D00022F0FB0E6F008FFFF6FFFC0E6F008FFFC7
:1045E000F7FF000EF86E0F0EF76403D00800F550C9
:1045F00007D06F00DBFFE9FF6F00DFFFEAFFEF503E
:10460000386E396A3950000AD8B409EF23F014EF34
:1046100023F038500A0AD8B414EF23F0010AD8B4B2
:1046200014EF23F014EF23F0DA0EE126FF0EE2225E
:1046300012000A0EE126000EE222EF0E6F008CFF40
:1046400036F0F00E6F008CFF37F0F10E6F008CFF2C
:1046500038F0F20E6F008CFF39F0F60E6000DBF0E0
:10466000E3FFF70E6000DFF0E3FFF80E6000E3F019
:10467000E3FFF90E6000E7F0E3FFF90EE124D96EE5
:10468000FF0EE220DA6EDF50396EFA0E6000E7F0BE
:10469000E3FFF80EE124D96EFF0EE220DA6EFB0E86
:1046A000E124E96EFF0EE220EA6E6F007FFFEFFF6C
:1046B000F70EE124D96EFF0EE220DA6EFC0EE12443
:1046C000E96EFF0EE220EA6E6F007FFFEFFFFD0E46
:1046D000E124D96EFF0EE220DA6EF60E6F008FFF36
:1046E000DFFFEF0E6F008CFF2EF0FE0E6000BBF0C0
:1046F000E3FFF00E6F008CFF2EF0FF0E6000BBF0AA
:10470000E3FF30EF29F0F40EE350D8A48AEF23F052
:104710008CEF23F0DEEF23F0F70EE124D96EFF0ECD
:10472000E220DA6EDF50D8B498EF23F09AEF23F04E
:104730009CEF23F086EC64F0F60E6F008CFF01F026
:10474000F90EE124D96EFF0EE220DA6EDF50026E20
:104750000150E66E010EE66EA9EC63F00250E66EC3
:10476000020EE66EA9EC63F00250E66E7DEC64F09A
:104770006000BBF0E6FF6000BFF0E6FFFEEC5FF01C
:10478000000EE66E000EE66E000EE66E000EE66EA1
:10479000000EE66E000EE66E000EE66E000EE66E91
:1047A000000EE66E000EE66E7DEC64F06000BBF07D
:1047B000E6FF6000BFF0E6FF8FEC5CF0F40EE30470
:1047C000D8A4E5EF23F0E7EF23F00AEF24F0E1505F
:1047D000FA0FD96EE250DA6EFF0EDA226F0078FF20
:1047E00003F06F0078FF04F06F0078FF05F06F00B2
:1047F00078FF06F060000FF0E6FF600013F0E6FFC0
:10480000600017F0E6FF60001BF0E6FF030EE66EA7
:1048100073EC57F0F40E6F008CFF2EF0020E2E1882
:10482000D8A415EF24F017EF24F04CEF24F0E1505A
:10483000FA0FD96EE250DA6EFF0EDA226F0078FFBF
:1048400007F06F0078FF08F06F0078FF09F06F0045
:1048500078FF0AF060001FF0E6FF600023F0E6FF3B
:10486000600027F0E6FF60002BF0E6FF070EE66E23
:1048700073EC57F060001FF0E6FF600023F0E6FFE6
:10488000600027F0E6FF60002BF0E6FF050EE66E05
:10489000000EE66E48EC3BF0F40E6F008CFF2EF03D
:1048A000030E2E18D8A457EF24F059EF24F07CEF14
:1048B00024F0E150FA0FD96EE250DA6EFF0EDA22E0
:1048C0006F0078FF0BF06F0078FF0CF06F0078FF3F
:1048D0000DF06F0078FF0EF060002FF0E6FF600033
:1048E00033F0E6FF600037F0E6FF60003BF0E6FFE4
:1048F0000B0EE66E73EC57F0F40E6F008CFF2EF08B
:10490000040E2E18D8A487EF24F089EF24F0A1EF2D
:1049100024F0F60E6F008CFF0FF0F70EE124D96E35
:10492000FF0EE220DA6EDF50106E0F50E66E0F0EB3
:10493000E66EA9EC63F01050E66E100EE66EA9EC80
:1049400063F0F40E6F008CFF2EF0050E2E18D8A425
:10495000ACEF24F0AEEF24F0D2EF24F0F60E6F00AF
:104960008CFF15F0F70EE124D96EFF0EE220DA6E0F
:10497000DF50196E1550E66E150EE66EA9EC63F069
:104980001950E66E190EE66EA9EC63F0000EE66EA5
:10499000000EE66E51EC60F0020EE66E100EE66E52
:1049A000FCEC51F0F40E6F008CFF2EF0060E2E186A
:1049B000D8A4DDEF24F0DFEF24F043EF25F0F60E6E
:1049C0006F008CFF11F0F70EE124D96EFF0EE2208C
:1049D000DA6EDF50126EF80EE124D96EFF0EE2207F
:1049E000DA6EDF50136EF90EE124D96EFF0EE2206D
:1049F000DA6EDF50146E1150E66E110EE66EA9EC01
:104A000063F01250E66E120EE66EA9EC63F01350DE
:104A1000E66E130EE66EA9EC63F01450E66E140E0B
:104A2000E66EA9EC63F01450E66E74EC64F060007E
:104A3000BBF0E6FF6000BFF0E6FFFEEC5FF0000EAB
:104A4000E66E000EE66E000EE66E000EE66E000EDE
:104A5000E66E000EE66E000EE66E000EE66E000ECE
:104A6000E66E000EE66E74EC64F06000BBF0E6FFEC
:104A70006000BFF0E6FF8FEC5CF0000EE66E000E0B
:104A8000E66E09EC5AF0F40E6F008CFF2EF0070E64
:104A90002E18D8A44EEF25F050EF25F0AEEF25F0FC
:104AA000F60E6F008CFF18F0F70EE124D96EFF0EA2
:104AB000E220DA6EDF50166EF80EE124D96EFF0E9A
:104AC000E220DA6EDF50176E1850E66E180EE66EB2
:104AD000A9EC63F01650E66E160EE66EA9EC63F0D4
:104AE0001750E66E170EE66EA9EC63F01850E66EEE
:104AF00062EC64F0010E2E26000E2F226000BBF047
:104B0000E6FF6000BFF0E6FFFEEC5FF0000EE66E31
:104B1000000EE66E000EE66E000EE66E000EE66E0D
:104B2000000EE66E000EE66E000EE66E000EE66EFD
:104B3000000EE66E62EC64F0010E2E26000E2F22AF
:104B40006000BBF0E6FF6000BFF0E6FF8FEC5CF0BA
:104B5000030EE66E100EE66E15EC59F0F40E6F00C3
:104B60008CFF2EF0080E2E18D8A4B9EF25F0BBEF5D
:104B700025F0F5EF25F0F60E6F008CFF1AF0F70E1A
:104B8000E124D96EFF0EE220DA6EDF501B6EF80EC4
:104B9000E124D96EFF0EE220DA6EDF501C6EF90EB2
:104BA000E124D96EFF0EE220DA6EDF501D6E1A503E
:104BB000E66E1A0EE66EA9EC63F01B50E66E1B0E55
:104BC000E66EA9EC63F01C50E66E1C0EE66EA9ECD6
:104BD00063F01D50E66E1D0EE66EA9EC63F0000E4C
:104BE000E66E000EE66ECEEC59F0F40E6F008CFF10
:104BF0002EF0090E2E18D8A400EF26F002EF26F0B2
:104C00005AEF29F0F60E6F008CFF1EF0F70EE1242C
:104C1000D96EFF0EE220DA6EDF501F6E1E50E66E78
:104C20001E0EE66EA9EC63F01F50E66E1F0EE66ED8
:104C3000A9EC63F05AEF29F0F40EE304D8A423EFB3
:104C400026F025EF26F03EEF26F0F70EE124D96E90
:104C5000FF0EE220DA6EDF50E66EF8EC45F0F60E5D
:104C6000E350E66E20EC43F050EC64F06000BBF0E3
:104C7000E6FF6000BFF0E6FF1BEC5CF0F40E6F0097
:104C80008CFF2EF00F0E2E18D8A449EF26F04BEF14
:104C900026F05AEF29F074EC64F06000BBF0E6FFF8
:104CA0006000BFF0E6FF73EC63F074EC64F060004A
:104CB000BBF0D9FF6000BFF0DAFF180EDE18D8A4F1
:104CC00064EF26F066EF26F05AEF29F0110EE66E3B
:104CD0006BEC64F02E50116E120EE66E6BEC64F00D
:104CE0002E50126E130EE66E6BEC64F02E50136EA7
:104CF000140EE66E6BEC64F02E50146E1450E66EDB
:104D000074EC64F06000BBF0E6FF6000BFF0E6FF0B
:104D1000FEEC5FF0000EE66E000EE66E000EE66E34
:104D2000000EE66E000EE66E000EE66E000EE66EFB
:104D3000000EE66E000EE66E000EE66E74EC64F099
:104D40006000BBF0E6FF6000BFF0E6FFC9EC5CF07E
:104D5000000EE66E000EE66E000EE66E000EE66ECB
:104D6000000EE66E000EE66E000EE66E000EE66EBB
:104D7000000EE66E000EE66E74EC64F06000BBF0B0
:104D8000E6FF6000BFF0E6FF3DEC5DF0000EE66E72
:104D9000000EE66E000EE66E000EE66E000EE66E8B
:104DA000000EE66E000EE66E000EE66E000EE66E7B
:104DB000000EE66E74EC64F06000BBF0E6FF60008D
:104DC000BFF0E6FF03EC5DF05AEF29F0F40E6F0040
:104DD0008CFF2EF00F0E2E18D8A4F1EF26F0F3EF73
:104DE00026F05AEF29F0F60E6F008CFFD5F0000187
:104DF000D551D8A4FEEF26F000EF27F008EF27F0FA
:104E0000030EE66E100EE66E0EEC61F05AEF29F01E
:104E1000040EE66E100EE66E0EEC61F05AEF29F00D
:104E2000F40EE350D8A417EF27F019EF27F032EF74
:104E300027F0FA0E6F008FFFE6FF6F008FFFE6FF8F
:104E40006F008FFFE6FF6F008FFFE6FFB8EC4EF0BC
:104E500062EC64F06000BBF0E6FF6000BFF0E6FFCC
:104E600055EC5CF0F40E6F008CFF2EF00F0E2E1838
:104E7000D8A43DEF27F03FEF27F05AEF29F062EC7E
:104E800064F0010E2E26000E2F226000BBF0E6FF1C
:104E90006000BFF0E6FF73EC63F062EC64F0010EBB
:104EA0002E24D96E000E2F20DA6E180EDE18D8A42C
:104EB0005CEF27F05EEF27F05AEF29F0160EE66E52
:104EC0006BEC64F02E50166E170EE66E6BEC64F011
:104ED0002E50176E180EE66E6BEC64F02E50186EA6
:104EE000000EE66E000EE66E000EE66E000EE66E3A
:104EF000000EE66E000EE66E000EE66E000EE66E2A
:104F0000000EE66E000EE66E62EC64F0010E2E26D8
:104F1000000E2F226000BBF0E6FF6000BFF0E6FF4E
:104F2000C9EC5CF0000EE66E000EE66E000EE66E5A
:104F3000000EE66E000EE66E000EE66E000EE66EE9
:104F4000000EE66E000EE66E000EE66E62EC64F099
:104F5000010E2E26000E2F226000BBF0E6FF60003F
:104F6000BFF0E6FF3DEC5DF05AEF29F0F40EE304EC
:104F7000D8A4BDEF27F0BFEF27F0F4EF27F0E15002
:104F8000FA0FD96EE250DA6EFF0EDA226F0078FF68
:104F9000CBF06F0078FFCCF06F0078FFCDF06F00A2
:104FA00078FFCEF0000EE66E000EE66E000EE66EA6
:104FB000000EE66E000EE66E000EE66E000EE66E69
:104FC000000EE66E000EE66E000EE66E50EC64F02B
:104FD000010E2E26000E2F226000BBF0E6FF6000BF
:104FE000BFF0E6FF03EC5DF0F40E6F008CFF2EF0D7
:104FF0000E0E2E18D8A4FFEF27F001EF28F00EEFC9
:1050000028F0F60EE350D8A408EF28F00BEF28F0B4
:10501000010E0CEF28F0000E0001D46FF40E6F00AB
:105020008CFF2EF00F0E2E18D8A419EF28F01BEFCE
:1050300028F05AEF29F050EC64F0010E2E26000EF5
:105040002F226000BBF0E6FF6000BFF0E6FF73ECCC
:1050500063F050EC64F0010E2E24D96E000E2F2068
:10506000DA6E180EDE18D8A438EF28F03AEF28F0E0
:1050700084EF28F0190EE66E6BEC64F02E50196E7A
:10508000000EE66E000EE66E000EE66E000EE66E98
:10509000000EE66E000EE66E000EE66E000EE66E88
:1050A000F40EE66E010EE66E50EC64F0010E2E2654
:1050B000000E2F226000BBF0E6FF6000BFF0E6FFAD
:1050C000C9EC5CF0000EE66E000EE66E000EE66EB9
:1050D000000EE66E000EE66E000EE66E000EE66E48
:1050E000000EE66EE80EE66E030EE66E50EC64F01F
:1050F000010E2E26000E2F226000BBF0E6FF60009E
:10510000BFF0E6FF3DEC5DF0E150FE0FD96EE250DE
:10511000DA6EFF0EDA22DFA890EF28F092EF28F087
:105120005AEF29F050EC64F0010E2E24D96E000ED7
:105130002F20DA6E160EDE18D8A4A1EF28F0A3EF08
:1051400028F05AEF29F0000EE66E000EE66E000E13
:10515000E66E000EE66E000EE66E000EE66E000EC7
:10516000E66E000EE66EE80EE66E030EE66E50EC9E
:1051700064F0010E2E26000E2F226000BBF0E6FF29
:105180006000BFF0E6FF03EC5DF05AEF29F0F40E8B
:105190006F008CFF2EF0040E2E18D8A4D2EF28F04A
:1051A000D4EF28F05AEF29F062EC64F06000BBF015
:1051B000E6FF6000BFF0E6FF9EEC60F050EC64F0AC
:1051C0006000BBF0E6FF6000BFF0E6FF78EC60F047
:1051D00074EC64F06000BBF0E6FF6000BFF0E6FF37
:1051E0000DEC5FF0000EE66E000EE66E000EE66E51
:1051F000000EE66E000EE66E000EE66E000EE66E27
:10520000000EE66E640EE66E000EE66E74EC64F060
:105210006000BBF0E6FF6000BFF0E6FF3DEC5DF034
:10522000000EE66E000EE66E000EE66E000EE66EF6
:10523000000EE66E000EE66E000EE66E000EE66EE6
:10524000C80EE66E000EE66E74EC64F06000BBF013
:10525000E6FF6000BFF0E6FF03EC5DF05AEF29F0D7
:10526000F50EE350386E396A3950000AD8B43BEF76
:1052700029F05AEF29F03850000AD8B483EF23F010
:10528000020AD8B41CEF26F0010AD8B4E6EF26F0E3
:10529000070AD8B410EF27F0010AD8B4B6EF27F008
:1052A000030AD8B4C7EF28F0010AD8B45AEF29F09E
:1052B0005AEF29F0EF0EE126FF0EE2221200E6522D
:1052C000E652E652E652FA0E6F008FFFE6FF6F00DD
:1052D0008FFFE6FFCFEC62F0FD0E6000BFF0E3FF52
:1052E000FC0E6000BBF0E3FFFC0E6F008FFFF6FFCB
:1052F000FD0E6F008FFFF7FF000EF86E0F0EF764C4
:1053000003D00800F55007D06F00DBFFE9FF6F0006
:10531000DFFFEAFFEF50396EFF0E6000E7F0E3FFBA
:10532000FA0E6F008FFFE6FF6F008FFFE6FF8FEC36
:1053300063F0FE0E6000BBF0E3FF19EF2DF0FA0EF4
:105340006F008FFFD9FFFB0E6F008FFFDAFFDF507A
:10535000C80AD8A4AEEF29F0B0EF29F04CEF2DF039
:10536000FC0E6F008FFFF6FFFD0E6F008FFFF7FF43
:10537000000EF86E0F0EF76404D0010EF56E0C00EF
:1053800008D06F00DBFFE9FF6F00DFFFEAFF010ECF
:10539000EF6E4CEF2DF0FC0EE350050F386EFD0E56
:1053A0006F008CFF39F0000E39226000E3F0F6FF49
:1053B0006000E7F0F7FF000EF86E0F0EF76403D001
:1053C0000800F55007D06F00DBFFE9FF6F00DFFF3B
:1053D000EAFFEF50396EFC0EE350070F366EFD0EFC
:1053E0006F008CFF37F0000E37226000DBF0F6FF15
:1053F0006000DFF0F7FF000EF86E0F0EF76405D0C7
:105400006000E7F0F5FF0C0009D06F00DBFFE9FF5B
:105410006F00DFFFEAFF6000E7F0EFFFFE0E6F00B6
:105420008CFF2EF0CA0E2E18D8A419EF2AF01BEF0D
:105430002AF08EEF2AF0FC0E6F008FFFF6FFFD0EB4
:105440006F008FFFF7FF000EF86E0F0EF76404D0A9
:10545000020EF56E0C0008D06F00DBFFE9FF6F0055
:10546000DFFFEAFF020EEF6EFC0EE350060F386E10
:10547000FD0E6F008CFF39F0000E39226000E3F062
:10548000F6FF6000E7F0F7FF000EF86E0F0EF7640E
:1054900004D0010EF56E0C0008D06F00DBFFE9FFB1
:1054A0006F00DFFFEAFF010EEF6EFC0EE350010F0D
:1054B000386EFD0E6F008CFF39F0000E392260004F
:1054C000E3F0F6FF6000E7F0F7FF000EF86E0F0E56
:1054D000F76409D009006F00D4FF38F009006F00AD
:1054E000D4FF39F00CD06F00DBFFE9FF6F00DFFF66
:1054F000EAFF6F00B8FF38F06F00B8FF39F06000C6
:10550000E3F0E6FF6000E7F0E6FFFA0E6F008FFFC2
:10551000E6FF6F008FFFE6FFA8EC5FF0FE0E6F0066
:105520008CFF2EF0C90E2E18D8A499EF2AF09BEF0D
:105530002AF04CEF2DF0FC0E6F008FFFF6FFFD0EF2
:105540006F008FFFF7FF000EF86E0F0EF76404D0A8
:10555000020EF56E0C0008D06F00DBFFE9FF6F0054
:10556000DFFFEAFF020EEF6EFC0EE350060F386E0F
:10557000FD0E6F008CFF39F0000E39226000E3F061
:10558000F6FF6000E7F0F7FF000EF86E0F0EF7640D
:1055900004D0000EF56E0C0008D06F00DBFFE9FFB1
:1055A0006F00DFFFEAFF000EEF6EFC0EE350010F0D
:1055B000386EFD0E6F008CFF39F0000E392260004E
:1055C000E3F0F6FF6000E7F0F7FF000EF86E0F0E55
:1055D000F76409D009006F00D4FF38F009006F00AC
:1055E000D4FF39F00CD06F00DBFFE9FF6F00DFFF65
:1055F000EAFF6F00B8FF38F06F00B8FF39F06000C5
:10560000E3F0E6FF6000E7F0E6FFFA0E6F008FFFC1
:10561000E6FF6F008FFFE6FFA8EC5FF04CEF2DF088
:10562000FC0EE350060F386EFD0E6F008CFF39F054
:10563000000E39226000E3F0F6FF6000E7F0F7FFAC
:10564000000EF86E0F0EF76403D00800F55007D077
:105650006F00DBFFE9FF6F00DFFFEAFFEF5000099B
:10566000D8B435EF2BF037EF2BF07CEF2BF0FC0E9E
:10567000E350070F386EFD0E6F008CFF39F0000EFF
:1056800039226000E3F0F6FF6000E7F0F7FF000E5C
:10569000F86E0F0EF76403D00800F55007D06F00C6
:1056A000DBFFE9FF6F00DFFFEAFFEF50396EFF0E0F
:1056B0003926FC0EE350070F366EFD0E6F008CFF8F
:1056C00037F0000E37226000DBF0F6FF6000DFF0FD
:1056D000F7FF000EF86E0F0EF76405D06000E7F0DC
:1056E000F5FF0C0009D06F00DBFFE9FF6F00DFFF63
:1056F000EAFF6000E7F0EFFFFE0E6F008CFF2EF078
:10570000CB0E2E18D8A487EF2BF089EF2BF04CEF9F
:105710002DF0FC0E6F008FFFF6FFFD0E6F008FFF68
:10572000F7FF000EF86E0F0EF76404D0030EF56E4F
:105730000C0008D06F00DBFFE9FF6F00DFFFEAFF1E
:10574000030EEF6EFC0EE350030F386EFD0E6F007C
:105750008CFF39F0000E39226000E3F0F6FF6000A4
:10576000E7F0F7FF000EF86E0F0EF76409D009009E
:105770006F00D4FF38F009006F00D4FF39F00CD06F
:105780006F00DBFFE9FF6F00DFFFEAFF6F00B8FF8C
:1057900038F06F00B8FF39F06000E3F0E6FF60001A
:1057A000E7F0E6FFFA0E6F008FFFE6FF6F008FFF56
:1057B000E6FFA8EC5FF04CEF2DF0FE0E6F008CFFC3
:1057C0002EF0CB0E2E18D8A4E8EF2BF0EAEF2BF03A
:1057D0004CEF2DF0FC0EE350070F386EFD0E6F00FE
:1057E0008CFF39F0000E39226000E3F0F6FF600014
:1057F000E7F0F7FF000EF86E0F0EF76403D0080015
:10580000F55007D06F00DBFFE9FF6F00DFFFEAFF15
:10581000EF500009D8A40FEF2CF011EF2CF0C5EFDA
:105820002CF0FC0E6F008FFFF6FFFD0E6F008FFF58
:10583000F7FF000EF86E0F0EF76404D0010EF56E40
:105840000C0008D06F00DBFFE9FF6F00DFFFEAFF0D
:10585000010EEF6EFC0EE350140F386EFD0E6F005C
:105860008CFF39F0000E39226000E3F0F6FF600093
:10587000E7F0F7FF000EF86E0F0EF76409D009008D
:105880006F00D4FF38F009006F00D4FF39F00CD05E
:105890006F00DBFFE9FF6F00DFFFEAFF6F00B8FF7B
:1058A00038F06F00B8FF39F038503910D8B45BEFDA
:1058B0002CF05DEF2CF04CEF2DF0FC0EE350160FAA
:1058C000386EFD0E6F008CFF39F0000E392260003B
:1058D000E3F0F6FF6000E7F0F7FF000EF86E0F0E42
:1058E000F76409D009006F00D4FF38F009006F0099
:1058F000D4FF39F00CD06F00DBFFE9FF6F00DFFF52
:10590000EAFF6F00B8FF38F06F00B8FF39F06000B1
:10591000E3F0E6FF6000E7F0E6FFFA0EE350140F55
:10592000386EFB0E6F008CFF39F0000E39226000DC
:10593000E3F0F6FF6000E7F0F7FF000EF86E0F0EE1
:10594000F76409D009006F00D4FF38F009006F0038
:10595000D4FF39F00CD06F00DBFFE9FF6F00DFFFF1
:10596000EAFF6F00B8FF38F06F00B8FF39F002D8D7
:10597000C3EF2CF00500FA6E3850FD6E3950FE6E04
:10598000FF6AFA5012004CEF2DF0FC0E6F008FFFF3
:10599000F6FFFD0E6F008FFFF7FF000EF86E0F0E83
:1059A000F76404D0020EF56E0C0008D06F00DBFF28
:1059B000E9FF6F00DFFFEAFF020EEF6EFC0EE3501F
:1059C000010F386EFD0E6F008CFF39F0000E39228A
:1059D0006000E3F0F6FF6000E7F0F7FF000EF86EFE
:1059E0000F0EF76409D009006F00D4FF38F00900EA
:1059F0006F00D4FF39F00CD06F00DBFFE9FF6F00C0
:105A0000DFFFEAFF6F00B8FF38F06F00B8FF39F032
:105A10006000E3F0E6FF6000E7F0E6FFFA0E6F00DB
:105A20008FFFE6FF6F008FFFE6FFA8EC5FF04CEF03
:105A30002DF0FC0E6F008FFFF6FFFD0E6F008FFF45
:105A4000F7FF000EF86E0F0EF76403D00800F55054
:105A500007D06F00DBFFE9FF6F00DFFFEAFFEF50C9
:105A6000386E396A3950000AD8B439EF2DF04CEF4E
:105A70002DF03850000AD8B49FEF29F0010AD8B4AD
:105A8000CBEF29F0030AD8B410EF2BF0010AD8B4F9
:105A9000DDEF2BF04CEF2DF0FF0E6F008CFF39F097
:105AA000FC0E6F008FFFF6FFFD0E6F008FFFF7FFFC
:105AB000000EF86E0F0EF76403D00800F55007D003
:105AC0006F00DBFFE9FF6F00DFFFEAFFEF503918DF
:105AD000D8B46DEF2DF06FEF2DF091EF2FF0FF0E9A
:105AE000E350386E396A3950000AD8B47AEF2DF095
:105AF0005EEF2FF03850000AD8B45EEF2FF0010AA5
:105B0000D8B45EEF2FF0030AD8B45EEF2FF0010A8D
:105B1000D8B45EEF2FF05EEF2FF0FC0EE350080FCD
:105B2000386EFD0E6F008CFF39F0000E39226000D8
:105B3000E3F0F6FF6000E7F0F7FF000EF86E0F0EDF
:105B4000F76409D009006F00D4FF38F009006F0036
:105B5000D4FF39F00CD06F00DBFFE9FF6F00DFFFEF
:105B6000EAFF6F00B8FF38F06F00B8FF39F0385027
:105B70003910D8B4BEEF2DF0C0EF2DF091EF2FF01B
:105B8000FC0EE3500A0F386EFD0E6F008CFF39F0EB
:105B9000000E39226000E3F0F6FF6000E7F0F7FF47
:105BA000000EF86E0F0EF76409D009006F00D4FFE5
:105BB00038F009006F00D4FF39F00CD06F00DBFF24
:105BC000E9FF6F00DFFFEAFF6F00B8FF38F06F00FA
:105BD000B8FF39F06000E3F0E6FF6000E7F0E6FFB1
:105BE000FA0EE350080F386EFB0E6F008CFF39F091
:105BF000000E39226000E3F0F6FF6000E7F0F7FFE7
:105C0000000EF86E0F0EF76409D009006F00D4FF84
:105C100038F009006F00D4FF39F00CD06F00DBFFC3
:105C2000E9FF6F00DFFFEAFF6F00B8FF38F06F0099
:105C3000B8FF39F002D826EF2EF00500FA6E385082
:105C4000FD6E3950FE6EFF6AFA50120091EF2FF090
:105C5000FC0EE3500C0F386EFD0E6F008CFF39F018
:105C6000000E39226000E3F0F6FF6000E7F0F7FF76
:105C7000000EF86E0F0EF76409D009006F00D4FF14
:105C800038F009006F00D4FF39F00CD06F00DBFF53
:105C9000E9FF6F00DFFFEAFF6F00B8FF38F06F0029
:105CA000B8FF39F038503910D8B459EF2EF05BEF07
:105CB0002EF091EF2FF0FC0EE3500E0F386EFD0E1C
:105CC0006F008CFF39F0000E39226000E3F0F6FF20
:105CD0006000E7F0F7FF000EF86E0F0EF76409D0D2
:105CE00009006F00D4FF38F009006F00D4FF39F0CD
:105CF0000CD06F00DBFFE9FF6F00DFFFEAFF6F00F2
:105D0000B8FF38F06F00B8FF39F06000E3F0E6FF4D
:105D10006000E7F0E6FFFA0EE3500C0F386EFB0E62
:105D20006F008CFF39F0000E39226000E3F0F6FFBF
:105D30006000E7F0F7FF000EF86E0F0EF76409D071
:105D400009006F00D4FF38F009006F00D4FF39F06C
:105D50000CD06F00DBFFE9FF6F00DFFFEAFF6F0091
:105D6000B8FF38F06F00B8FF39F002D8C1EF2EF05D
:105D70000500FA6E3850FD6E3950FE6EFF6AFA501B
:105D8000120091EF2FF0FC0EE350100F386EFD0E55
:105D90006F008CFF39F0000E39226000E3F0F6FF4F
:105DA0006000E7F0F7FF000EF86E0F0EF76409D001
:105DB00009006F00D4FF38F009006F00D4FF39F0FC
:105DC0000CD06F00DBFFE9FF6F00DFFFEAFF6F0021
:105DD000B8FF38F06F00B8FF39F038503910D8B438
:105DE000F4EF2EF0F6EF2EF091EF2FF0FC0EE350D3
:105DF000120F386EFD0E6F008CFF39F0000E392245
:105E00006000E3F0F6FF6000E7F0F7FF000EF86EC9
:105E10000F0EF76409D009006F00D4FF38F00900B5
:105E20006F00D4FF39F00CD06F00DBFFE9FF6F008B
:105E3000DFFFEAFF6F00B8FF38F06F00B8FF39F0FE
:105E40006000E3F0E6FF6000E7F0E6FFFA0EE350E3
:105E5000100F386EFB0E6F008CFF39F0000E3922E8
:105E60006000E3F0F6FF6000E7F0F7FF000EF86E69
:105E70000F0EF76409D009006F00D4FF38F0090055
:105E80006F00D4FF39F00CD06F00DBFFE9FF6F002B
:105E9000DFFFEAFF6F00B8FF38F06F00B8FF39F09E
:105EA00002D85CEF2FF00500FA6E3850FD6E3950C5
:105EB000FE6EFF6AFA50120091EF2FF0FC0E6F0099
:105EC0008FFFF6FFFD0E6F008FFFF7FF000EF86EDD
:105ED0000F0EF76403D00800F55007D06F00DBFF0A
:105EE000E9FF6F00DFFFEAFFEF50386E396A395083
:105EF000000AD8B47EEF2FF091EF2FF03850000A4F
:105F0000D8B491EF2FF0010AD8B48DEF2DF0030A29
:105F1000D8B428EF2EF0010AD8B4C3EF2EF091EFD9
:105F20002FF0FA0EE126FF0EE2221200E652E652B0
:105F3000E652FB0E6F008FFFE6FF6F008FFFE6FF5C
:105F4000CFEC62F0FE0E6000BFF0E3FFFD0E6000DC
:105F5000BBF0E3FFFD0E6F008FFFF6FFFE0E6F003C
:105F60008FFFF7FF000EF86E0F0EF76403D00800E6
:105F7000F55007D06F00DBFFE9FF6F00DFFFEAFF9E
:105F8000EF50396EFF0E6000E7F0E3FFFB0E6F008D
:105F90008FFFE6FF6F008FFFE6FF8FEC63F0FB0ED5
:105FA0006F008FFFE6FF6F008FFFE6FF31EC62F0BE
:105FB000F80EE126FF0EE2225FEF31F0FB0E6F00DC
:105FC0008FFFD9FFFC0E6F008FFFDAFFDF50640AEE
:105FD000D8A4EDEF2FF0EFEF2FF092EF31F0FD0EA0
:105FE0006F008FFFF6FFFE0E6F008FFFF7FF000EB2
:105FF000F86E0F0EF76404D0650EF56E0C0008D035
:106000006F00DBFFE9FF6F00DFFFEAFF650EEF6E59
:10601000FD0EE350010F386EFE0E6F008CFF39F05D
:10602000000E39226000E3F0E6FF6000E7F0E6FFD3
:106030000DEC5FF092EF31F0FB0E6F008FFFD9FF98
:10604000FC0E6F008FFFDAFFDF50650AD8A42BEF3C
:1060500030F02DEF30F046EF30F0FD0E6F008FFF87
:10606000F6FFFE0E6F008FFFF7FF000EF86E0F0EAB
:10607000F76404D0660EF56E0C0008D06F00DBFFED
:10608000E9FF6F00DFFFEAFF660EEF6E1850E66E65
:10609000FC0EE350010F386EFD0E6F008CFF39F0DF
:1060A000000E39226000E3F0E6FF6000E7F0E6FF53
:1060B000FEEC5FF0000EE66E000EE66E000EE66E81
:1060C000000EE66E000EE66E000EE66E000EE66E48
:1060D000000EE66E640EE66E000EE66EF30EE35002
:1060E000010F386EF40E6F008CFF39F0000E39226C
:1060F0006000E3F0E6FF6000E7F0E6FF3DEC5DF0F6
:10610000000EE66E000EE66E000EE66E000EE66E07
:10611000000EE66E000EE66E000EE66E000EE66EF7
:10612000C80EE66E000EE66EF30EE350010F386EF9
:10613000F40E6F008CFF39F0000E39226000E3F09E
:10614000E6FF6000E7F0E6FF03EC5DF092EF31F070
:10615000FB0E6F008FFFD9FFFC0E6F008FFFDAFF81
:10616000DF50660AD8A4B7EF30F0B9EF30F0D2EFC5
:1061700030F0FD0E6F008FFFF6FFFE0E6F008FFFF9
:10618000F7FF000EF86E0F0EF76404D0670EF56E81
:106190000C0008D06F00DBFFE9FF6F00DFFFEAFFB4
:1061A000670EEF6EFB0E6F008FFFD9FFFC0E6F00C6
:1061B0008FFFDAFFDF50690AD8A4E1EF30F0E3EF98
:1061C00030F01AEF31F0C90EE66E000EE66E28ECE4
:1061D00058F01750D8A4EFEF30F0F1EF30F0F3EFB4
:1061E00030F0010E176E000EE66E000EE66E000E29
:1061F000E66E000EE66E000EE66E000EE66E000E17
:10620000E66E000EE66E1750050D6F00CCFF38F0FD
:106210006F00D0FF39F06000E3F0E6FF6000E7F0C8
:10622000E6FFF30E6F008FFFE6FF6F008FFFE6FFC4
:10623000E1EC5BF0FB0E6F008FFFD9FFFC0E6F00EF
:106240008FFFDAFFDF50680AD8A429EF31F02BEF77
:1062500031F092EF31F0D30EE66E000EE66E54ECA4
:1062600059F092EF31F0FB0E6F008FFFD9FFFC0E5B
:106270006F008FFFDAFFDF50670AD8A442EF31F0DA
:1062800044EF31F092EF31F0FD0E6F008FFFF6FF1B
:10629000FE0E6F008FFFF7FF000EF86E0F0EF76413
:1062A00004D0650EF56E0C0008D06F00DBFFE9FF2F
:1062B0006F00DFFFEAFF650EEF6E92EF31F0FD0E2B
:1062C0006F008FFFF6FFFE0E6F008FFFF7FF000ECF
:1062D000F86E0F0EF76403D00800F55007D06F007A
:1062E000DBFFE9FF6F00DFFFEAFFEF50386E396A2E
:1062F0003950000AD8B47FEF31F092EF31F03850C6
:10630000640AD8B4DEEF2FF0010AD8B41CEF30F0E5
:10631000030AD8B4A8EF30F0010AD8B433EF31F053
:1063200092EF31F0FF0E6F008CFF39F0FD0E6F0021
:106330008FFFF6FFFE0E6F008FFFF7FF000EF86E67
:106340000F0EF76403D00800F55007D06F00DBFF95
:10635000E9FF6F00DFFFEAFFEF503918D8B4B3EF61
:1063600031F0B5EF31F008EF34F0FF0EE350386E46
:10637000396A3950000AD8B4C0EF31F0D5EF33F0A4
:106380003850640AD8B4D5EF33F0010AD8B4D5EF49
:1063900033F0030AD8B4D5EF33F0010AD8B4D5EFFF
:1063A00033F0D5EF33F0FD0EE350380F386EFE0EAC
:1063B0006F008CFF39F0000E39226000E3F0F6FF29
:1063C0006000E7F0F7FF000EF86E0F0EF76409D0DB
:1063D00009006F00D4FF38F009006F00D4FF39F0D6
:1063E0000CD06F00DBFFE9FF6F00DFFFEAFF6F00FB
:1063F000B8FF38F06F00B8FF39F038503910D8B412
:1064000004EF32F006EF32F008EF34F0FD0EE35007
:106410003A0F386EFE0E6F008CFF39F0000E3922F5
:106420006000E3F0F6FF6000E7F0F7FF000EF86EA3
:106430000F0EF76409D009006F00D4FF38F009008F
:106440006F00D4FF39F00CD06F00DBFFE9FF6F0065
:10645000DFFFEAFF6F00B8FF38F06F00B8FF39F0D8
:106460006000E3F0E6FF6000E7F0E6FFFB0EE350BC
:10647000380F386EFC0E6F008CFF39F0000E392299
:106480006000E3F0F6FF6000E7F0F7FF000EF86E43
:106490000F0EF76409D009006F00D4FF38F009002F
:1064A0006F00D4FF39F00CD06F00DBFFE9FF6F0005
:1064B000DFFFEAFF6F00B8FF38F06F00B8FF39F078
:1064C00002D86CEF32F00500FA6E3850FD6E39508C
:1064D000FE6EFF6AFA50120008EF34F01750D8A48D
:1064E00074EF32F076EF32F078EF32F0010E176E83
:1064F000000EE66E000EE66E000EE66E000EE66E14
:10650000000EE66E000EE66E000EE66E000EE66E03
:106510001750050D6F00CCFF38F06F00D0FF39F039
:106520006000E3F0E6FF6000E7F0E6FFF30E6F00C7
:106530008FFFE6FF6F008FFFE6FFE1EC5BF0FD0EE3
:10654000E3503C0F386EFE0E6F008CFF39F0000EEA
:1065500039226000E3F0F6FF6000E7F0F7FF000E7D
:10656000F86E0F0EF76409D009006F00D4FF38F001
:1065700009006F00D4FF39F00CD06F00DBFFE9FF9A
:106580006F00DFFFEAFF6F00B8FF38F06F00B8FF61
:1065900039F038503910D8B4D0EF32F0D2EF32F0B1
:1065A00008EF34F0FD0EE3503E0F386EFE0E6F0024
:1065B0008CFF39F0000E39226000E3F0F6FF600036
:1065C000E7F0F7FF000EF86E0F0EF76409D0090030
:1065D0006F00D4FF38F009006F00D4FF39F00CD001
:1065E0006F00DBFFE9FF6F00DFFFEAFF6F00B8FF1E
:1065F00038F06F00B8FF39F06000E3F0E6FF6000AC
:10660000E7F0E6FFFB0EE3503C0F386EFC0E6F0028
:106610008CFF39F0000E39226000E3F0F6FF6000D5
:10662000E7F0F7FF000EF86E0F0EF76409D00900CF
:106630006F00D4FF38F009006F00D4FF39F00CD0A0
:106640006F00DBFFE9FF6F00DFFFEAFF6F00B8FFBD
:1066500038F06F00B8FF39F002D838EF33F005009A
:10666000FA6E3850FD6E3950FE6EFF6AFA50120015
:1066700008EF34F0FD0EE350400F386EFE0E6F0051
:106680008CFF39F0000E39226000E3F0F6FF600065
:10669000E7F0F7FF000EF86E0F0EF76409D009005F
:1066A0006F00D4FF38F009006F00D4FF39F00CD030
:1066B0006F00DBFFE9FF6F00DFFFEAFF6F00B8FF4D
:1066C00038F06F00B8FF39F038503910D8B46BEF9C
:1066D00033F06DEF33F008EF34F0FD0EE350420F6E
:1066E000386EFE0E6F008CFF39F0000E392260000C
:1066F000E3F0F6FF6000E7F0F7FF000EF86E0F0E14
:10670000F76409D009006F00D4FF38F009006F006A
:10671000D4FF39F00CD06F00DBFFE9FF6F00DFFF23
:10672000EAFF6F00B8FF38F06F00B8FF39F0600083
:10673000E3F0E6FF6000E7F0E6FFFB0EE350400FFA
:10674000386EFC0E6F008CFF39F0000E39226000AD
:10675000E3F0F6FF6000E7F0F7FF000EF86E0F0EB3
:10676000F76409D009006F00D4FF38F009006F000A
:10677000D4FF39F00CD06F00DBFFE9FF6F00DFFFC3
:10678000EAFF6F00B8FF38F06F00B8FF39F002D8A9
:10679000D3EF33F00500FA6E3850FD6E3950FE6EBF
:1067A000FF6AFA50120008EF34F0FD0E6F008FFF01
:1067B000F6FFFE0E6F008FFFF7FF000EF86E0F0E54
:1067C000F76403D00800F55007D06F00DBFFE9FF46
:1067D0006F00DFFFEAFFEF50386E396A3950000A68
:1067E000D8B4F5EF33F008EF34F03850640AD8B479
:1067F00008EF34F0010AD8B4D3EF31F0030AD8B46B
:106800006EEF32F0010AD8B43AEF33F008EF34F00B
:10681000FB0EE126FF0EE2221200E652E652E6529D
:10682000FB0E6F008FFFE6FF6F008FFFE6FFCFECE0
:1068300062F0FE0E6000BFF0E3FFFD0E6000BBF0F3
:10684000E3FFFD0E6F008FFFF6FFFE0E6F008FFF60
:10685000F7FF000EF86E0F0EF76403D00800F55036
:1068600007D06F00DBFFE9FF6F00DFFFEAFFEF50AB
:10687000396EFF0E6000E7F0E3FFFB0E6F008FFF45
:10688000E6FF6F008FFFE6FF8FEC63F0FB0E6F00FB
:106890008FFFE6FF6F008FFFE6FF31EC62F0F80E2E
:1068A000E126FF0EE2222EEF35F0FB0E6F008FFF88
:1068B000D9FFFC0E6F008FFFDAFFDF506E0AD8A4FD
:1068C00064EF34F066EF34F061EF35F0FD0E6F00E9
:1068D0008FFFF6FFFE0E6F008FFFF7FF000EF86EC2
:1068E0000F0EF76404D06F0EF56E0C0008D06F0029
:1068F000DBFFE9FF6F00DFFFEAFF6F0EEF6EFD0EBB
:10690000E350010F386EFE0E6F008CFF39F0000E61
:1069100039226000E3F0E6FF6000E7F0E6FF0DECEF
:106920005FF061EF35F0FB0E6F008FFFD9FFFC0EBB
:106930006F008FFFDAFFDF506F0AD8A4A2EF34F0A8
:10694000A4EF34F061EF35F0FD0E6F008FFFF6FF1E
:10695000FE0E6F008FFFF7FF000EF86E0F0EF7644C
:1069600004D0700EF56E0C0008D06F00DBFFE9FF5D
:106970006F00DFFFEAFF700EEF6E61EF35F0FB0E88
:106980006F008FFFD9FFFC0E6F008FFFDAFFDF5023
:10699000700AD8A4CEEF34F0D0EF34F0E9EF34F041
:1069A000FD0E6F008FFFF6FFFE0E6F008FFFF7FFEB
:1069B000000EF86E0F0EF76404D0710EF56E0C0029
:1069C00008D06F00DBFFE9FF6F00DFFFEAFF710E09
:1069D000EF6EFB0E6F008FFFD9FFFC0E6F008FFF75
:1069E000DAFFDF50720AD8A4F8EF34F0FAEF34F08F
:1069F00061EF35F0CF0EE66E000EE66EFFEC53F061
:106A000061EF35F0FB0E6F008FFFD9FFFC0E6F00BA
:106A10008FFFDAFFDF50710AD8A411EF35F013EFC2
:106A200035F061EF35F0FD0E6F008FFFF6FFFE0EC3
:106A30006F008FFFF7FF000EF86E0F0EF76404D0A3
:106A40006F0EF56E0C0008D06F00DBFFE9FF6F00E2
:106A5000DFFFEAFF6F0EEF6E61EF35F0FD0E6F00A6
:106A60008FFFF6FFFE0E6F008FFFF7FF000EF86E30
:106A70000F0EF76403D00800F55007D06F00DBFF5E
:106A8000E9FF6F00DFFFEAFFEF50386E396A3950D7
:106A9000000AD8B44EEF35F061EF35F038506E0A89
:106AA000D8B455EF34F0010AD8B493EF34F01F0A8C
:106AB000D8B4BFEF34F0010AD8B402EF35F061EF7B
:106AC00035F0FF0E6F008CFF39F0FD0E6F008FFF69
:106AD000F6FFFE0E6F008FFFF7FF000EF86E0F0E31
:106AE000F76403D00800F55007D06F00DBFFE9FF23
:106AF0006F00DFFFEAFFEF503918D8B482EF35F0AE
:106B000084EF35F0E0EF37F0FF0EE350386E396A6E
:106B10003950000AD8B48FEF35F0ADEF37F0385068
:106B20006E0AD8B4ADEF37F0010AD8B4ADEF37F044
:106B30001F0AD8B4ADEF37F0010AD8B4ADEF37F083
:106B4000ADEF37F0FD0EE350380F386EFE0E6F00DC
:106B50008CFF39F0000E39226000E3F0F6FF600090
:106B6000E7F0F7FF000EF86E0F0EF76409D009008A
:106B70006F00D4FF38F009006F00D4FF39F00CD05B
:106B80006F00DBFFE9FF6F00DFFFEAFF6F00B8FF78
:106B900038F06F00B8FF39F038503910D8B4D3EF5F
:106BA00035F0D5EF35F03BEF36F0FD0EE3503A0F00
:106BB000386EFE0E6F008CFF39F0000E3922600037
:106BC000E3F0F6FF6000E7F0F7FF000EF86E0F0E3F
:106BD000F76409D009006F00D4FF38F009006F0096
:106BE000D4FF39F00CD06F00DBFFE9FF6F00DFFF4F
:106BF000EAFF6F00B8FF38F06F00B8FF39F06000AF
:106C0000E3F0E6FF6000E7F0E6FFFB0EE350380F2D
:106C1000386EFC0E6F008CFF39F0000E39226000D8
:106C2000E3F0F6FF6000E7F0F7FF000EF86E0F0EDE
:106C3000F76409D009006F00D4FF38F009006F0035
:106C4000D4FF39F00CD06F00DBFFE9FF6F00DFFFEE
:106C5000EAFF6F00B8FF38F06F00B8FF39F002D8D4
:106C60003BEF36F00500FA6E3850FD6E3950FE6E7F
:106C7000FF6AFA5012001950E66EFC0EE350010F45
:106C8000386EFD0E6F008CFF39F0000E3922600067
:106C9000E3F0E6FF6000E7F0E6FFFEEC5FF0000ED9
:106CA000E66E000EE66E000EE66E000EE66E000E5C
:106CB000E66E000EE66E000EE66E000EE66EF40E58
:106CC000E66E010EE66EF30EE350010F386EF40E21
:106CD0006F008CFF39F0000E39226000E3F0E6FF10
:106CE0006000E7F0E6FF3DEC5DF0E0EF37F0FD0E11
:106CF000E3503C0F386EFE0E6F008CFF39F0000E33
:106D000039226000E3F0F6FF6000E7F0F7FF000EC5
:106D1000F86E0F0EF76409D009006F00D4FF38F049
:106D200009006F00D4FF39F00CD06F00DBFFE9FFE2
:106D30006F00DFFFEAFF6F00B8FF38F06F00B8FFA9
:106D400039F038503910D8B4A8EF36F0AAEF36F041
:106D5000E0EF37F0FD0EE3503E0F386EFE0E6F0091
:106D60008CFF39F0000E39226000E3F0F6FF60007E
:106D7000E7F0F7FF000EF86E0F0EF76409D0090078
:106D80006F00D4FF38F009006F00D4FF39F00CD049
:106D90006F00DBFFE9FF6F00DFFFEAFF6F00B8FF66
:106DA00038F06F00B8FF39F06000E3F0E6FF6000F4
:106DB000E7F0E6FFFB0EE3503C0F386EFC0E6F0071
:106DC0008CFF39F0000E39226000E3F0F6FF60001E
:106DD000E7F0F7FF000EF86E0F0EF76409D0090018
:106DE0006F00D4FF38F009006F00D4FF39F00CD0E9
:106DF0006F00DBFFE9FF6F00DFFFEAFF6F00B8FF06
:106E000038F06F00B8FF39F002D810EF37F0050006
:106E1000FA6E3850FD6E3950FE6EFF6AFA5012005D
:106E2000E0EF37F0FD0EE350400F386EFE0E6F00BE
:106E30008CFF39F0000E39226000E3F0F6FF6000AD
:106E4000E7F0F7FF000EF86E0F0EF76409D00900A7
:106E50006F00D4FF38F009006F00D4FF39F00CD078
:106E60006F00DBFFE9FF6F00DFFFEAFF6F00B8FF95
:106E700038F06F00B8FF39F038503910D8B443EF0C
:106E800037F045EF37F0E0EF37F0FD0EE350420FFB
:106E9000386EFE0E6F008CFF39F0000E3922600054
:106EA000E3F0F6FF6000E7F0F7FF000EF86E0F0E5C
:106EB000F76409D009006F00D4FF38F009006F00B3
:106EC000D4FF39F00CD06F00DBFFE9FF6F00DFFF6C
:106ED000EAFF6F00B8FF38F06F00B8FF39F06000CC
:106EE000E3F0E6FF6000E7F0E6FFFB0EE350400F43
:106EF000386EFC0E6F008CFF39F0000E39226000F6
:106F0000E3F0F6FF6000E7F0F7FF000EF86E0F0EFB
:106F1000F76409D009006F00D4FF38F009006F0052
:106F2000D4FF39F00CD06F00DBFFE9FF6F00DFFF0B
:106F3000EAFF6F00B8FF38F06F00B8FF39F002D8F1
:106F4000ABEF37F00500FA6E3850FD6E3950FE6E2B
:106F5000FF6AFA501200E0EF37F0FD0E6F008FFF6E
:106F6000F6FFFE0E6F008FFFF7FF000EF86E0F0E9C
:106F7000F76403D00800F55007D06F00DBFFE9FF8E
:106F80006F00DFFFEAFFEF50386E396A3950000AB0
:106F9000D8B4CDEF37F0E0EF37F038506E0AD8B400
:106FA000E0EF37F0010AD8B4A2EF35F01F0AD8B4E9
:106FB00077EF36F0010AD8B412EF37F0E0EF37F090
:106FC000FB0EE126FF0EE2221200E652E652E652E6
:106FD000E652FF0EE36AFE0EE36AFD0EE36AFC0E64
:106FE000E36A3701E0B7F7EF37F0F9EF37F00DEF6D
:106FF00039F0FC0EE1242E6EFF0EE2202F6E6000B1
:10700000BBF0E6FF6000BFF0E6FFFB0EE1242E6E52
:10701000FF0EE2202F6E6000BBF0E6FF6000BFF0C5
:10702000E6FFFA0EE1242E6EFF0EE2202F6E6000C6
:10703000BBF0E6FF6000BFF0E6FFF90EE1242E6E24
:10704000FF0EE2202F6E6000BBF0E6FF6000BFF095
:10705000E6FFF20E6F008FFFD9FFF30E6F008FFF78
:10706000DAFFDF50E66EF10E6F008CFF38F0F20EA3
:107070006F008CFF39F0010E3824D96E000E3920D4
:10708000DA6E6F007BFFE6FF6F007BFFE6FF6F00AD
:107090007BFFE6FF6F007BFFE6FF22EC47F0FF0E71
:1070A0006F008FFFE3F7FE0E6F008FFFE4F7FD0E1A
:1070B0006F008FFFE1F7FC0E6F008FFFE2F7FA0E13
:1070C0006F008CFF38F0FB0E6F008CFF39F0050E5F
:1070D0003824D96E000E3920DA6EDF50396EFA0E80
:1070E0006F008CFF36F0FB0E6F008CFF37F00E0E3A
:1070F0003624D96E000E3720DA6EDF50386E060E59
:107100002E6ED89038362E2E81EF38F03850391048
:107110003701E56FFA0E6F008CFF38F0FB0E6F0041
:107120008CFF39F0060E3824D96E000E3920DA6E45
:10713000DF50E66FFA0E6F008CFF38F0FB0E6F0029
:107140008CFF39F0070E3824D96E000E3920DA6E24
:10715000DF50E76FFA0E6F008CFF38F0FB0E6F0008
:107160008CFF39F0080E3824D96E000E3920DA6E03
:10717000DF50E86FFA0E6F008CFF38F0FB0E6F00E7
:107180008CFF39F0090E3824D96E000E3920DA6EE2
:10719000DF50E96FFA0E6F008CFF38F0FB0E6F00C6
:1071A0008CFF39F00A0E3824D96E000E3920DA6EC1
:1071B000DF50EA6FFA0E6F008CFF38F0FB0E6F00A5
:1071C0008CFF39F00B0E3824D96E000E3920DA6EA0
:1071D000DF50EB6FFA0E6F008CFF38F0FB0E6F0084
:1071E0008CFF39F00C0E3824D96E000E3920DA6E7F
:1071F000DF50EC6FFA0E6F008CFF38F0FB0E6F0063
:107200008CFF39F00D0E3824D96E000E3920DA6E5D
:10721000DF50ED6FE08743EF3BF0D0B712EF39F06E
:1072200014EF39F028EF3AF0FC0EE1242E6EFF0E39
:10723000E2202F6E6000BBF0E6FF6000BFF0E6FFCB
:10724000FB0EE1242E6EFF0EE2202F6E6000BBF0DD
:10725000E6FF6000BFF0E6FFFA0EE1242E6EFF0E9F
:10726000E2202F6E6000BBF0E6FF6000BFF0E6FF9B
:10727000F90EE1242E6EFF0EE2202F6E6000BBF0AF
:10728000E6FF6000BFF0E6FFF20E6F008FFFD9FF50
:10729000F30E6F008FFFDAFFDF50E66EF10E6F0026
:1072A0008CFF38F0F20E6F008CFF39F0010E38249D
:1072B000D96E000E3920DA6E6F007BFFE6FF6F009B
:1072C0007BFFE6FF6F007BFFE6FF6F007BFFE6FFC3
:1072D00022EC47F0FF0E6F008FFFD3F7FE0E6F001A
:1072E0008FFFD4F7FD0E6F008FFFD1F7FC0E6F00FC
:1072F0008FFFD2F7FA0E6F008CFF38F0FB0E6F0095
:107300008CFF39F0050E3824D96E000E3920DA6E64
:10731000DF50396EFA0E6F008CFF36F0FB0E6F00F7
:107320008CFF37F00E0E3624D96E000E3720DA6E41
:10733000DF50386E060E2E6ED89038362E2E9CEF0B
:1073400039F0385039103701D56FFA0E6F008CFFC5
:1073500038F0FB0E6F008CFF39F0060E3824D96E22
:10736000000E3920DA6EDF50D66FFA0E6F008CFFF8
:1073700038F0FB0E6F008CFF39F0070E3824D96E01
:10738000000E3920DA6EDF50D76FFA0E6F008CFFD7
:1073900038F0FB0E6F008CFF39F0080E3824D96EE0
:1073A000000E3920DA6EDF50D86FFA0E6F008CFFB6
:1073B00038F0FB0E6F008CFF39F0090E3824D96EBF
:1073C000000E3920DA6EDF50D96FFA0E6F008CFF95
:1073D00038F0FB0E6F008CFF39F00A0E3824D96E9E
:1073E000000E3920DA6EDF50DA6FFA0E6F008CFF74
:1073F00038F0FB0E6F008CFF39F00B0E3824D96E7D
:10740000000E3920DA6EDF50DB6FFA0E6F008CFF52
:1074100038F0FB0E6F008CFF39F00C0E3824D96E5B
:10742000000E3920DA6EDF50DC6FFA0E6F008CFF31
:1074300038F0FB0E6F008CFF39F00D0E3824D96E3A
:10744000000E3920DA6EDF50DD6FD0870BEF39F098
:10745000C0B72DEF3AF02FEF3AF043EF3BF0FC0EC0
:10746000E1242E6EFF0EE2202F6E6000BBF0E6FFDF
:107470006000BFF0E6FFFB0EE1242E6EFF0EE2205F
:107480002F6E6000BBF0E6FF6000BFF0E6FFFA0E73
:10749000E1242E6EFF0EE2202F6E6000BBF0E6FFAF
:1074A0006000BFF0E6FFF90EE1242E6EFF0EE22031
:1074B0002F6E6000BBF0E6FF6000BFF0E6FFF20E4B
:1074C0006F008FFFD9FFF30E6F008FFFDAFFDF50E1
:1074D000E66EF10E6F008CFF38F0F20E6F008CFF3D
:1074E00039F0010E3824D96E000E3920DA6E6F00A3
:1074F0007BFFE6FF6F007BFFE6FF6F007BFFE6FF91
:107500006F007BFFE6FF22EC47F0FF0E6F008FFF5E
:10751000C3F7FE0E6F008FFFC4F7FD0E6F008FFFE5
:10752000C1F7FC0E6F008FFFC2F7FA0E6F008CFFE1
:1075300038F0FB0E6F008CFF39F0050E3824D96E41
:10754000000E3920DA6EDF50396EFA0E6F008CFFB4
:1075500036F0FB0E6F008CFF37F00E0E3624D96E1E
:10756000000E3720DA6EDF50386E060E2E6ED89081
:1075700038362E2EB7EF3AF0385039103701C56F34
:10758000FA0E6F008CFF38F0FB0E6F008CFF39F0A5
:10759000060E3824D96E000E3920DA6EDF50C66F21
:1075A000FA0E6F008CFF38F0FB0E6F008CFF39F085
:1075B000070E3824D96E000E3920DA6EDF50C76FFF
:1075C000FA0E6F008CFF38F0FB0E6F008CFF39F065
:1075D000080E3824D96E000E3920DA6EDF50C86FDD
:1075E000FA0E6F008CFF38F0FB0E6F008CFF39F045
:1075F000090E3824D96E000E3920DA6EDF50C96FBB
:10760000FA0E6F008CFF38F0FB0E6F008CFF39F024
:107610000A0E3824D96E000E3920DA6EDF50CA6F98
:10762000FA0E6F008CFF38F0FB0E6F008CFF39F004
:107630000B0E3824D96E000E3920DA6EDF50CB6F76
:10764000FA0E6F008CFF38F0FB0E6F008CFF39F0E4
:107650000C0E3824D96E000E3920DA6EDF50CC6F54
:10766000FA0E6F008CFF38F0FB0E6F008CFF39F0C4
:107670000D0E3824D96E000E3920DA6EDF50CD6F32
:10768000C0870BEF39F0FA0EE126FF0EE22212005E
:10769000080EE126000EE2226000ACF03EF03F6AE8
:1076A000406A416A426A436A446A456AF80E600069
:1076B000FBF0E3FFF90E6000FFF0E3FFFA0E60005D
:1076C00003F1E3FFFB0E600007F1E3FFFC0E600037
:1076D0000BF1E3FFFD0E60000FF1E3FFFE0E600013
:1076E00013F1E3FFFF0E600017F1E3FFF80E6F00E8
:1076F0008CFF3EF0F90E6F008CFF3FF0FA0E6F002A
:107700008CFF40F0FB0E6F008CFF41F0FC0E6F0011
:107710008CFF42F0FD0E6F008CFF43F0FE0E6F00F9
:107720008CFF44F0FF0E6F008CFF45F0040ED890E4
:107730003E363F364036413642364336443645368D
:10774000E82E97EF3BF0F70EE3503E10466E3F50A9
:10775000476E4050486E4150496E42504A6E435009
:107760004B6E44504C6E45504D6EF80E60001BF150
:10777000E3FFF90E60001FF1E3FFFA0E600023F152
:10778000E3FFFB0E600027F1E3FFFC0E60002BF12E
:10779000E3FFFD0E60002FF1E3FFFE0E600033F10A
:1077A000E3FFFF0E600037F1E3FFF80E6F008CFF80
:1077B0003EF0F90E6F008CFF3FF0FA0E6F008CFF69
:1077C00040F0FB0E6F008CFF41F0FC0E6F008CFF51
:1077D00042F0FD0E6F008CFF43F0FE0E6F008CFF39
:1077E00044F0FF0E6F008CFF45F0040ED8903E363B
:1077F0003F36403641364236433644364536E82E2B
:10780000F6EF3BF0F60EE3503E10466E3F50476EEB
:107810004050486E4150496E42504A6E43504B6E44
:1078200044504C6E45504D6EF80E60001BF1E3FF66
:10783000F90E60001FF1E3FFFA0E600023F1E3FF91
:10784000FB0E600027F1E3FFFC0E60002BF1E3FF6D
:10785000FD0E60002FF1E3FFFE0E600033F1E3FF49
:10786000FF0E600037F1E3FFF20E6F008CFF36F081
:10787000F30E6F008CFF37F0F40E6F008CFF38F0C2
:10788000F50E6F008CFF39F036503E6E37503F6E6C
:107890003850406E3950416E426A436A446A456AC4
:1078A000F80E6F008CFF46F0F90E6F008CFF47F06A
:1078B000FA0E6F008CFF48F0FB0E6F008CFF49F052
:1078C000FC0E6F008CFF4AF0FD0E6F008CFF4BF03A
:1078D000FE0E6F008CFF4CF0FF0E6F008CFF4DF022
:1078E000200ED89046364736483649364A364B360B
:1078F0004C364D36E82E71EF3CF03E504610366E59
:107900003F504710376E40504810386E4150491074
:10791000396E42504A103A6E43504B103B6E445001
:107920004C103C6E45504D103D6EF80E6000DBF083
:10793000E3FFF90E6000DFF0E3FFFA0E6000E3F012
:10794000E3FFFB0E6000E7F0E3FFFC0E6000EBF0EE
:10795000E3FFFD0E6000EFF0E3FFFE0E6000F3F0CA
:10796000E3FFFF0E6000F7F0E3FFE150F80FD96E80
:10797000E250DA6EFF0EDA226F007BFFE6FF6F0047
:107980007BFFE6FF6F007BFFE6FF6F007BFFE6FFFC
:107990006F007BFFE6FF6F007BFFE6FF6F007BFF62
:1079A000E6FF6F007BFFE6FF000EE66E000EE66E60
:1079B0000D0EE66E9E0EE66E350EE66E2A0EE66E35
:1079C000000EE66E01EC4EF0F20EE126FF0EE22212
:1079D0001200E652000EE66E6BEC64F0FF0E6000E3
:1079E000BBF0E3FFFF0E6F008CFF2EF0420E2E184F
:1079F000D8B4FDEF3CF0FFEF3CF0E5EF3DF0016A5D
:107A0000320E026E070E036EB20E046E010E056E8C
:107A1000000E066E100E076E270E086E000E096E21
:107A2000000E0A6EF00E0B6E730E0C6E550E0D6E80
:107A3000000E0E6E320E0F6E190E106E116A050ECC
:107A4000126E010E136E190E146E640E156E140E66
:107A5000166E0A0E176EFA0E186E640E196E320E3E
:107A60001A6E320E1B6E320E1C6E320E1D6E0A0E18
:107A70001E6E0A0E1F6E0150E66E010EE66EA9EC38
:107A800063F00250E66E020EE66EA9EC63F0600051
:107A90000FF0E6FF600013F0E6FF600017F0E6FF6E
:107AA00060001BF0E6FF030EE66E73EC57F060001B
:107AB0001FF0E6FF600023F0E6FF600027F0E6FF1E
:107AC00060002BF0E6FF070EE66E73EC57F06000E7
:107AD0002FF0E6FF600033F0E6FF600037F0E6FFCE
:107AE00060003BF0E6FF0B0EE66E73EC57F00F50B4
:107AF000E66E0F0EE66EA9EC63F01050E66E100E07
:107B0000E66EA9EC63F01150E66E110EE66EA9EC7C
:107B100063F01250E66E120EE66EA9EC63F013509D
:107B2000E66E130EE66EA9EC63F01450E66E140ECA
:107B3000E66EA9EC63F01550E66E150EE66EA9EC44
:107B400063F01650E66E160EE66EA9EC63F0175061
:107B5000E66E170EE66EA9EC63F01850E66E180E8E
:107B6000E66EA9EC63F01950E66E190EE66EA9EC0C
:107B700063F01A50E66E1A0EE66EA9EC63F01B5025
:107B8000E66E1B0EE66EA9EC63F01C50E66E1C0E52
:107B9000E66EA9EC63F01D50E66E1D0EE66EA9ECD4
:107BA00063F01F50E66E1F0EE66EA9EC63F01E50E8
:107BB000E66E1E0EE66EA9EC63F0420EE66E000E57
:107BC000E66EA9EC63F087EF3EF0010EE66E6BEC1B
:107BD00064F02E50016E020EE66E6BEC64F02E50D7
:107BE000026E030EE66ED5EC57F06000B8F003F0BD
:107BF0006000BCF004F06000C0F005F06000C4F06C
:107C000006F0070EE66ED5EC57F06000B8F007F00E
:107C10006000BCF008F06000C0F009F06000C4F043
:107C20000AF00B0EE66ED5EC57F06000B8F00BF0E2
:107C30006000BCF00CF06000C0F00DF06000C4F01B
:107C40000EF00F0EE66E6BEC64F02E500F6E100E01
:107C5000E66E6BEC64F02E50106E110EE66E6BEC5F
:107C600064F02E50116E120EE66E6BEC64F02E5026
:107C7000126E130EE66E6BEC64F02E50136E140E43
:107C8000E66E6BEC64F02E50146E150EE66E6BEC27
:107C900064F02E50156E160EE66E6BEC64F02E50EE
:107CA000166E170EE66E6BEC64F02E50176E180E03
:107CB000E66E6BEC64F02E50186E190EE66E6BECEF
:107CC00064F02E50196E1A0EE66E6BEC64F02E50B6
:107CD0001A6E1B0EE66E6BEC64F02E501B6E1C0EC3
:107CE000E66E6BEC64F02E501C6E1D0EE66E6BECB7
:107CF00064F02E501D6E1F0EE66E6BEC64F02E507D
:107D00001F6E1E0EE66E6BEC64F02E501E6EE5527A
:107D100012000001606B030E616F050E626F070EAB
:107D2000636F0A0E646F0C0E656F0E0E666F100E99
:107D3000676F120E686F140E696F160E6A6F180E59
:107D40006B6F190E6C6F1B0E6D6F1C0E6E6F1E0E1F
:107D50006F6F1F0E706F210E716F220E726F240EE7
:107D6000736F250E746F260E756F270E766F280EB3
:107D7000776F290E786F2A0E796F2B0E7A6F2C0E83
:107D80007B6F2D0E7C6F2E0E7D6F2F0E7E6F2F0E54
:107D90007F6F300E806F310E816F320E826F320E28
:107DA000836F330E846F330E856F340E866F350EFE
:107DB000876F350E886F350E896F360E8A6F360ED7
:107DC0008B6F370E8C6F370E8D6F380E8E6F380EAF
:107DD0008F6F380E906F390E916F390E926F3A0E89
:107DE000936F3A0E946F3A0E956F3B0E966F3B0E63
:107DF000976F3B0E986F3C0E996F3C0E9A6F3C0E3E
:107E00009B6F3D0E9C6F3D0E9D6F3E0E9E6F3E0E16
:107E10009F6F3E0EA06F3F0EA16F3F0EA26F400EF0
:107E2000A36F400EA46F410EA56F410EA66F420EC8
:107E3000A76F430EA86F430EA96F440EAA6F450E9D
:107E4000AB6F450EAC6F460EAD6F470EAE6F480E72
:107E5000AF6F480EB06F490EB16F4A0EB26F4B0E46
:107E6000B36F4C0EB46F4D0EB56F4E0EB66F500E15
:107E7000B76F510EB86F520EB96F530EBA6F550EE1
:107E8000BB6F560EBC6F580EBD6F590EBE6F5B0EAA
:107E9000BF6F5D0EC06F5E0EC16F600EC26F620E6F
:107EA000C36F640EC46F0101006B016B026B036B47
:107EB000046B010E056F010E066F010E076F020EB7
:107EC000086F020E096F030E0A6F030E0B6F040E8C
:107ED0000C6F050E0D6F050E0E6F060E0F6F070E61
:107EE000106F080E116F090E126F090E136F0A0E34
:107EF000146F0B0E156F0C0E166F0D0E176F0F0E05
:107F0000186F100E196F110E1A6F120E1B6F130ED1
:107F10001C6F140E1D6F160E1E6F170E1F6F180E9E
:107F2000206F190E216F1B0E226F1C0E236F1E0E69
:107F3000246F1F0E256F200E266F220E276F230E33
:107F4000286F250E296F260E2A6F280E2B6F290EFB
:107F50002C6F2B0E2D6F2C0E2E6F2E0E2F6F2F0EC3
:107F6000306F310E316F320E326F330E336F350E8C
:107F7000346F360E356F380E366F390E376F3B0E55
:107F8000386F3C0E396F3E0E3A6F3F0E3B6F410E1D
:107F90003C6F420E3D6F440E3E6F450E3F6F460EE6
:107FA000406F480E416F490E426F4B0E436F4C0EAF
:107FB000446F4D0E456F4E0E466F500E476F510E7B
:107FC000486F520E496F530E4A6F540E4B6F550E49
:107FD0004C6F570E4D6F580E4E6F590E4F6F5A0E15
:107FE000506F5B0E516F5B0E526F5C0E536F5D0EE8
:107FF000546F5E0E556F5F0E566F5F0E576F600EBB
:10800000586F610E596F610E5A6F620E5B6F620E90
:108010005C6F630E5D6F630E5E6F630E5F6F640E69
:10802000606F640E616F640E626F640E636F640E46
:10803000646F1200170EE126000EE222E90EE12421
:108040002E6EFF0EE2202F6E6000BBF0E6FF600098
:10805000BFF0E6FFC5EC11F0EA0EE124D96EFF0E89
:10806000E220DA6E6F0078FF36F06F0078FF37F0AD
:108070006F0078FF38F06F0078FF39F036503E6EB1
:1080800037503F6E3850406E3950416E426A436AF5
:10809000446A456AF80E6000FBF0E3FFF90E6000E9
:1080A000FFF0E3FFFA0E600003F1E3FFFB0E600058
:1080B00007F1E3FFFC0E60000BF1E3FFFD0E600033
:1080C0000FF1E3FFFE0E600013F1E3FFFF0E60000F
:1080D00017F1E3FFE150F80FD96EE250DA6EFF0EB0
:1080E000DA220C0ED890DE36DE36DE36DE36DE36AE
:1080F000DE36DE36DD36DD52DD52DD52DD52DD525A
:10810000DD52E82E72EF40F0E150F80FD96EE250E8
:10811000DA6EFF0EDA22F20EE124E96EFF0EE220A3
:10812000EA6EEF50DE12000EDE12DE12DE12DE12FA
:10813000DE12DE12DE12E150F80FD96EE250DA6E76
:10814000FF0EDA22080ED890DE36DE36DE36DE3658
:10815000DE36DE36DE36DD36DD52DD52DD52DD5214
:10816000DD52DD52E82EA3EF40F0E150F80FD96E5A
:10817000E250DA6EFF0EDA22F10EE124E96EFF0E14
:10818000E220EA6EEF50DE12000EDE12DE12DE1288
:10819000DE12DE12DE12DE12E150F80FD96EE2506E
:1081A000DA6EFF0EDA22080ED890DE36DE36DE36C4
:1081B000DE36DE36DE36DE36DD36DD52DD52DD52CF
:1081C000DD52DD52DD52E82ED4EF40F0E150F80FE1
:1081D000D96EE250DA6EFF0EDA22F00EE124E96E7B
:1081E000FF0EE220EA6EEF50DE12000EDE12DE120B
:1081F000DE12DE12DE12DE12DE12E150F80FD96E50
:10820000E250DA6EFF0EDA22080ED890DE36DE3645
:10821000DE36DE36DE36DE36DE36DD36DD52DD5289
:10822000DD52DD52DD52DD52E82E05EF41F0E15026
:10823000F80FD96EE250DA6EFF0EDA22EF0EE1246B
:10824000E96EFF0EE220EA6EEF50DE12000EDE1243
:10825000DE12DE12DE12DE12DE12DE12F70EE12474
:10826000D96EFF0EE220DA6EDF50D8B43AEF41F05B
:108270003CEF41F06DEF41F0E150F80FD96EE25064
:10828000DA6EFF0EDA226F007BFFE6FF6F007BFFE6
:10829000E6FF6F007BFFE6FF6F007BFFE6FF6F00EE
:1082A0007BFFE6FF6F007BFFE6FF6F007BFFE6FFD3
:1082B0006F007BFFE6FF000EE66E000EE66E0C0E12
:1082C000E66E9E0EE66E350EE66E2A0EE66E000E29
:1082D000E66E01EC4EF09CEF41F0E150F80FD96EE4
:1082E000E250DA6EFF0EDA226F007BFFE6FF6F00CE
:1082F0007BFFE6FF6F007BFFE6FF6F007BFFE6FF83
:108300006F007BFFE6FF6F007BFFE6FF6F007BFFE8
:10831000E6FF6F007BFFE6FF000EE66E000EE66EE6
:108320000B0EE66E9E0EE66E350EE66E2A0EE66EBD
:10833000000EE66E01EC4EF0E90EE126FF0EE222A1
:108340001200080EE126000EE2226000ACF03EF0C2
:108350003F6A406A416A426A436A446A456AF80E63
:108360006000FBF0E3FFF90E6000FFF0E3FFFA0EA0
:10837000600003F1E3FFFB0E600007F1E3FFFC0E7A
:1083800060000BF1E3FFFD0E60000FF1E3FFFE0E56
:10839000600013F1E3FFFF0E600017F1E3FFF80E3A
:1083A0006F008CFF3EF0F90E6F008CFF3FF0FA0E6D
:1083B0006F008CFF40F0FB0E6F008CFF41F0FC0E55
:1083C0006F008CFF42F0FD0E6F008CFF43F0FE0E3D
:1083D0006F008CFF44F0FF0E6F008CFF45F0040E21
:1083E000D8903E363F3640364136423643364436E4
:1083F0004536E82EF0EF41F0F70EE3503E10466EA2
:108400003F50476E4050486E4150496E42504A6E50
:1084100043504B6E44504C6E45504D6EF80E60000C
:108420001BF1E3FFF90E60001FF1E3FFFA0E60009D
:1084300023F1E3FFFB0E600027F1E3FFFC0E600079
:108440002BF1E3FFFD0E60002FF1E3FFFE0E600055
:1084500033F1E3FFFF0E600037F1E3FFF80E6F002A
:108460008CFF3EF0F90E6F008CFF3FF0FA0E6F00AC
:108470008CFF40F0FB0E6F008CFF41F0FC0E6F0094
:108480008CFF42F0FD0E6F008CFF43F0FE0E6F007C
:108490008CFF44F0FF0E6F008CFF45F0040ED89067
:1084A0003E363F3640364136423643364436453610
:1084B000E82E4FEF42F0F60EE3503E10466E3F506E
:1084C000476E4050486E4150496E42504A6E43508C
:1084D0004B6E44504C6E45504D6EF80E60001BF1D3
:1084E000E3FFF90E60001FF1E3FFFA0E600023F1D5
:1084F000E3FFFB0E600027F1E3FFFC0E60002BF1B1
:10850000E3FFFD0E60002FF1E3FFFE0E600033F18C
:10851000E3FFFF0E600037F1E3FFF80E6F008CFF02
:108520003EF0F90E6F008CFF3FF0FA0E6F008CFFEB
:1085300040F0FB0E6F008CFF41F0FC0E6F008CFFD3
:1085400042F0FD0E6F008CFF43F0FE0E6F008CFFBB
:1085500044F0FF0E6F008CFF45F0200ED8903E36A1
:108560003F36403641364236433644364536E82EAD
:10857000AEEF42F0F50EE3503E10466E3F50476EB0
:108580004050486E4150496E42504A6E43504B6EC7
:1085900044504C6E45504D6EF80E60001BF1E3FFE9
:1085A000F90E60001FF1E3FFFA0E600023F1E3FF14
:1085B000FB0E600027F1E3FFFC0E60002BF1E3FFF0
:1085C000FD0E60002FF1E3FFFE0E600033F1E3FFCC
:1085D000FF0E600037F1E3FFE150F80FD96EE25073
:1085E000DA6EFF0EDA226F007BFFE6FF6F007BFF83
:1085F000E6FF6F007BFFE6FF6F007BFFE6FF6F008B
:108600007BFFE6FF6F007BFFE6FF6F007BFFE6FF6F
:108610006F007BFFE6FF000EE66E000EE66E0F0EAB
:10862000E66E9E0EE66E350EE66E2A0EE66E000EC5
:10863000E66E01EC4EF0F50EE126FF0EE22212008E
:10864000E652E652E652E652FB0EE350366E000E5C
:1086500036BEFF0E376E386E396EFC0E6000DBF0F2
:10866000E3FFFD0E6000DFF0E3FFFE0E6000E3F0CD
:10867000E3FFFF0E6000E7F0E3FFFF0EE66EFF0E84
:10868000E66EFF0EE66EFF0EE66EF80E6F008FFFD1
:10869000E6FF6F008FFFE6FF6F008FFFE6FF6F00C2
:1086A0008FFFE6FF8AEC53F0FC0E6000BBF0E3FFA7
:1086B000FD0E6000BFF0E3FFFE0E6000C3F0E3FFBD
:1086C000FF0E6000C7F0E3FF020E0001D519D8A429
:1086D0006CEF43F06EEF43F012EF44F0FF0EE3BE99
:1086E00074EF43F076EF43F09EEF43F0FC0E6F0023
:1086F0008CFF38F0FD0E6F008CFF39F0000E38242F
:10870000D96E010E3920DA6EDF50396E6000E4F068
:1087100032F0336A346A356AFC0E6000CBF0E3FF56
:10872000FD0E6000CFF0E3FFFE0E6000D3F0E3FF2C
:10873000FF0E6000D7F0E3FF12EF44F0FF0EE66E8D
:10874000FF0EE66EFF0EE66EFF0EE66EF80E6F0091
:108750008FFFE6FF6F008FFFE6FF6F008FFFE6FFE2
:108760006F008FFFE6FF8AEC53F0FC0E6000BBF059
:10877000E3FFFD0E6000BFF0E3FFFE0E6000C3F0FC
:10878000E3FFFF0E6000C7F0E3FFFC0E6F008CFFFD
:1087900038F0FD0E6F008CFF39F0000E3824D96ED2
:1087A000010E3920DA6EDF50396E6000E4F032F0ED
:1087B000336A346A356AFC0E6000CBF0E3FFFD0ECD
:1087C0006000CFF0E3FFFE0E6000D3F0E3FFFF0E8A
:1087D0006000D7F0E3FFFF0EE66EFF0EE66EFF0EC1
:1087E000E66EFF0EE66EF80E6F008FFFE6FF6F007D
:1087F0008FFFE6FF6F008FFFE6FF6F008FFFE6FF42
:108800008AEC53F0FC0E6000BBF0E3FFFD0E60004D
:10881000BFF0E3FFFE0E6000C3F0E3FFFF0E600059
:10882000C7F0E3FF60002FF0E6FF600033F0E6FFE3
:10883000600037F0E6FF60003BF0E6FFF80E6F00E7
:108840008FFFE6FF6F008FFFE6FF6F008FFFE6FFF1
:108850006F008FFFE6FF8AEC53F0FC0E6000BBF068
:10886000E3FFFD0E6000BFF0E3FFFE0E6000C3F00B
:10887000E3FFFF0E6000C7F0E3FFE80EE66E030EB5
:10888000E66E000EE66E000EE66EF80E6F008FFFCD
:10889000E6FF6F008FFFE6FF6F008FFFE6FF6F00C0
:1088A0008FFFE6FF40EC48F0FC0E6000BBF0E3FFFA
:1088B000FD0E6000BFF0E3FFFE0E6000C3F0E3FFBB
:1088C000FF0E6000C7F0E3FFE150FC0FD96EE250ED
:1088D000DA6EFF0EDA220001CB51DE26CC51DE2209
:1088E000CD51DE22CE51DE22E150FC0FD96EE25096
:1088F000DA6EFF0EDA226F0078FFCFF06F0078FF9C
:10890000D0F06F0078FFD1F06F0078FFD2F0FB0E4F
:10891000E126FF0EE2221200FE0E6F008FFFD9FF4C
:10892000FF0E6F008FFFDAFF140EDF6EFE0E6F007A
:108930008CFF38F0FF0E6F008CFF39F01A0E3824D0
:10894000D96E000E3920DA6EDF6AFE0E6F008CFFE2
:1089500038F0FF0E6F008CFF39F01B0E3824D96EF3
:10896000000E3920DA6EDF6AFE0E6F008CFF38F0E1
:10897000FF0E6F008CFF39F01C0E3824D96E000EEC
:108980003920DA6EDF6AFE0E6F008CFF38F0FF0EC2
:108990006F008CFF39F01D0E3824D96E000E39207F
:1089A000DA6E010EDF6EFE0E6F008CFF38F0FF0EE8
:1089B0006F008CFF39F01E0E3824D96E000E39205E
:1089C000DA6E0A0EDF6EFE0E6F008CFF38F0FF0EBF
:1089D0006F008CFF39F01F0E3824D96E000E39203D
:1089E000DA6EDE6ADD6AFE0E6F008CFF38F0FF0E75
:1089F0006F008CFF39F0230E3824D96E000E392019
:108A0000DA6EDE6ADD6AFE0E6F008CFF38F0FF0E54
:108A10006F008CFF39F0270E3824D96E000E3920F4
:108A2000DA6EDE6ADD6AFE0E6F008CFF38F0FF0E34
:108A30006F008CFF39F02B0E3824D96E000E3920D0
:108A4000DA6EDE6ADD6AFE0E6F008CFF38F0FF0E14
:108A50006F008CFF39F02F0E3824D96E000E3920AC
:108A6000DA6EDE6ADD6AFE0E6F008CFF38F0FF0EF4
:108A70006F008CFF39F0330E3824D96E000E392088
:108A8000DA6EDE6ADD6AFD0EE350E66EFD0EE3503F
:108A9000010F386EFE0E6F008CFF39F0000E392288
:108AA0006000E3F0E6FF6000E7F0E6FF45EC63F00E
:108AB000FE0EE350010F386EFF0E6F008CFF39F091
:108AC000000E39226000E3F0E6FF6000E7F0E6FF09
:108AD000CEEC63F0FE0EE350020F386EFF0E6F0017
:108AE0008CFF39F0000E39226000E3F0E6FF6000F1
:108AF000E7F0E6FFC1EC50F0320EE66E000EE66ED7
:108B0000FC0EE350020F386EFD0E6F008CFF39F043
:108B1000000E39226000E3F0E6FF6000E7F0E6FFB8
:108B2000F1EC61F0320EE66E000EE66EFC0EE350E4
:108B3000020F386EFD0E6F008CFF39F0000E3922E7
:108B40006000E3F0E6FF6000E7F0E6FF11EC62F0A2
:108B5000FE0EE350010F386EFF0E6F008CFF39F0F0
:108B6000000E39226000E3F0E6FF6000E7F0E6FF68
:108B7000E60EE66EA80EE66EFA0EE350020F386EB1
:108B8000FB0E6F008CFF39F0000E39226000E3F01D
:108B9000E6FF6000E7F0E6FFBAEC5AF0FE0EE350A5
:108BA000010F386EFF0E6F008CFF39F0000E392276
:108BB0006000E3F0E6FF6000E7F0E6FFCE0EE66E51
:108BC000A90EE66EFA0EE350020F386EFB0E6F0030
:108BD0008CFF39F0000E39226000E3F0E6FF600000
:108BE000E7F0E6FFF5EC5AF0E552E552E5521200E7
:108BF000E652E652E652E652FB0EE350366E000EA7
:108C000036BEFF0E376E386E396EFC0E6000DBF03C
:108C1000E3FFFD0E6000DFF0E3FFFE0E6000E3F017
:108C2000E3FFFF0E6000E7F0E3FF020E0001D5193D
:108C3000D8A41DEF46F01FEF46F0C3EF46F0FF0E3D
:108C4000E3BE25EF46F027EF46F04FEF46F0FC0E6F
:108C50006F008CFF38F0FD0E6F008CFF39F0600E56
:108C60003824D96E000E3920DA6EDF50396E60007C
:108C7000E4F032F0336A346A356AFC0E6000CBF0FF
:108C8000E3FFFD0E6000CFF0E3FFFE0E6000D3F0C7
:108C9000E3FFFF0E6000D7F0E3FFC3EF46F0FF0EE7
:108CA000E66EFF0EE66EFF0EE66EFF0EE66EF80E47
:108CB0006F008FFFE6FF6F008FFFE6FF6F008FFFF3
:108CC000E6FF6F008FFFE6FF8AEC53F0FC0E6000BA
:108CD000BBF0E3FFFD0E6000BFF0E3FFFE0E60009F
:108CE000C3F0E3FFFF0E6000C7F0E3FFFC0E6F0070
:108CF0008CFF38F0FD0E6F008CFF39F0600E3824C9
:108D0000D96E000E3920DA6EDF50396E6000E4F063
:108D100032F0336A346A356AFC0E6000CBF0E3FF50
:108D2000FD0E6000CFF0E3FFFE0E6000D3F0E3FF26
:108D3000FF0E6000D7F0E3FFFF0EE66EFF0EE66E5B
:108D4000FF0EE66EFF0EE66EF80E6F008FFFE6FF79
:108D50006F008FFFE6FF6F008FFFE6FF6F008FFF52
:108D6000E6FF8AEC53F0FC0E6000BBF0E3FFFD0E63
:108D70006000BFF0E3FFFE0E6000C3F0E3FFFF0EF4
:108D80006000C7F0E3FF60001FF0E6FF600023F023
:108D9000E6FF600027F0E6FF60002BF0E6FFF80E2C
:108DA0006F008FFFE6FF6F008FFFE6FF6F008FFF02
:108DB000E6FF6F008FFFE6FF8AEC53F0FC0E6000C9
:108DC000BBF0E3FFFD0E6000BFF0E3FFFE0E6000AE
:108DD000C3F0E3FFFF0E6000C7F0E3FFE80EE66EAE
:108DE000030EE66E000EE66E000EE66EF80E6F00E5
:108DF0008FFFE6FF6F008FFFE6FF6F008FFFE6FF3C
:108E00006F008FFFE6FF40EC48F0FC0E6000BBF007
:108E1000E3FFFD0E6000BFF0E3FFFE0E6000C3F055
:108E2000E3FFFF0E6000C7F0E3FFFC0E6F008CFF56
:108E3000C9F0FD0E6F008CFFCAF0FB0EE126FF0E9D
:108E4000E2221200E652FA0E6F008CFF2EF0020EA4
:108E50002E18D8A42EEF47F030EF47F009EF48F076
:108E6000F60E6F008FFFD9FFF70E6F008FFFDAFF4E
:108E7000FB0E6F008FFFDFFFFC0EE124D96EFF0EAB
:108E8000E220DA6E6F0078FF37F06F0078FF38F07D
:108E90006F0078FF39F03750326E3850336E3950EA
:108EA000346E356AFB0E6000CBF0E3FFFC0E600011
:108EB000CFF0E3FFFD0E6000D3F0E3FFFE0E600095
:108EC000D7F0E3FFF80E6F008FFFD9FFF90E6F00A8
:108ED0008FFFDAFFFB0E6F008FFFDFFFFC0EE12438
:108EE000D96EFF0EE220DA6E6F0078FF37F06F0068
:108EF00078FF38F06F0078FF39F03750326E385015
:108F0000336E3950346E356AFB0E6000CBF0E3FFF0
:108F1000FC0E6000CFF0E3FFFD0E6000D3F0E3FF36
:108F2000FE0E6000D7F0E3FFFB0E6F008CFF39F000
:108F3000030E3916FF0E6000E7F0E3FFE150FB0F70
:108F4000D96EE250DA6EFF0EDA22030ED890DE36CA
:108F5000DE36DE36DD36DD52DD52E82EA6EF47F096
:108F6000FB0E6F008CFF39F0E00E3916E150FF0F59
:108F7000D96EE250DA6EFF0EDA223950DF26FF0E8C
:108F80006F008CFF2EF0080E2E26FF0E6000BBF047
:108F9000E3FFF20E6F008FFFD9FFF30E6F008FFF1C
:108FA000DAFFFF0EE350EB0BDF6EFC0EE124D96E0F
:108FB000FF0EE220DA6E6F0078FF37F06F0078FF67
:108FC00038F06F0078FF39F03750326E3850336E1A
:108FD0003950346E356AFB0E6000CBF0E3FFFC0EB7
:108FE0006000CFF0E3FFFD0E6000D3F0E3FFFE0E64
:108FF0006000D7F0E3FFF40E6F008FFFD9FFF50E8E
:109000006F008FFFDAFFFB0E6F008FFFDFFF3BEF7C
:1090100048F0F80E6F008FFFD9FFF90E6F008FFF39
:10902000DAFFDF6AF60E6F008FFFD9FFF70E6F00D1
:109030008FFFDAFFDF6AE150FB0FD96EE250DA6E84
:10904000FF0EDA22050ED890DE36DE36DE36DD364D
:10905000DD52DD52E82E23EF48F0F20E6F008FFF55
:10906000D9FFF30E6F008FFFDAFFFB0E6F008FFF4B
:10907000DFFFD5EF47F0F20EE126FF0EE2221200ED
:10908000060EE126000EE222FE0EE36AF50EE3BEB6
:109090004EEF48F04CEF48F062EF48F0F20EE36C10
:1090A000F30EE31EF40EE31EF50EE31E08E3F30ECB
:1090B000E32A05E3F40EE32A02E3F50EE32AFE0EAB
:1090C000E36AE32AF90EE3BE6AEF48F068EF48F07E
:1090D0007DEF48F0F60EE36CF70EE31EF80EE31E8C
:1090E000F90EE31E08E3F70EE32A05E3F80EE32A80
:1090F00002E3F90EE32AFE0EE370FA0EE36AFB0EBA
:10910000E36AFC0EE36AFD0EE36AF20EE3500FE140
:10911000F30EE3500CE1F40EE35009E1F50EE350D9
:10912000D8B495EF48F097EF48F000EF49F0FF0E04
:10913000E36AE32AA7EF48F0D890F20EE336F30E85
:10914000E336F40EE336F50EE336FF0EE32AF50EB2
:10915000E3AEADEF48F0AFEF48F09CEF48F0D890A9
:10916000FA0EE336FB0EE336FC0EE336FD0EE33675
:10917000E150F60FD96EE250DA6EFF0EDA22F20EEF
:10918000E350DE5CF30EE350DE58F40EE350DE589D
:10919000F50EE350DE58D8A0D0EF48F0D2EF48F0FB
:1091A000E7EF48F0E150F60FD96EE250DA6EFF0EAD
:1091B000DA22F20EE350DE5EF30EE350DE5AF40ED6
:1091C000E350DE5AF50EE350DE5AFA0EE380D890F3
:1091D000F50EE332F40EE332F30EE332F20EE33235
:1091E000FF0EE3502E6E010E2E5EFF0E6000BBF0F0
:1091F000E3FFD8A4FEEF48F000EF49F0AFEF48F0EE
:10920000FE0EE350D8B407EF49F009EF49F01AEF2A
:1092100049F0FA0EE36CFB0EE31EFC0EE31EFD0E9E
:10922000E31E08E3FB0EE32A05E3FC0EE32A02E358
:10923000FD0EE32AFA0E6F008CFF2EF0FB0E6F007E
:109240008CFF2FF0FC0E6F008CFF30F0FD0E6F00D6
:109250008CFF31F0F20EE126FF0EE22212000A0E20
:10926000E126000EE222F60EE36AF70EE36AF80E3C
:10927000E36AF90EE36AF20E6F008CFF39F0030E19
:109280003916FF0E6000E7F0E3FFF20E6F008CFF6F
:1092900039F0050E2E6ED89039322E2E4BEF49F054
:1092A000FE0E6000E7F0E3FFF30EE350386E396A1C
:1092B000D89038363936D89038363936D89038364E
:1092C0003936F60E6000E3F0E3FFF70E6000E7F0DA
:1092D000E3FF2E6AE3BE2E68F80E6000BBF0E3FFEA
:1092E000F90E6000BBF0E3FFE150F60FD96EE250DB
:1092F000DA6EFF0EDA22FE0EE350DE26000EDE22CC
:10930000DE22DE22E150F60FD96EE250DA6EFF0E59
:10931000DA22020ED890DE36DE36DE36DD36DD525B
:10932000DD52E82E8AEF49F0E150F60FD96EE25097
:10933000DA6EFF0EDA22FF0EE350DE26000EDE228A
:10934000DE22DE22E150F60FD96EE250DA6EFF0E19
:10935000DA22080ED890DE36DE36DE36DD36DD5215
:10936000DD52E82EAAEF49F0E150F60FD96EE25037
:10937000DA6EFF0EDA22F50EE350DE26000EDE2254
:10938000DE22DE22E150F60FD96EE250DA6EFF0ED9
:10939000DA22080ED890DE36DE36DE36DD36DD52D5
:1093A000DD52E82ECAEF49F0E150F60FD96EE250D7
:1093B000DA6EFF0EDA22F40EE350DE26000EDE2215
:1093C000DE22DE22F60E6F008CFF36F0F70E6F0005
:1093D0008CFF37F0F80E6F008CFF38F0F90E6F003D
:1093E0008CFF39F0FA0E6000DBF0E3FFFB0E60004B
:1093F000DFF0E3FFFC0E6000E3F0E3FFFD0E600032
:10940000E7F0E3FFFA0E6F008CFF2EF0FB0E6F000B
:109410008CFF2FF0FC0E6F008CFF30F0FD0E6F0004
:109420008CFF31F0F20EE126FF0EE2221200800ED8
:109430008F6E8E50E00B800AD8A421EF4AF023EF04
:109440004AF019EF4AF0900E916E3701006B3D6BB8
:10945000B90EE66E370EE66EB80EE66E370EE66EA5
:10946000BB0EE66E370EE66EBA0EE66E370EE66E91
:10947000010EE66E700EE66E000EE66E000EE66EF3
:10948000000EE66E22EC47F0BD0EE66E370EE66E7D
:10949000BC0EE66E370EE66EBF0EE66E370EE66E5B
:1094A000BE0EE66E370EE66E010EE66E700EE66ECE
:1094B000000EE66E000EE66E000EE66E22EC47F041
:1094C000A10EE66E370EE66EA00EE66E370EE66E65
:1094D000A30EE66E370EE66EA20EE66E370EE66E51
:1094E000010EE66E000EE66E000EE66E000EE66EF3
:1094F000000EE66E22EC47F0A50EE66E370EE66E25
:10950000A40EE66E370EE66EA70EE66E370EE66E1A
:10951000A60EE66E370EE66E010EE66E100EE66ED5
:10952000000EE66E000EE66E000EE66E22EC47F0D0
:10953000A90EE66E370EE66EA80EE66E370EE66EE4
:10954000AB0EE66E370EE66EAA0EE66E370EE66ED0
:10955000010EE66E700EE66E000EE66E000EE66E12
:10956000000EE66E22EC47F0070E3701066F100E74
:10957000396F0F0E036F980E046F810E056F4E0E3C
:10958000E66EC90EE66E27EC64F03901A59395836B
:10959000580EE66EC90EE66E11EC64F05A0EE66ED9
:1095A000C90EE66E1CEC64F0520EE66EC90EE66E55
:1095B000F0EC63F0560EE66EC90EE66E06EC64F053
:1095C000500EE66EC90EE66EE5EC63F0540EE66EE4
:1095D000C90EE66EFBEC63F03901A59B958B8F6A93
:1095E0006F0038FE39F0E00E3916D8A4FAEF4AF0D1
:1095F000FCEF4AF0F0EF4AF01200FE0E6F008FFF12
:10960000D9FFFF0E6F008FFFDAFF6E0EDF6E030EC5
:10961000E66EFD0EE350010F386EFE0E6F008CFFFC
:1096200039F0000E39226000E3F0E6FF6000E7F059
:10963000E6FF8CEC44F0010EE66E100EE66EF80EBE
:10964000E66EA30EE66EFA0EE350010F386EFB0EC7
:109650006F008CFF39F0000E39226000E3F0E6FF66
:109660006000E7F0E6FF30EC5BF0FE0E6F008FFF6E
:10967000E6FF6F008FFFE6FF620EE66EBB0EE66E42
:10968000FA0EE350010F386EFB0E6F008CFF39F0BD
:10969000000E39226000E3F0E6FF6000E7F0E6FF2D
:1096A00044EC5AF0FE0E6F008FFFE6FF6F008FFF55
:1096B000E6FFEE0EE66EBA0EE66EFA0EE350010F0E
:1096C000386EFB0E6F008CFF39F0000E39226000FF
:1096D000E3F0E6FF6000E7F0E6FF6BEC5BF0FE0E08
:1096E0006F008FFFE6FF6F008FFFE6FFE20EE66E72
:1096F000C20EE66EFA0EE350010F386EFB0E6F00DD
:109700008CFF39F0000E39226000E3F0E6FF6000C4
:10971000E7F0E6FF7FEC5AF0FE0E6F008CFF38F0AA
:10972000FF0E6F008CFF39F0380E3824D96E000E12
:109730003920DA6EDE6ADD6AFE0E6F008CFF38F0CB
:10974000FF0E6F008CFF39F03C0E3824D96E000EEE
:109750003920DA6EDE6ADD6AFE0E6F008CFF38F0AB
:10976000FF0E6F008CFF39F0400E3824D96E000ECA
:109770003920DA6EDE6ADD6A980E0001CB6F8B0E3F
:10978000CC6F080ECD6F000ECE6FE552E552120081
:10979000FE0E6F008FFFD9FFFF0E6F008FFFDAFF05
:1097A000640EDF6E020EE66EFD0EE350010F386EA2
:1097B000FE0E6F008CFF39F0000E39226000E3F0DE
:1097C000E6FF6000E7F0E6FF8CEC44F0040EE66E86
:1097D000100EE66E2A0EE66EB20EE66EFA0EE3503C
:1097E000010F386EFB0E6F008CFF39F0000E39222E
:1097F0006000E3F0E6FF6000E7F0E6FF30EC5BF0CE
:10980000FE0E6F008FFFE6FF6F008FFFE6FFBE0EBC
:10981000E66EBC0EE66EFA0EE350010F386EFB0EDC
:109820006F008CFF39F0000E39226000E3F0E6FF94
:109830006000E7F0E6FF44EC5AF0FE0E6F008FFF89
:10984000E6FF6F008FFFE6FF4A0EE66EBC0EE66E87
:10985000FA0EE350010F386EFB0E6F008CFF39F0EB
:10986000000E39226000E3F0E6FF6000E7F0E6FF5B
:109870006BEC5BF0FE0E6F008FFFE6FF6F008FFF5B
:10988000E6FFD60EE66EBB0EE66EFA0EE350010F53
:10989000386EFB0E6F008CFF39F0000E392260002D
:1098A000E3F0E6FF6000E7F0E6FF7FEC5AF0FE0E23
:1098B0006F008CFF38F0FF0E6F008CFF39F0380E10
:1098C0003824D96E000E3920DA6EDE6ADD6AFE0EAB
:1098D0006F008CFF38F0FF0E6F008CFF39F03C0EEC
:1098E0003824D96E000E3920DA6EDE6ADD6AFE0E8B
:1098F0006F008CFF38F0FF0E6F008CFF39F0400EC8
:109900003824D96E000E3920DA6EDE6ADD6AE5523F
:10991000E5521200E652E652FE0EE36AFF0EE36ADB
:10992000FE0E6F008CFF38F0FF0E6F008CFF39F0D9
:109930000F0E38026F00CCFF36F06F00D0FF37F00B
:109940003902F3503726A10E3624386E040E372024
:10995000396E6000E3F0E6FF6000E7F0E6FFC7EC79
:1099600058F0FE0EE350010F2E6EFE0E6000BBF0AD
:10997000E3FF2E6AFF0EE3502E202E6EFF0E6000D6
:10998000BBF0E3FFFF0EE3BED4EF4CF0FF0EE3505D
:109990000DE1FE0E6F008CFF2EF0140E2E5ED8A08F
:1099A000D4EF4CF0D6EF4CF090EF4CF0FE0EE36AA3
:1099B000FF0EE36AFE0E6F008CFF38F0FF0E6F00A3
:1099C0008CFF39F0110E38026F00CCFF36F06F00BB
:1099D000D0FF37F03902F3503726F80E3624D96E0F
:1099E000020E3720DA6EDE6ADD6AFE0E6F008CFF33
:1099F00038F0FF0E6F008CFF39F0110E38026F0047
:109A0000CCFF36F06F00D0FF37F03902F350372625
:109A1000FA0E3624386E020E3720396E6000E3F0FD
:109A2000E6FF6000E7F0E6FFC7EC58F0FE0EE350FB
:109A3000010F2E6EFE0E6000BBF0E3FF2E6AFF0EDC
:109A4000E3502E202E6EFF0E6000BBF0E3FFFF0EF2
:109A5000E3BE39EF4DF0FF0EE3500DE1FE0E6F0057
:109A60008CFF2EF0190E2E5ED8A039EF4DF03BEF93
:109A70004DF0DAEF4CF0000E6F00A0FFCDF5000EB8
:109A80006F00A0FFCEF5E552E5521200E652E65215
:109A9000E652EE0EE1242E6EFF0EE2202F6E6000E5
:109AA000BBF0E6FF6000BFF0E6FFE6EC62F0FD0E03
:109AB0006000BBF0E3FFFE0E6000BFF0E3FFFD0EB1
:109AC0006F008CFF2EF0FE0EE3502E10D8B46BEF1B
:109AD0004DF06DEF4DF0A5EF4DF0000EE66E000E6F
:109AE000E66EEC0EE1242E6EFF0EE2202F6E60007B
:109AF000BBF0E6FF6000BFF0E6FF91EC61F0ED0E19
:109B0000E350E66EED0EE124D96EFF0EE220DA6E30
:109B10000F0E6F007BFFE6FFE82C89EF4DF0ED0E96
:109B20006F008FFFE6FF6F008FFFE6FF11EC57F02D
:109B3000EB0E6F008FFFD9FFEC0E6F008FFFDAFF87
:109B40006000BBF0DFFFFAEF4DF0ED0EE350E66E84
:109B5000C2EC63F0140EE66E000EE66E21EECDF15F
:109B6000DF50386E396A010E3826000E3922600047
:109B7000E3F0E6FF6000E7F0E6FF6AEC4FF0FF0E6F
:109B80006000BBF0E3FF21EECEF1FF0EE350DE18E4
:109B9000D8A4CDEF4DF0CFEF4DF0D8EF4DF0ED0E56
:109BA000E350E66EB6EC63F0000E2E6EFCEF4DF067
:109BB000EE0EE124D96EFF0EE220DA6E01EECDF159
:109BC000EF500F0DA10EF324E96E040EF420EA6E9F
:109BD0000E0E6F006FFFEBFFE806FBE2FF0E6F005B
:109BE0008CFF39F06000E4F0CDF5ED0EE350E66E49
:109BF000B6EC63F0010E2E6EEB0EE126FF0EE222B4
:109C00001200100EE126000EE222190E396EFF0E30
:109C10006000E7F0E3FFF00EE1242E6EFF0EE2207D
:109C20002F6E6000BBF0E6FF6000BFF0E6FFC7EC00
:109C300058F0EE0E6F008FFFE6FF6F008FFFE6FF1C
:109C4000EE0EE1242E6EFF0EE2202F6E6000BBF0C0
:109C5000E6FF6000BFF0E6FFB1EC61F0EC0E6F00D4
:109C60008FFFE6FF6F008FFFE6FFEE0EE1242E6E02
:109C7000FF0EE2202F6E6000BBF0E6FF6000BFF039
:109C8000E6FFD1EC61F0EB0EE350E66EEF0EE1245F
:109C90002E6EFF0EE2202F6E6000BBF0E6FF60002C
:109CA000BFF0E6FF35EC63F0E90E6F008FFFE6FFD3
:109CB0006F008FFFE6FFEE0EE1242E6EFF0EE22016
:109CC0002F6E6000BBF0E6FF6000BFF0E6FF91EC96
:109CD00061F0E150E10FD96EE250DA6EFF0EDA2248
:109CE0006F007BFFE6FF6F007BFFE6FF6F007BFFEF
:109CF000E6FF6F007BFFE6FF6F007BFFE6FF6F0074
:109D00007BFFE6FF6F007BFFE6FF6F007BFFE6FF58
:109D1000E80EE1242E6EFF0EE2202F6E6000BBF0F5
:109D2000E6FF6000BFF0E6FF4DEC62F0FF0EE124BD
:109D30002E6EFF0EE2202F6E6000BBF0E6FF60008B
:109D4000BFF0E6FF000EE66EED0EE124D96EFF0EC9
:109D5000E220DA6E0F0E6F007BFFE6FFE82CABEF20
:109D60004EF046EC4DF0E10EE126FF0EE22212002D
:109D7000E652E652E652E652FB0EE3BEC2EF4EF06A
:109D8000C4EF4EF0E6EF4EF0F80E6F008CFF36F0A9
:109D9000F90E6F008CFF37F0FA0E6F008CFF38F071
:109DA000FB0E6F008CFF39F0FC0E6000DBF0E3FF70
:109DB000FD0E6000DFF0E3FFFE0E6000E3F0E3FF66
:109DC000FF0E6000E7F0E3FF0FEF4FF0F80E6F00BB
:109DD0008CFF36F0F90E6F008CFF37F0FA0E6F0033
:109DE0008CFF38F0FB0E6F008CFF39F0361E371EEB
:109DF000381E391E362A000E372238223922FC0E30
:109E00006000DBF0E3FFFD0E6000DFF0E3FFFE0E1D
:109E10006000E3F0E3FFFF0E6000E7F0E3FFE80E11
:109E2000E66E030EE66E000EE66E000EE66EF80EAF
:109E30006F008FFFE6FF6F008FFFE6FF6F008FFF61
:109E4000E6FF6F008FFFE6FF8AEC53F0FC0E600028
:109E5000BBF0E3FFFD0E6000BFF0E3FFFE0E60000D
:109E6000C3F0E3FFFF0E6000C7F0E3FF60000FF0F8
:109E7000E6FF600013F0E6FF600017F0E6FF600009
:109E80001BF0E6FFF80E6F008FFFE6FF6F008FFFFD
:109E9000E6FF6F008FFFE6FF6F008FFFE6FF60ECCD
:109EA00051F0FC0E6000BBF0E3FFFD0E6000BFF060
:109EB000E3FFFE0E6000C3F0E3FFFF0E6000C7F09B
:109EC000E3FFFC0E6F008CFFD3F0F80EE126FF0ECF
:109ED000E2221200E652E652FE0EE36AFD0EE3BEF7
:109EE00076EF4FF074EF4FF07FEF4FF0FC0EE36C26
:109EF000FD0EE31ED8B0E32AFE0EE36AE32AFB0E52
:109F0000E3BE87EF4FF085EF4FF08DEF4FF0FA0E85
:109F1000E36CFB0EE31ED8B0E32AFA0E6F008CFF51
:109F20002EF0FB0EE3502E10D8B499EF4FF09BEFBC
:109F30004FF0FFEF4FF0FF0EE36AE32AB3EF4FF06D
:109F4000FA0EE350D890E8342E6EFA0E6000BBF0A3
:109F5000E3FFFB0EE350E8342E6EFB0E6000BBF017
:109F6000E3FFFF0EE32AFB0EE3AEB9EF4FF0BBEFCA
:109F70004FF0A0EF4FF0FA0E6F008CFF38F0FB0EA1
:109F80006F008CFF39F0FC0E6F008CFF36F0FD0E79
:109F90006F008CFF37F03850365C39503758D8A0F6
:109FA000D4EF4FF0D6EF4FF0EAEF4FF0FC0EE35056
:109FB0002E6EFA0EE3502E5EFC0E6000BBF0E3FF47
:109FC000FD0EE3502E6EFB0EE3502E5AFD0E600088
:109FD000BBF0E3FFD890FB0EE332FA0EE332FF0E44
:109FE000E3502E6E010E2E5EFF0E6000BBF0E3FF0D
:109FF000D8A4FDEF4FF0FFEF4FF0BBEF4FF0FE0E98
:10A00000E350D8B406EF50F008EF50F00EEF50F0E8
:10A01000FC0EE36CFD0EE31ED8B0E32AFC0E6F00CD
:10A020008CFF2EF0FD0E6F008CFF2FF0FA0EE12654
:10A03000FF0EE22212006F00E8FF4EF06F00ECFF0F
:10A040004FF06000B8F050F06000BCF051F06000DC
:10A05000C0F052F06000C4F053F06000D8F054F04B
:10A060006000DCF055F06000E0F056F06000E4F0D5
:10A0700057F06000F8F058F06000FCF059F0600014
:10A0800000F15AF0600004F15BF0600008F15CF050
:10A0900060000CF15DF0600010F15EF0600014F102
:10A0A0005FF012EEE8F2390193AF59EF50F05BEF39
:10A0B00050F066EF50F0A3AF60EF50F062EF50F059
:10A0C00066EF50F0B6EC62F08AEF50F095AB6BEFB4
:10A0D00050F06DEF50F078EF50F0A5AB72EF50F00C
:10A0E00074EF50F078EF50F012EC53F08AEF50F02C
:10A0F00095A37DEF50F07FEF50F08AEF50F0A5A3CD
:10A1000084EF50F086EF50F08AEF50F064EC63F08B
:10A110008AEF50F060007CF145F0600078F144F087
:10A12000600074F143F0600070F142F060006CF187
:10A1300041F0600068F140F0600064F13FF06000C1
:10A1400060F13EF060005CF139F0600058F138F0E9
:10A15000600054F137F0600050F136F060004CF1CF
:10A1600031F0600048F130F0600044F12FF0600001
:10A1700040F12EF060003FF1FBFF60003BF1FAFF81
:10A180001100FE0E6F008FFFD9FFFF0E6F008FFFD3
:10A19000DAFFDF6AFE0E6F008CFF38F0FF0E6F00F3
:10A1A0008CFF39F0010E3824D96E000E3920DA6E9A
:10A1B000F40EDE6E010EDD6EFE0E6F008CFF38F0C9
:10A1C000FF0E6F008CFF39F0030E3824D96E000E9D
:10A1D0003920DA6EF40EDE6E010EDD6EFE0E6F00BB
:10A1E0008CFF38F0FF0E6F008CFF39F0050E38241D
:10A1F000D96E000E3920DA6E030EDF6EFE0E6F0090
:10A200008CFF38F0FF0E6F008CFF39F0060E3824FB
:10A21000D96E000E3920DA6EDF6AFE0E6F008CFFF9
:10A2200038F0FF0E6F008CFF39F0070E3824D96E1E
:10A23000000E3920DA6E030EDF6EFE0E6F008CFF0B
:10A2400038F0FF0E6F008CFF39F0080E3824D96EFD
:10A25000000E3920DA6EDE6ADD6AFE0E6F008CFFBA
:10A2600038F0FF0E6F008CFF39F00C0E3824D96ED9
:10A27000000E3920DA6EDE6ADD6AFE0E6F008CFF9A
:10A2800038F0FF0E6F008CFF39F0100E3824D96EB5
:10A29000000E3920DA6EDE6ADD6AFE0E6F008CFF7A
:10A2A00038F0FF0E6F008CFF39F0140E3824D96E91
:10A2B000000E3920DA6EDE6ADD6AE552E5521200E0
:10A2C000050EE126000EE222FB0EE36AFC0EE36AB5
:10A2D000FD0EE36AFE0EE36AF30EE3500FE1F40EA7
:10A2E000E3500CE1F50EE35009E1F60EE350D8B46B
:10A2F0007CEF51F07EEF51F0E7EF51F0FF0EE36A93
:10A30000E32A8EEF51F0D890F30EE336F40EE336E5
:10A31000F50EE336F60EE336FF0EE32AF60EE3AE55
:10A3200094EF51F096EF51F083EF51F0D890FB0E7F
:10A33000E336FC0EE336FD0EE336FE0EE336E15067
:10A34000F70FD96EE250DA6EFF0EDA22F30EE35009
:10A35000DE5CF40EE350DE58F50EE350DE58F60EE8
:10A36000E350DE58D8A0B7EF51F0B9EF51F0CEEF7F
:10A3700051F0E150F70FD96EE250DA6EFF0EDA229B
:10A38000F30EE350DE5EF40EE350DE5AF50EE350BA
:10A39000DE5AF60EE350DE5AFB0EE380D890F60E3E
:10A3A000E332F50EE332F40EE332F30EE332FF0E46
:10A3B000E3502E6E010E2E5EFF0E6000BBF0E3FF39
:10A3C000D8A4E5EF51F0E7EF51F096EF51F0FB0E16
:10A3D0006F008CFF2EF0FC0E6F008CFF2FF0FD0E37
:10A3E0006F008CFF30F0FE0E6F008CFF31F0F30E2B
:10A3F000E126FF0EE2221200050EE126000EE22207
:10A40000F90E6F008FFFF6FFFA0E6F008FFFF7FF58
:10A41000000EF86E0F0EF76403D00800F55007D059
:10A420006F00DBFFE9FF6F00DFFFEAFFEF50396EDF
:10A43000FF0E6000E7F0E3FF54EF52F0FB0EE36A1B
:10A44000E32AFC0EE124D96EFF0EE220DA6EDF6A09
:10A45000FD0EE124D96EFF0EE220DA6EDF6A6EEFA8
:10A4600052F0FB0EE36AFC0EE124D96EFF0EE220EF
:10A47000DA6E010EDF6E28EF52F0FB0EE36AFC0E7F
:10A48000E124D96EFF0EE220DA6EDF6AFD0EE124D0
:10A49000D96EFF0EE220DA6E010EDF6E6EEF52F023
:10A4A000FB0EE36A21EF52F0FF0EE350386E396A7B
:10A4B0003950000AD8B45FEF52F050EF52F03850E4
:10A4C000010AD8B41EEF52F0030AD8B431EF52F0AB
:10A4D000010AD8B43DEF52F050EF52F0FE0EE124E5
:10A4E000D96EFF0EE220DA6E600067F0DFFFFB0E30
:10A4F0006F008FFFE6FF6F008FFFE6FF6F008FFF9B
:10A50000E6FF6F008FFFE6FF000EE66E050EE66EBB
:10A5100048EC3BF0F90EE126FF0EE2221200E65273
:10A52000E652FF0EE36AFF0EE350110DFA0EF3241C
:10A53000D96E020EF420DA6EDF50D8B4A2EF52F0DA
:10A54000A4EF52F001EF53F0FF0EE350110DF80E9F
:10A55000F324D96E020EF420DA6E0A0EDE5E000ECF
:10A56000DD5AFF0EE350110DF80EF324D96E020EE2
:10A57000F420DA6EDE50DE10D8A4C1EF52F0C3EF43
:10A5800052F001EF53F0FE0EE1242E6EFF0EE2209A
:10A590002F6E6000BBF0E6FF6000BFF0E6FF010E2B
:10A5A000E66EFC0EE350110DFA0EF324D96E020E86
:10A5B000F420DA6E0F0E6F007BFFE6FFE82CDBEF76
:10A5C00052F046EC4DF02E04D8A4E9EF52F0EBEF38
:10A5D00052F0F4EF52F0010EE66EFE0EE350E66E1E
:10A5E00028EC60F001EF53F0FF0EE350110DF80E70
:10A5F000F324D96E020EF420DA6E010EDE6E000E28
:10A60000DD6EFF0EE32AFF0E6F008CFF2EF0180E9A
:10A610002E640DEF53F00FEF53F093EF52F0E5522D
:10A62000E552120090AC17EF53F019EF53F026EFFC
:10A6300053F002D825EF53F00500FA6E2650FD6E58
:10A640002750FE6EFF6AFA501200909C90AA2BEFE2
:10A6500053F02DEF53F039EF53F002D839EF53F0A8
:10A660000500FA6E2450FD6E2550FE6EFF6AFA500A
:10A67000120090A83EEF53F040EF53F04CEF53F030
:10A6800002D84CEF53F00500FA6E2250FD6E2350B5
:10A69000FE6EFF6AFA50120090A651EF53F053EF8E
:10A6A00053F05FEF53F002D85FEF53F00500FA6EFE
:10A6B0002050FD6E2150FE6EFF6AFA50120090A4E9
:10A6C00064EF53F066EF53F073EF53F002D873EF7B
:10A6D00053F00500FA6E0001C751FD6EC851FE6EC1
:10A6E000FF6AFA50120090A278EF53F07AEF53F01D
:10A6F00087EF53F002D887EF53F00500FA6E0001A0
:10A70000C551FD6EC651FE6EFF6AFA501200390146
:10A71000A59B1200E652E652E652E652FC0EE36AB0
:10A72000FD0EE36AFE0EE36AFF0EE36AF80EE3A095
:10A730009CEF53F09EEF53F0C6EF53F0FC0EE35046
:10A740002E6EF40EE3502E26FC0E6000BBF0E3FFED
:10A75000FD0EE3502E6EF50EE3502E22FD0E60002E
:10A76000BBF0E3FFFE0EE3502E6EF60EE3502E22FA
:10A77000FE0E6000BBF0E3FFFF0EE3502E6EF70EFF
:10A78000E3502E22FF0E6000BBF0E3FFD890F40EE2
:10A79000E336F50EE336F60EE336F70EE336D890E1
:10A7A000FB0EE332FA0EE332F90EE332F80EE33237
:10A7B000F80EE3500DE1F90EE3500AE1FA0EE35012
:10A7C00007E1FB0EE350D8A4E8EF53F0EAEF53F0B3
:10A7D00096EF53F0FC0E6F008CFF2EF0FD0E6F0015
:10A7E0008CFF2FF0FE0E6F008CFF30F0FF0E6F001D
:10A7F0008CFF31F0F40EE126FF0EE2221200080E6B
:10A80000E126000EE222F60E6F008FFFD9FFF70E51
:10A810006F008FFFDAFF6F0078FF36F06F0078FF70
:10A8200037F06F0078FF38F06F0078FF39F0FC0EDA
:10A830006000DBF0E3FFFD0E6000DFF0E3FFFE0EE3
:10A840006000E3F0E3FFFF0E6000E7F0E3FFFF0EC0
:10A85000E124D96EFF0EE220DA6EDF50396EF80E79
:10A860006000E7F0E3FFFE0EE124D96EFF0EE22068
:10A87000DA6EF90EE124E96EFF0EE220EA6E6F0057
:10A880007FFFEFFFFD0EE124D96EFF0EE220DA6EAE
:10A89000FA0EE124E96EFF0EE220EA6E6F007FFF00
:10A8A000EFFFFB0EE124D96EFF0EE220DA6EFC0E04
:10A8B0006F008FFFDFFFF80E6F008FFFE6FF6F0066
:10A8C0008FFFE6FF6F008FFFE6FF6F008FFFE6FF51
:10A8D000010EE66E050EE66E48EC3BF0F60EE12644
:10A8E000FF0EE2221200E652E652FC0E6F008CFFD1
:10A8F00038F0FD0E6F008CFF39F0FF0E6000E7F0BE
:10A90000E3FFFE0E6000E3F0E3FF9FEF54F0BA8038
:10A91000E2EF54F0BA82E2EF54F0BA84E2EF54F07E
:10A92000BA86E2EF54F0BA88E2EF54F0BA8AE2EF66
:10A9300054F0BA8CE2EF54F0BA8EE2EF54F0FE0E0F
:10A940006F008FFFF6FFFF0E6F008FFFF7FF000E07
:10A95000F86E0F0EF76403D00800F55007D06F00B3
:10A96000DBFFE9FF6F00DFFFEAFFEF50386E396A67
:10A970003950000AD8B4BFEF54F0E2EF54F0385029
:10A98000010AD8B487EF54F0030AD8B48AEF54F020
:10A99000010AD8B48DEF54F0070AD8B490EF54F000
:10A9A000010AD8B493EF54F0030AD8B496EF54F0E8
:10A9B000010AD8B499EF54F00F0AD8B49CEF54F0C0
:10A9C000E2EF54F0E552E552E552E5521200E6524C
:10A9D000E652FC0E6F008CFF38F0FD0E6F008CFF0E
:10A9E00039F0FF0E6000E7F0E3FFFE0E6000E3F0D9
:10A9F000E3FF13EF55F0BA9056EF55F0BA9256EFC9
:10AA000055F0BA9456EF55F0BA9656EF55F0BA98FD
:10AA100056EF55F0BA9A56EF55F0BA9C56EF55F0EE
:10AA2000BA9E56EF55F0FE0E6F008FFFF6FFFF0E39
:10AA30006F008FFFF7FF000EF86E0F0EF76403D064
:10AA40000800F55007D06F00DBFFE9FF6F00DFFF64
:10AA5000EAFFEF50386E396A3950000AD8B433EF44
:10AA600055F056EF55F03850010AD8B4FBEF54F0CA
:10AA7000030AD8B4FEEF54F0010AD8B401EF55F040
:10AA8000070AD8B404EF55F0010AD8B407EF55F01F
:10AA9000030AD8B40AEF55F0010AD8B40DEF55F007
:10AAA0000F0AD8B410EF55F056EF55F0E552E552C5
:10AAB000E552E5521200080EE126000EE222F70EE2
:10AAC000E350386E396AD89038363936D8903836EF
:10AAD0003936D89038363936F80E6000E3F0E3FFA7
:10AAE000F90E6000E7F0E3FF2E6AE3BE2E68FA0E6F
:10AAF0006000BBF0E3FFFB0E6000BBF0E3FFE15042
:10AB0000F80FD96EE250DA6EFF0EDA22F60E6F0001
:10AB10008CFF39F0050E2E6ED89039322E2E8CEF28
:10AB200055F03950DE26000EDE22DE22DE22F80E3F
:10AB30006F008CFF36F0F90E6F008CFF37F0FA0EC5
:10AB40006F008CFF38F0FB0E6F008CFF39F0FC0EAD
:10AB50006000DBF0E3FFFD0E6000DFF0E3FFFE0EC0
:10AB60006000E3F0E3FFFF0E6000E7F0E3FFFC0EA0
:10AB70006F008CFF2EF0FD0E6F008CFF2FF0FE0E8D
:10AB80006F008CFF30F0FF0E6F008CFF31F0F60E7F
:10AB9000E126FF0EE22212001D0EE126000EE22247
:10ABA000F10EE36AF40EE124D96EFF0EE220DA6EB4
:10ABB000DE6ADD6AF20EE124D96EFF0EE220DA6E63
:10ABC000DE6ADD6AE20EE350E66EC2EC63F021EE6F
:10ABD000CEF101EECDF1DE50EE18D8A4F2EF55F033
:10ABE000F4EF55F00AEF56F0E20EE350E66EB6ECE5
:10ABF00063F0F10EE124D96EFF0EE220DA6E0F0E43
:10AC00002E6EE20E6F007BFFE3FFE8282E2EFAD7B0
:10AC100037EF56F021EECEF1DF500F0DA10EF324E9
:10AC2000D96E040EF420DA6E0F0E2E6EF10E6F0048
:10AC30007BFFE3FFE8282E2EFAD7140EE66E000EF7
:10AC4000E66E21EECEF1DF50386E396A010E3826FD
:10AC5000000E39226000E3F0E6FF6000E7F0E6FF57
:10AC60006AEC4FF06000B8F0CEF5F4EF55F0F10E5D
:10AC7000E126FF0EE2221200070EE66E9FEC64F062
:10AC80006000BBF0E6FF6000BFF0E6FF45EC63F05C
:10AC9000080EE66E59EC64F06000BBF0E6FF600061
:10ACA000BFF0E6FF45EC63F09FEC64F06000BBF0A2
:10ACB000E6FF6000BFF0E6FFCEEC63F059EC64F015
:10ACC0006000BBF0E6FF6000BFF0E6FFCEEC63F093
:10ACD00099EC64F0010EE66E93EC64F0E9EC3CF064
:10ACE00089EC3EF0060EE66E7DEC64F06000BBF091
:10ACF000E6FF6000BFF0E6FF8CEC44F00250E66E29
:10AD00007DEC64F06000BBF0E6FF6000BFF0E6FFA2
:10AD1000FEEC5FF0010EE66E74EC64F06000BBF0D8
:10AD2000E6FF6000BFF0E6FF8CEC44F062EC64F0FC
:10AD30006000BBF0E6FF6000BFF0E6FFC8EC4BF040
:10AD400050EC64F06000BBF0E6FF6000BFF0E6FF8F
:10AD5000FDEC4AF012000F0EE126000EE222000E7A
:10AD6000E66ECCEC55F0F10EE124D96EFF0EE22038
:10AD7000DA6E0F0E2E6EDD50E552E750DF6E2E2E8E
:10AD8000FAD7F10EE350D8B4C8EF56F0CAEF56F038
:10AD90000CEF57F0F40EE124D96EFF0EE220DA6ECC
:10ADA000DE50DE10D8B4D7EF56F0D9EF56F00CEFE6
:10ADB00057F0F20EE124D96EFF0EE220DA6EDE507B
:10ADC000DE10D8B4E6EF56F0E8EF56F00CEF57F08F
:10ADD000F10EE1242E6EFF0EE2202F6E6000BBF01C
:10ADE000E6FF6000BFF0E6FFF00EE124D96EFF0E33
:10ADF000E220DA6E6F0078FF38F06F0074FF39F0F0
:10AE000002D80CEF57F00500FA6E3850FD6E39503D
:10AE1000FE6EFF6AFA501200F10EE126FF0EE222EA
:10AE20001200E652ED0EE350E66EC2EC63F0FF0E48
:10AE3000E36AFF0EE350110DFA0EF324D96E020EF1
:10AE4000F420DA6EDF50D8A428EF57F02AEF57F03D
:10AE500057EF57F0E150FD0FD96EE250DA6EFF0E5A
:10AE6000DA22FF0EE350110DF80EF324E96E020E04
:10AE7000F420EA6E6F007BFFEEFF6F0077FFEDFFBF
:10AE8000EE0EE124D96EFF0EE220DA6EFF0EE350E3
:10AE9000110DFA0EF324E96E020EF420EA6E0E0E86
:10AEA0006F006FFFEBFFE806FBE265EF57F0FF0E68
:10AEB000E32AFF0E6F008CFF2EF0180E2E6463EF56
:10AEC00057F065EF57F019EF57F0ED0EE350E66ECF
:10AED000B6EC63F0FF0E6F008CFF2EF0ED0EE12656
:10AEE000FF0EE2221200060EE126000EE222F50E0F
:10AEF0006F008CFF36F0F60E6F008CFF37F0F70E08
:10AF00006F008CFF38F0F80E6F008CFF39F0FC0EEC
:10AF10006000DBF0E3FFFD0E6000DFF0E3FFFE0EFC
:10AF20006000E3F0E3FFFF0E6000E7F0E3FFFB0EDD
:10AF3000E36AF90E6F008CFF2EF0FA0E6000BBF092
:10AF4000E3FFFA0EE3502E6EFB0EE3502E26FA0EB0
:10AF50006000BBF0E3FFFB0E6F008CFF39F0FC0ECE
:10AF6000E124366EFF0EE220376E39503624D96E5A
:10AF7000000E3720DA6EDF50E66EF90EE350E66E13
:10AF8000A9EC63F0FB0EE32AFB0E6F008CFF2EF0A2
:10AF9000030E2E64CEEF57F0D0EF57F099EF57F035
:10AFA000F50EE126FF0EE2221200060EE126000E4B
:10AFB000E222FB0EE36AF90E6F008CFF2EF0FA0E10
:10AFC0006000BBF0E3FFFA0EE3502E6EFB0EE35081
:10AFD0002E26FA0E6000BBF0E3FFFA0EE350E66E99
:10AFE0006BEC64F0FB0E6F008CFF39F0FC0EE1247B
:10AFF000366EFF0EE220376E39503624D96E000EC1
:10B000003720DA6E6000BBF0DFFFFB0EE32AFB0E99
:10B010006F008CFF2EF0030E2E6411EF58F013EF2B
:10B0200058F0DBEF57F0FC0E6F008CFF2EF0FD0E9A
:10B030006F008CFF2FF0FE0E6F008CFF30F0FF0EC4
:10B040006F008CFF31F0F90EE126FF0EE2221200B4
:10B05000060EE126000EE222F80E6F008FFFE9FFD8
:10B06000F90E6F008FFFEAFFFE0E6F00BBFFE3FFDC
:10B07000FF0E6F00B7FFE3FFFF0EE124D96EFF0E56
:10B08000E220DA6EDF50396EFA0E6000E7F0E3FF7F
:10B09000FB0EE124D96EFF0EE220DA6EFE0E6F0089
:10B0A0008FFFDFFFFC0EE124D96EFF0EE220DA6E87
:10B0B000DF6AFD0EE124D96EFF0EE220DA6EDF6A50
:10B0C000FA0E6F008FFFE6FF6F008FFFE6FF6F0045
:10B0D0008FFFE6FF6F008FFFE6FF010EE66E040EA6
:10B0E000E66E48EC3BF0F80EE126FF0EE22212007D
:10B0F000340EE66E800EE66E27EC64F0320EE66EDD
:10B10000460EE66E32EC64F0000EE66E000EE66E61
:10B11000260EE66EC60EE66E7DEC64F06000BBF0B7
:10B12000E6FF6000BFF0E6FFA6EC5BF0000EE66E07
:10B13000000EE66E120EE66EB40EE66E74EC64F06F
:10B140006000BBF0E6FF6000BFF0E6FF30EC5BF0B4
:10B150001450E66E74EC64F06000BBF0E6FF600033
:10B16000BFF0E6FFFEEC5FF0000EE66E000EE66E4E
:10B17000020EE66EC70EE66E74EC64F06000BBF083
:10B18000E6FF6000BFF0E6FF6BEC5BF01200FE0E26
:10B190006F008FFFD9FFFF0E6F008FFFDAFFDF6AAE
:10B1A000FE0E6F008CFF38F0FF0E6F008CFF39F041
:10B1B000050E3824D96E000E3920DA6EDE6ADD6A9B
:10B1C000FE0E6F008CFF38F0FF0E6F008CFF39F021
:10B1D000030E3824D96E000E3920DA6EDE6ADD6A7D
:10B1E000FE0E6F008CFF38F0FF0E6F008CFF39F001
:10B1F000070E3824D96E000E3920DA6E070EDE6A8B
:10B20000E806FDE2FE0E6F008CFF38F0FF0E6F00C7
:10B210008CFF39F0010E3824D96E000E3920DA6E19
:10B22000DE6ADD6AE552E5521200E652E652E65267
:10B23000E652FA0E6F008CFF2EF0FC0E6000BBF0A1
:10B24000E3FFFD0EE124D96EFF0EE220DA6E60000E
:10B250005BF0DFFFFE0EE124D96EFF0EE220DA6E16
:10B2600060005FF0DFFFFF0EE124D96EFF0EE220E9
:10B27000DA6E600063F0DFFFFC0E6F008FFFE6FF09
:10B280006F008FFFE6FF6F008FFFE6FF6F008FFFFD
:10B29000E6FF000EE66E040EE66E48EC3BF0FA0E9A
:10B2A000E126FF0EE2221200E652E652E652E65294
:10B2B000FC0EE36AFA0E6F008FFFD9FFFB0E6F00E2
:10B2C0008FFFDAFFFD0EE124E96EFF0EE220EA6E49
:10B2D0006F007FFFEFFFFE0EE124D96EFF0EE2202C
:10B2E000DA6EDF6AFF0EE124D96EFF0EE220DA6E1D
:10B2F000DF6AFC0E6F008FFFE6FF6F008FFFE6FF37
:10B300006F008FFFE6FF6F008FFFE6FF020EE66E15
:10B31000030EE66E48EC3BF0FA0EE126FF0EE22249
:10B320001200E652D2BE97EF59F09BEF59F0396AFE
:10B33000392A9CEF59F0396AFF0E6000E7F0E3FF0D
:10B34000FE0EE124D96EFF0EE220DA6EDF50030B11
:10B350003901E16FFD0E6F008FFFE0F9FC0E6F0009
:10B360008FFFE3F93F0EE517E585D29E550EE66F98
:10B37000AA0EE66FE583E5B3C0EF59F0C2EF59F0CE
:10B38000BBEF59F0E595FF0EE3B002D0D29E01D09D
:10B39000D28EE552E552E552E5521200E652E652EF
:10B3A000E652E652FC0E60006BF0E3FFFD0EE12476
:10B3B000D96EFF0EE220DA6E60006FF0DFFFFE0E46
:10B3C000E124D96EFF0EE220DA6E600073F0DFFF39
:10B3D000FF0EE124D96EFF0EE220DA6E600077F0F6
:10B3E000DFFFFC0E6F008FFFE6FF6F008FFFE6FFB1
:10B3F0006F008FFFE6FF6F008FFFE6FF000EE66E27
:10B40000060EE66E48EC3BF0FA0EE126FF0EE22255
:10B410001200E652E652E652E652FC0E600047F099
:10B42000E3FFFD0EE124D96EFF0EE220DA6E60002C
:10B430004BF0DFFFFE0EE124D96EFF0EE220DA6E44
:10B4400060004FF0DFFFFF0EE124D96EFF0EE22017
:10B45000DA6E600053F0DFFFFC0E6F008FFFE6FF37
:10B460006F008FFFE6FF6F008FFFE6FF6F008FFF1B
:10B47000E6FF000EE66E020EE66E48EC3BF0FA0EBA
:10B48000E126FF0EE2221200E150FC0FD96EE250DD
:10B49000DA6EFF0EDA22FE0E6F008CFF38F0FF0E20
:10B4A0006F008CFF39F0270E3824E96E000E39202A
:10B4B000EA6E6F007BFFEEFF6F0077FFEDFFE1505C
:10B4C000FA0FD96EE250DA6EFF0EDA22FE0E6F002E
:10B4D0008CFF38F0FF0E6F008CFF39F0290E3824F6
:10B4E000E96E000E3920EA6E6F007BFFEEFF6F0001
:10B4F00077FFEDFFFA0EE126FF0EE2221200E15087
:10B50000FC0FD96EE250DA6EFF0EDA22FE0E6F00EB
:10B510008CFF38F0FF0E6F008CFF39F0230E3824BB
:10B52000E96E000E3920EA6E6F007BFFEEFF6F00C0
:10B5300077FFEDFFE150FA0FD96EE250DA6EFF0EA1
:10B54000DA22FE0E6F008CFF38F0FF0E6F008CFFCA
:10B5500039F0250E3824E96E000E3920EA6E6F00AE
:10B560007BFFEEFF6F0077FFEDFFFA0EE126FF0E87
:10B57000E2221200E150FC0FD96EE250DA6EFF0EAB
:10B58000DA22FE0E6F008CFF38F0FF0E6F008CFF8A
:10B5900039F00C0E3824E96E000E3920EA6E6F0087
:10B5A0007BFFEEFF6F0077FFEDFFE150FA0FD96EE2
:10B5B000E250DA6EFF0EDA22FE0E6F008CFF38F0DA
:10B5C000FF0E6F008CFF39F00E0E3824E96E000E6E
:10B5D0003920EA6E6F007BFFEEFF6F0077FFEDFF13
:10B5E000FA0EE126FF0EE2221200E150FC0FD96EA6
:10B5F000E250DA6EFF0EDA22FE0E6F008CFF38F09A
:10B60000FF0E6F008CFF39F0100E3824E96E000E2B
:10B610003920EA6E6F007BFFEEFF6F0077FFEDFFD2
:10B62000E150FA0FD96EE250DA6EFF0EDA22FE0E0A
:10B630006F008CFF38F0FF0E6F008CFF39F0120E98
:10B640003824E96E000E3920EA6E6F007BFFEEFFB2
:10B650006F0077FFEDFFFA0EE126FF0EE2221200E7
:10B66000E150FC0FD96EE250DA6EFF0EDA22FE0EC8
:10B670006F008CFF38F0FF0E6F008CFF39F01F0E4B
:10B680003824E96E000E3920EA6E6F007BFFEEFF72
:10B690006F0077FFEDFFE150FA0FD96EE250DA6EDE
:10B6A000FF0EDA22FE0E6F008CFF38F0FF0E6F00E7
:10B6B0008CFF39F0210E3824E96E000E3920EA6E35
:10B6C0006F007BFFEEFF6F0077FFEDFFFA0EE126C4
:10B6D000FF0EE2221200E150FC0FD96EE250DA6E4A
:10B6E000FF0EDA22FE0E6F008CFF38F0FF0E6F00A7
:10B6F0008CFF39F02B0E3824E96E000E3920EA6EEB
:10B700006F007BFFEEFF6F0077FFEDFFE150FA0F58
:10B71000D96EE250DA6EFF0EDA22FE0E6F008CFF59
:10B7200038F0FF0E6F008CFF39F02D0E3824E96ED3
:10B73000000E3920EA6E6F007BFFEEFF6F0077FF8F
:10B74000EDFFFA0EE126FF0EE2221200E150FC0F9F
:10B75000D96EE250DA6EFF0EDA22FE0E6F008CFF19
:10B7600038F0FF0E6F008CFF39F02F0E3824E96E91
:10B77000000E3920EA6E6F007BFFEEFF6F0077FF4F
:10B78000EDFFE150FA0FD96EE250DA6EFF0EDA22C9
:10B79000FE0E6F008CFF38F0FF0E6F008CFF39F04B
:10B7A000310E3824E96E000E3920EA6E6F007BFFFF
:10B7B000EEFF6F0077FFEDFFFA0EE126FF0EE222AB
:10B7C0001200E150F40FD96EE250DA6EFF0EDA2269
:10B7D0006F007BFFE6FF6F007BFFE6FF6F007BFFE4
:10B7E000E6FF6F007BFFE6FF6F007BFFE6FF6F0069
:10B7F0007BFFE6FF6F007BFFE6FF6F007BFFE6FF4E
:10B80000F40E6F008FFFE6FF6F008FFFE6FF690EFB
:10B81000E66E2C0EE66E5F0EE66EF10E6F008FFF89
:10B82000E6FF6F008FFFE6FF01EC4EF0F40EE1261D
:10B83000FF0EE2221200E652E652FC0E6F008CFF71
:10B8400038F0FD0E6F008CFF39F0FF0E6000E7F05E
:10B85000E3FFFE0E6000E3F0E3FF000EE66E000E75
:10B86000E66E000EE66E000EE66E000EE66E000E50
:10B87000E66E000EE66E000EE66E000EE66E000E40
:10B88000E66E720EE66E1A0EE66E680EE66EF10E4B
:10B890006F008FFFE6FF6F008FFFE6FF01EC4EF0B9
:10B8A000E552E552E552E5521200E652E652FC0E30
:10B8B0006F008CFF38F0FD0E6F008CFF39F0FF0E2B
:10B8C0006000E7F0E3FFFE0E6000E3F0E3FF000E30
:10B8D000E66E000EE66E000EE66E000EE66E000EE0
:10B8E000E66E000EE66E000EE66E000EE66E000ED0
:10B8F000E66E000EE66E680EE66E2C0EE66E5F0ECD
:10B90000E66EF10E6F008FFFE6FF6F008FFFE6FF20
:10B9100001EC4EF0E552E552E552E5521200E150DD
:10B92000F40FD96EE250DA6EFF0EDA226F007BFF61
:10B93000E6FF6F007BFFE6FF6F007BFFE6FF6F0017
:10B940007BFFE6FF6F007BFFE6FF6F007BFFE6FFFC
:10B950006F007BFFE6FF6F007BFFE6FFF40E6F00DA
:10B960008FFFE6FF6F008FFFE6FF190EE66E060EF3
:10B97000E66E100EE66EF10E6F008FFFE6FF6F00B1
:10B980008FFFE6FF01EC4EF0F40EE126FF0EE222FF
:10B990001200E150F40FD96EE250DA6EFF0EDA2297
:10B9A0006F007BFFE6FF6F007BFFE6FF6F007BFF12
:10B9B000E6FF6F007BFFE6FF6F007BFFE6FF6F0097
:10B9C0007BFFE6FF6F007BFFE6FF6F007BFFE6FF7C
:10B9D000F40E6F008FFFE6FF6F008FFFE6FF1A0E79
:10B9E000E66E060EE66E100EE66EF10E6F008FFF2D
:10B9F000E6FF6F008FFFE6FF01EC4EF0F40EE1264C
:10BA0000FF0EE2221200E150F40FD96EE250DA6E1E
:10BA1000FF0EDA226F007BFFE6FF6F007BFFE6FF81
:10BA20006F007BFFE6FF6F007BFFE6FF6F007BFF91
:10BA3000E6FF6F007BFFE6FF6F007BFFE6FF6F0016
:10BA40007BFFE6FFF40E6F008FFFE6FF6F008FFFB6
:10BA5000E6FF170EE66E060EE66E100EE66EF10EAF
:10BA60006F008FFFE6FF6F008FFFE6FF01EC4EF0E7
:10BA7000F40EE126FF0EE2221200E150F40FD96E1F
:10BA8000E250DA6EFF0EDA226F007BFFE6FF6F00F6
:10BA90007BFFE6FF6F007BFFE6FF6F007BFFE6FFAB
:10BAA0006F007BFFE6FF6F007BFFE6FF6F007BFF11
:10BAB000E6FF6F007BFFE6FFF40E6F008FFFE6FFEF
:10BAC0006F008FFFE6FF160EE66E060EE66E100E96
:10BAD000E66EF10E6F008FFFE6FF6F008FFFE6FF4F
:10BAE00001EC4EF0F40EE126FF0EE2221200E652C7
:10BAF000E652FC0E6F008CFF38F0FD0E6F008CFFDD
:10BB000039F0FF0E6000E7F0E3FFFE0E6000E3F0A7
:10BB1000E3FF000EE66E000EE66E000EE66E000E0F
:10BB2000E66E000EE66E000EE66E000EE66E000E8D
:10BB3000E66E000EE66E000EE66E700EE66E1A0EF3
:10BB4000E66E680EE66EF10E6F008FFFE6FF6F0087
:10BB50008FFFE6FF01EC4EF0E552E552E552E5526B
:10BB60001200E652E652FC0E6F008CFF38F0FD0E1C
:10BB70006F008CFF39F0FF0E6000E7F0E3FFFE0E70
:10BB80006000E3F0E3FF000EE66E000EE66E000ECE
:10BB9000E66E000EE66E000EE66E000EE66E000E1D
:10BBA000E66E000EE66E000EE66E000EE66E6F0E9E
:10BBB000E66E1A0EE66E680EE66EF10E6F008FFFEF
:10BBC000E6FF6F008FFFE6FF01EC4EF0E552E55215
:10BBD000E552E5521200E652E652FC0E6F008CFF71
:10BBE00038F0FD0E6F008CFF39F0FF0E6000E7F0BB
:10BBF000E3FFFE0E6000E3F0E3FF000EE66E000ED2
:10BC0000E66E000EE66E000EE66E000EE66E000EAC
:10BC1000E66E000EE66E000EE66E000EE66E000E9C
:10BC2000E66E670EE66E2C0EE66E5F0EE66EF10EA9
:10BC30006F008FFFE6FF6F008FFFE6FF01EC4EF015
:10BC4000E552E552E552E5521200E652E652FC0E8C
:10BC50006F008CFF38F0FD0E6F008CFF39F0FF0E87
:10BC60006000E7F0E3FFFE0E6000E3F0E3FF000E8C
:10BC7000E66E000EE66E000EE66E000EE66E000E3C
:10BC8000E66E000EE66E000EE66E000EE66E000E2C
:10BC9000E66E000EE66E660EE66E2C0EE66E5F0E2B
:10BCA000E66EF10E6F008FFFE6FF6F008FFFE6FF7D
:10BCB00001EC4EF0E552E552E552E5521200E65233
:10BCC000E652FC0E6F008CFF38F0FD0E6F008CFF0B
:10BCD00039F0FF0E6000E7F0E3FFFE0E6000E3F0D6
:10BCE000E3FF000EE66E000EE66E000EE66E000E3E
:10BCF000E66E000EE66E000EE66E000EE66E000EBC
:10BD0000E66E000EE66E000EE66E650EE66E2C0E1A
:10BD1000E66E5F0EE66EF10E6F008FFFE6FF6F00BE
:10BD20008FFFE6FF01EC4EF0E552E552E552E55299
:10BD30001200E652E652FC0E6F008CFF38F0FD0E4A
:10BD40006F008CFF39F0FF0E6000E7F0E3FFFE0E9E
:10BD50006000E3F0E3FF000EE66E000EE66E000EFC
:10BD6000E66E000EE66E000EE66E000EE66E000E4B
:10BD7000E66E000EE66E000EE66E000EE66E710ECA
:10BD8000E66E1A0EE66E680EE66EF10E6F008FFF1D
:10BD9000E6FF6F008FFFE6FF01EC4EF0E552E55243
:10BDA000E552E5521200E150F40FD96EE250DA6E1E
:10BDB000FF0EDA226F007BFFE6FF6F007BFFE6FFDE
:10BDC0006F007BFFE6FF6F007BFFE6FF6F007BFFEE
:10BDD000E6FF6F007BFFE6FF6F007BFFE6FF6F0073
:10BDE0007BFFE6FFF40E6F008FFFE6FF6F008FFF13
:10BDF000E6FF180EE66E060EE66E100EE66EF10E0B
:10BE00006F008FFFE6FF6F008FFFE6FF01EC4EF043
:10BE1000F40EE126FF0EE2221200FE0EE350020FA6
:10BE2000386EFF0E6F008CFF39F0000E3922600073
:10BE3000E3F0E6FF6000E7F0E6FFC4EC60F0000E20
:10BE4000E66E000EE66E000EE66E000EE66E000E6A
:10BE5000E66E000EE66E000EE66E000EE66E0A0E50
:10BE6000E66E000EE66E140EE66E060EE66E100E20
:10BE7000E66EF10E6F008FFFE6FF6F008FFFE6FFAB
:10BE800001EC4EF0E552E5521200FE0EE350020FB7
:10BE9000386EFF0E6F008CFF39F0000E3922600003
:10BEA000E3F0E6FF6000E7F0E6FFC4EC60F0000EB0
:10BEB000E66E000EE66E000EE66E000EE66E000EFA
:10BEC000E66E000EE66E000EE66E000EE66E0A0EE0
:10BED000E66E000EE66E150EE66E060EE66E100EAF
:10BEE000E66EF10E6F008FFFE6FF6F008FFFE6FF3B
:10BEF00001EC4EF0E552E552120000EEF8F220EEB1
:10BF0000D7F2EE6ADD50D950FCE1DA50FAE100EEEA
:10BF100000F2F80EEE6AE806FDE100EE00F1650EB3
:10BF2000EE6AE806FDE100EE60F0760EEE6AE806E5
:10BF3000FDE100EE01F02D0EEE6AE806FDE1080ECF
:10BF4000D56E000ED66E000ED76E000184EF62F043
:10BF5000000EE66E000EE66E000EE66E000EE66E59
:10BF6000000EE66E000EE66E000EE66E000EE66E49
:10BF7000F40E6F008FFFE6FF6F008FFFE6FFCB0E22
:10BF8000E66EBE0EE66E520EE66EF10E6F008FFF8D
:10BF9000E6FF6F008FFFE6FF01EC4EF0E552E55241
:10BFA000E552E5521200000EE66E000EE66E000E3F
:10BFB000E66E000EE66E000EE66E000EE66E000EF9
:10BFC000E66E000EE66EF40E6F008FFFE6FF6F0068
:10BFD0008FFFE6FFC90EE66EBE0EE66E520EE66EEF
:10BFE000F10E6F008FFFE6FF6F008FFFE6FF01ECA1
:10BFF0004EF0E552E552E552E5521200FE0EE350D6
:10C000001E0F386EFF0E6F008CFF39F0000E3922C4
:10C010006000E3F0F6FF6000E7F0F7FF000EF86E57
:10C02000FD0EE350396E0F0EF76405D06000E7F0A7
:10C03000F5FF0C0009D06F00DBFFE9FF6F00DFFFA9
:10C04000EAFF6000E7F0EFFFE552E552E55212002B
:10C05000FE0EE350E66EC2EC63F0FF0EE350110DEE
:10C06000F80EF324D96E020EF420DA6EDE6ADD6A71
:10C07000FF0EE350110DFA0EF324386E020EF42079
:10C08000396E6000E3F0E6FF6000E7F0E6FFC7EC22
:10C0900058F0FE0EE350E66EB6EC63F0E552E55262
:10C0A0001200E652E652E652E652FC0EE36AFF0E3A
:10C0B000E124D96EFF0EE220DA6E600057F0DFFF58
:10C0C000FC0E6F008FFFE6FF6F008FFFE6FF6F0033
:10C0D0008FFFE6FF6F008FFFE6FF000EE66E030E98
:10C0E000E66E48EC3BF0FA0EE126FF0EE22212006B
:10C0F000000EE66E000EE66E000EE66E000EE66EB8
:10C10000000EE66E000EE66E000EE66E000EE66EA7
:10C11000B80EE66E0B0EE66E6E0EE66E1A0EE66E4C
:10C12000680EE66EF10E6F008FFFE6FF6F008FFF67
:10C13000E6FF01EC4EF0E552E5521200000EE66E0D
:10C14000000EE66E000EE66E000EE66E000EE66E67
:10C15000000EE66E000EE66E000EE66EB80EE66E9F
:10C160000B0EE66E640EE66E2C0EE66E5F0EE66E4D
:10C17000F10E6F008FFFE6FF6F008FFFE6FF01EC0F
:10C180004EF0E552E5521200000EE66E000EE66E2D
:10C19000000EE66E000EE66E000EE66E000EE66E17
:10C1A000000EE66E000EE66E000EE66E000EE66E07
:10C1B000C80EE66EBE0EE66E520EE66EF10E6F0013
:10C1C0008FFFE6FF6F008FFFE6FF01EC4EF0E552B8
:10C1D000E5521200FE0EE350070F386EFF0E6F009F
:10C1E0008CFF39F0000E39226000E3F0F6FF6000AA
:10C1F000E7F0F7FF000EF86E0F0EF76404D0000EA4
:10C20000F56E0C0008D06F00DBFFE9FF6F00DFFF69
:10C21000EAFF000EEF6EE552E5521200E652E150E1
:10C22000FD0FD96EE250DA6EFF0EDA226F007BFF4F
:10C23000F6FF6F0077FFF7FFF86A0800FF0E6F0048
:10C24000D7FFE3FFFF0EE350E66E040EE66E000E2E
:10C25000E66EA1EC41F0E552E552E5521200BA6AF1
:10C26000BB6ABC6AC26AF60EC36EC4683A016069F2
:10C27000EE0E506F406B816B516B800E416F616BA6
:10C28000426B526B626B43695369636944695469D9
:10C290006469080E846F0C0EED6F330E0B6F120085
:10C2A000000EE66E000EE66E000EE66E000EE66E06
:10C2B000000EE66E000EE66E000EE66E000EE66EF6
:10C2C000000EE66E000EE66E0A0EE66E9E0EE66E3E
:10C2D000350EE66E2A0EE66E000EE66E01EC4EF0AE
:10C2E0001200E652E652FC0E6F008CFF38F0FD0E95
:10C2F0006F008CFF39F0FF0E6000E7F0E3FFFE0EE9
:10C300006000E3F0E3FFFE0E6F008FFFE6FF6F00BB
:10C310008FFFE6FF99EC5EF0E552E552E552E552FB
:10C320001200E150FC0FD96EE250DA6EFF0EDA22F5
:10C33000FE0E6F008CFF38F0FF0E6F008CFF39F09F
:10C34000050E3824E96E000E3920EA6E6F007BFF7F
:10C35000EEFF6F0077FFEDFFE552E552E552E55243
:10C360001200E150FC0FD96EE250DA6EFF0EDA22B5
:10C37000FE0E6F008CFF38F0FF0E6F008CFF39F05F
:10C38000030E3824E96E000E3920EA6E6F007BFF41
:10C39000EEFF6F0077FFEDFFE552E552E552E55203
:10C3A0001200E150FC0FD96EE250DA6EFF0EDA2275
:10C3B000FE0E6F008CFF38F0FF0E6F008CFF39F01F
:10C3C000010E3824E96E000E3920EA6E6F007BFF03
:10C3D000EEFF6F0077FFEDFFE552E552E552E552C3
:10C3E0001200E150FC0FD96EE250DA6EFF0EDA2235
:10C3F000FE0E6F008CFF38F0FF0E6F008CFF39F0DF
:10C40000010E3824E96E000E3920EA6E6F007BFFC2
:10C41000EEFF6F0077FFEDFFE552E552E552E55282
:10C420001200E150FC0FD96EE250DA6EFF0EDA22F4
:10C43000FE0E6F008CFF38F0FF0E6F008CFF39F09E
:10C44000030E3824E96E000E3920EA6E6F007BFF80
:10C45000EEFF6F0077FFEDFFE552E552E552E55242
:10C460001200060EE126000EE222F80E6F008CFF8D
:10C4700038F0F90E6F008CFF39F0070E3824D96EB2
:10C48000000E3920DA6E080E2E6EF80E6F007BFF5C
:10C49000E3FFE8282E2EFAD71200FE0E6F008CFF65
:10C4A00038F0FF0E6F008CFF39F0070E3824D96E7C
:10C4B000000E3920DA6E070E2E6EF60E6F008FFF1B
:10C4C000DEFFE82A2E06FAE2F60EE126FF0EE22251
:10C4D0001200E652D2BE6FEF62F073EF62F0396A7B
:10C4E000392A74EF62F0396AFF0E6000E7F0E3FF6B
:10C4F000D29E39015B510400FF0EE3B002D0D29E00
:10C5000001D0D28EE552120055EC63F08AEC4CF06B
:10C510003CEC56F078EC58F09CEC63F01E0EE66EA6
:10C52000A50EE66EDAEC63F0D28E69EC62F0ABEC4D
:10C5300056F095EF62F00DEF00F0FF0EE124D96E9A
:10C54000FF0EE220DA6EDF50030B3901E16FFE0EC1
:10C550006F008FFFE0F93F0EE517E58100F000F076
:10C560006E008CF72EF0E552E55212003901A39FC0
:10C570000001D651D711D8B4C0EF62F0C2EF62F01B
:10C58000CEEF62F002D8CEEF62F00500FA6ED6511F
:10C59000FD6ED751FE6EFF6AFA5012001200FE0EB9
:10C5A0006F008CFF38F0FF0E6F008CFF39F0030E28
:10C5B0003824D96E000E3920DA6E6F0078FF2EF025
:10C5C0006F0074FF2FF0E552E5521200FE0E6F006F
:10C5D0008CFF38F0FF0E6F008CFF39F0050E382409
:10C5E000D96E000E3920DA6E6F0078FF2EF06F00E2
:10C5F00074FF2FF0E552E5521200FE0E6F008CFF23
:10C6000038F0FF0E6F008CFF39F01A0E3824D96E07
:10C61000000E3920DA6EFD0E6F008FFFDFFFE5524E
:10C62000E552E5521200000EE66E000EE66E000EB8
:10C63000E66E000EE66E0F0EE66E000EE66E48EC3D
:10C640003BF0E552E5521200460EB96EF90EB76E98
:10C65000B66A3901A39F938F4C0EE66EC90EE66E43
:10C66000DAEC63F0890EB86E1200FE0E6F008FFFD9
:10C67000D9FFFF0E6F008FFFDAFFFD0E6F008FFFF7
:10C68000DFFFE552E552E5521200FE0E6F008FFF0C
:10C69000D9FFFF0E6F008FFFDAFFFD0E6F008FFFD7
:10C6A000DFFFE552E552E5521200A4EC64F03DECE8
:10C6B00064F02FEC61F047EC64F08DEC64F024EC56
:10C6C00063F017EC4AF0120002D870EF63F0050037
:10C6D000FA6E2850FD6E2950FE6EFF6AFA50120065
:10C6E0003901A5931200010EE66EFD0E6F008FFF5B
:10C6F000E6FF6F008FFFE6FFFDEC62F0E552E552CA
:10C7000012000001C96BCA6BCBC0CFF0CCC0D0F017
:10C71000CDC0D1F0CEC0D2F0E552E5521200FE0EEF
:10C720006F008FFFD9FFFF0E6F008FFFDAFFDF5022
:10C730002E6EE552E552120050EC61F07DEC64F093
:10C740006000BBF0E6FF6000BFF0E6FF45EC5FF085
:10C750001200FE0EE350E66EFE0EE350E66E000E93
:10C76000E66E91EC59F0E552E5521200FF0EE350EF
:10C77000D8A4BDEF63F0BFEF63F0C0EF63F0D28EDB
:10C78000E5521200FF0EE350D8A4C9EF63F0CBEFDF
:10C7900063F0CCEF63F0D29EE5521200FE0E6F0004
:10C7A0008FFFE6FF6F008FFFE6FFE7EC54F0E552E6
:10C7B000E5521200FE0E6F008CFFD6F0FF0E6F00E8
:10C7C0008CFFD7F0E552E5521200FE0E6F008CFF91
:10C7D000C7F0FF0E6F008CFFC8F0E552E552120063
:10C7E000FE0E6F008CFF22F0FF0E6F008CFF23F017
:10C7F000E552E5521200FE0E6F008CFFC5F0FF0EF1
:10C800006F008CFFC6F0E552E5521200FE0E6F007D
:10C810008CFF20F0FF0E6F008CFF21F0E552E552F7
:10C820001200FE0E6F008CFF26F0FF0E6F008CFFD3
:10C8300027F0E552E5521200FE0E6F008CFF24F047
:10C84000FF0E6F008CFF25F0E552E5521200FE0E40
:10C850006F008CFF28F0FF0E6F008CFF29F0E5526F
:10C86000E5521200FE0E6F008CFF2CF0FF0E6F00E1
:10C870008CFF2DF0E552E55212003901C06BC16BFF
:10C88000C26BC36BC46BC56BC66BC76B1200600E0B
:10C890003901D96FDB6BDD6B080EDF6FDE6B1200C9
:10C8A000000E2E6E020E2F6EB40E2E26000E2F22BC
:10C8B0001200000E2E6E020E2F6E010E2E26000E9E
:10C8C0002F221200000E2E6E020E2F6E700E2E26DC
:10C8D000000E2F221200FF0EE350E66E000EE66EF1
:10C8E0009DEC62F0E5521200000E2E6E020E2F6ECD
:10C8F000390E2E26000E2F221200000E2E6E020E72
:10C900002F6E020E2E26000E2F221200000EE66E53
:10C91000000EE66EA9EC63F012000C0E39015B6F9D
:10C92000370E5C6F1200FF0E6F008CFF2BF0E5528C
:10C9300012000A0E2A6E2C6A2D6A2B6A1200000E53
:10C940002E6E020E2F6E1200D29A120012001200EA
:0CC950001200120012001200120012006F
:020000040020DA
:10000000FFFFFFFFFFFFFFFFFFFFFFFFFFFFFFFF00
:020000040030CA
:0A0000008CFFF7FFA6FFFFFFFFFFD4
:00000001FF
